:020000040000fa
:080000000002040000000000f2
:020000040000fa
:100008000806000008060000900200009a0200009e
:1000180008060000080600000806000008060000a0
:100028000806000008060000080600001e1101006e
:100038000806000008060000080600000806000080
:100048000806000008060000080600000806000070
:100058000806000008060000080600000806000060
:100068000806000008060000080600000806000050
:100078000806000008060000080600000806000040
:100088000806000008060000080600000806000030
:1000980008060000080600002402010066020100ac
:1000a8000806000008060000080600000806000010
:1000b8000806000008060000080600000806000000
:1000c80008060000080600000806000008060000f0
:1000d80008060000080600000806000008060000e0
:1000e80008060000080600000806000008060000d0
:1000f80008060000080600000806000008060000c0
:1001080008060000080600000806000008060000af
:10011800080600000806000008060000080600009f
:10012800080600000806000008060000080600008f
:10013800080600000806000008060000080600007f
:10014800080600000806000008060000080600006f
:10015800080600000806000008060000080600005f
:10016800080600000806000008060000080600004f
:10017800080600000806000008060000080600003f
:10018800080600000806000008060000080600002f
:10019800080600000806000008060000080600001f
:1001a800080600000806000008060000080600000f
:1001b80008060000080600000806000008060000ff
:1001c80008060000080600000806000008060000ef
:1001d80008060000080600000806000008060000df
:1001e80008060000080600000806000008060000cf
:0801f8000806000008060000e3
:020000040000fa
:100208000806000008060000900200009a0200009c
:10021800080600000806000008060000080600009e
:100228000806000008060000080600001e1101006c
:10023800080600000806000008060000080600007e
:10024800080600000806000008060000080600006e
:10025800080600000806000008060000080600005e
:10026800080600000806000008060000080600004e
:10027800080600000806000008060000080600003e
:10028800080600000806000008060000080600002e
:1002980008060000080600002402010066020100aa
:1002a800080600000806000008060000080600000e
:1002b80008060000080600000806000008060000fe
:1002c80008060000080600000806000008060000ee
:1002d80008060000080600000806000008060000de
:1002e80008060000080600000806000008060000ce
:1002f80008060000080600000806000008060000be
:1003080008060000080600000806000008060000ad
:10031800080600000806000008060000080600009d
:10032800080600000806000008060000080600008d
:10033800080600000806000008060000080600007d
:10034800080600000806000008060000080600006d
:10035800080600000806000008060000080600005d
:10036800080600000806000008060000080600004d
:10037800080600000806000008060000080600003d
:10038800080600000806000008060000080600002d
:10039800080600000806000008060000080600001d
:1003a800080600000806000008060000080600000d
:1003b80008060000080600000806000008060000fd
:1003c80008060000080600000806000008060000ed
:1003d80008060000080600000806000008060000dd
:1003e80008060000080600000806000008060000cd
:0803f8000806000008060000e1
:020000040000fa
:100400000ffd20000e7f22000e018800000000007a
:100410000c000700802920001100200011000700b7
:10042000000020000000e000020032000000020096
:1004300000000000a4020200000000000040da00fa
:100440000000fe004440a900804721000000e000b9
:100450000300320000002000a00188004440a800f2
:100460000000060091018800800078000000eb0089
:1004700015003700e280400032a0b4009101ba00bc
:10048000e280400032a0b4009102ba00e280400055
:1004900032a0b4000002eb00472bde00f507b200eb
:1004a000602ce10004003a000059eb008301e900f0
:1004b000fdff3e00040037006128e100010032002a
:1004c0000082eb00040007001101ba000200e00006
:1004d000e8ff3a00000006003159ba008301e90044
:1004e0000c0032002159ba008301e90008003200f3
:1004f0000400e00003003a00e280400032a0b400b3
:10050000f5ff370011d9ba008301e900faff3a007c
:100510008100e800e180400032a0b4000000060045
:100520000000fa0000000000000000000080fa0057
:10053000004006000000fa0000000000000000007b
:100540000080fa00004006000400fa0005010700e0
:10055000be04020001000000400620005214020008
:100560000100000020e920001202200041cd2900f6
:10057000940a0200000000004c0502000100000087
:100580001a10020001000000b89e020000000000e6
:1005900020010700a116800000002200808060007a
:1005a0000000eb00808f500041003a009a100200da
:1005b00001000000008fbe00412c20000040eb0035
:1005c00080487800320037009a10020001000000d5
:1005d0003e015000ae81580000092d00310020007e
:1005e000800f5100818f5900290036006000b8004b
:1005f000a4ed02000000000000c0eb00b8ed020016
:100600000000000000c0eb00b8ed02000000000098
:1006100028ee02000000000050cf2900ec09020083
:1006200001000000412c2000f0c0b3008048780099
:10063000000000009a100200010000003e0150007e
:10064000ae8158000200be000001be0020aa2400b6
:1006500041002000800f5100818f5900f5ff3400c8
:10066000412c20000040eb00804878000000000092
:10067000a116800000002200808060000000eb00d6
:10068000808f5000faff32000000fe0006003700a5
:10069000a116800000002200808060000000eb00b6
:1006a000808f5000c8ff320020e8020000000000e8
:1006b000b0f6020000000000a600020001000000e9
:1006c00001003700000000009a1002000100000045
:1006d0000001be00706b8000816b80000001510042
:1006e0008181590010a1270001002000800f5100d6
:1006f000818f5900100036009a100200010000009e
:10070000706b8800816b88002016800000407800a4
:10071000614060000004a200614060000080fb00b6
:100720006100600022168000e1ff2f00810061005f
:10073000008070002016880006f70200000000000c
:1007400078f9020000000000140b02000100000014
:100750005812020001000000f40e02000100000027
:100760005813020001000000880c02000100000084
:10077000be0d02000100000040fc0200000000006d
:10078000710007008069800091698000926b800091
:10079000a36b8000820f5000838f5800c9ff320086
:1007a0008069800091698000906b8800a16b88004f
:1007b000f0d32900ec0902000100000080698000ec
:1007c000916980000600070020d52900ec0902008d
:1007d00001000000ec07020001000000baff370032
:1007e0000c00fa00881f7800400798005107980015
:1007f00000c1b300204798000040eb00004f780094
:100800003c0037009e4078000180fb00e800470074
:1008100000804000104078000080fb00e3004700ab
:10082000f0af02000000000063004700ec09020086
:10083000010000000040eb00104798000f00370057
:100840002e4090000081fb001e4090000080fb00c5
:10085000e30047006140780021e920008100410069
:10086000804878002e4090000040e8002047980023
:100870001e4090000040e800104798001e40900085
:100880000084fb0063004700de0a02000000000055
:10089000800f5400eaff39009e40780030c0b3005a
:1008a00080cf5000180032002e4090008080fb0066
:1008b00020e9200080804000e0c2b300804878003a
:1008c0002e4090000040e800204798000000000003
:1008d000c60a0200010000008040eb00814f50007a
:1008e000fbff3a00e0022000f60a020001000000cf
:1008f0001e4fe8009e40780030c0b30080cf50000b
:10090000c0ff36000100370000000000ae4090003c
:10091000f0c1b30080cf500006003e002e40900092
:100920008080fb0020e92000808040000040eb0038
:10093000804878004c050200010000004f04780058
:100940000080fa00000006000000fa000018800095
:1009500061d62000f0af0200000000000080fa0025
:10096000000006000000fa00c002a900c022a90091
:10097000c042a900c062a900c082a900c0a2a9000b
:10098000c0c2a900c4e2a900412c20000040eb0035
:1009900080487800213a8000f08f2f0000806000ae
:1009a000203a88000000eb00401988002c83a90041
:1009b0002ca3a900404e28000019880040402000c8
:1009c0001019880030002100201988000002200042
:1009d00080198800dea2a900de82a800000028009d
:1009e0008011880000402000901188003003200012
:1009f000c0118800d7c2a800d3c2a900d782a8001e
:100a0000d382a9003aec0200000000000080fa0046
:100a1000000006000800fa00881f78000040eb0084
:100a2000004f7800320320008000eb0000d320004c
:100a3000a20a0200000000005ccda8005ceda80046
:100a40006200200051d52900d0d52000940a020070
:100a50000000000090ea2f0011102000806988003b
:100a6000916988008069800091698000206a88000f
:100a7000316a8800f0ff2f0001002000a069880083
:100a8000b1698800a0698000b1698000406a88006f
:100a9000516a880090ea2f0011102000c069880078
:100aa000d169880090ea2f0011102000e0698800c9
:100ab000f16988006000b800006a8800116a880047
:100ac00002012000b1d52900c0d42000940a020000
:100ad00000000000c0d42000f0b2020000000000be
:100ae0003103200000d3200032b2020000000000d9
:100af000206b88009e4078000040eb0080cf5000c3
:100b00000200320000d32000290007000e80e80018
:100b100063002000000178006000b800b6ec02001d
:100b2000000000003303200002d3200060002000fa
:100b300001002000b6ec0200000000000e80e8007a
:100b40009000780030032000808f50000d003a00a4
:100b50000e80e80090009000206b8000808f500095
:100b600008003a000e80e8002004900031032000c5
:100b700000d3200032b2020000000000800f5400b9
:100b8000080032009e4078000040eb0080cf50000b
:100b900001003200ffff370010c0b300004f7800a3
:100ba000a0ff37004f0478000080fa000000060024
:100bb0000800fa0030079800206b800010079800aa
:100bc0003e0090003103200032b20200000000001d
:100bd0002007980030032000000f78006000b80064
:100be000a4ed0200000000000e007800610020006b
:100bf000faed0200000000003e00900031032000ea
:100c0000faed0200000000000080fa00000006007b
:100c10000040da000000fe00680107000400be008a
:100c2000000006000800fa00889fbe008a9fbe00f0
:100c300084bf9f0095bf9f00a6bf9f00b7bf9f00c6
:100c40003004be002005be000fba97009fba97007f
:100c50002fbb9700bfbb97000404440085844c0061
:100c600006054d0087854d000898be000a90be001d
:100c70000440e10005c8e10006d0e10007d8e1002a
:100c800002003100680040001008e8004f05be0077
:100c90004f04be000080fa0000000600fe874700f7
:100ca000889fbe008a9fbe008c9fbe008e1f78006a
:100cb000d0b79f00e1b79f00f2b79f0083bf9f00ae
:100cc00084b79f0095b79f00a6b79f00b7b79f0056
:100cd0008000eb00f1af9f00e1af9f00d1af9f001c
:100ce000c1af9f00b1af9f00010678000d04200046
:100cf000ccb79f000605be000404be007fae97007f
:100d00006faf97005fa89700e00f56000f003d00ff
:100d1000cf71de000c01460002817100f2af9f002e
:100d20005d0007004f20de008180400081007000e0
:100d3000640007000802be000a03be0060fd2f0029
:100d40000f004000b7ff07001d00370052000700ea
:100d50004f21de00818040008100710059000700b2
:100d60003faa9700cfaa97005fab9700efab970021
:100d70000800520089805a000a015b008b815b00e9
:100d8000b0af9f00c1af9f00d2af9f00e3af9f0005
:100d90004f70de000c0146000200700013002000be
:100da0000820e10009a8e1000ab0e1000bb8e10069
:100db000010039008001eb0003005000f0af9f00fc
:100dc0007fae9700e00f56000f00350010002000a6
:100dd000010020006011b8005fb29700efb29700e9
:100de0007fb397008fbb970004027000858270006c
:100df0000603710087837100d4b79f00e5b79f0099
:100e0000f6b79f0087bf9f00cfb297008502e8002a
:100e1000c5b79f008d8f5200b8ff3a000c017800d3
:100e2000e00f510007003d000fb297009fb29700fe
:100e30002fb39700bfb3970060fd2f000f00400055
:100e400078ff0700ffa09700e08f500008003a00ed
:100e50003fac9700cfac97005fad9700efad970028
:100e6000d8b79f00e9b79f00fab79f008bbf9f00dc
:100e70005fb09700efb097007fb197008fb99700f0
:100e80004f0778004f06be004f05be004f04be005e
:100e9000ef01b100000006004f01de008e004700a8
:100ea00081007100c1af9f00afa897004f09de001d
:100eb0000000400000007100b0af9f001faa970023
:100ec00000000600a1af9f000e0007004f18de00d3
:100ed000040242000002720094af9f000900070064
:100ee00000004000818048000201490083814900e0
:100ef000b0b79f00c1b79f00d2b79f00e3b79f0074
:100f0000000006001fb09700afb097003fb19700f8
:100f1000cfb1970000000600881f7800180020005d
:100f2000881f78005dff07008f87e9004f04780075
:100f300000000600801feb0058ff07008f87e900c4
:100f400000000600889fbe008a9fbe008c1f7800ac
:100f50006044b8006055b8000800e1000988e1006d
:100f60000a90e1000b98e1000d003d0000005400e4
:100f700081805c0002015d0083815d001c00200017
:100f80000820e10009a8e1000ab0e1000bb8e10087
:100f90000b003d00210007000006eb0008003700b1
:100fa0000006eb00e00f5200e08f5a00e00f5b00fc
:100fb000e08f5b0002003d00180007001c002000cd
:100fc000d5ff0700800578000105780082047800cd
:100fd000030478000b0278008a0278000903780085
:100fe00088037800e00f5600060032006000b80069
:100ff0006011b800040250008582580006035900b1
:10100000878359000400be000601be004f06780029
:101010004f05be004f04be0000000600040254004d
:1010200085825c0006035d0087835d00000006008a
:10103000889fbe008a9fbe008c1f78006044b80065
:101040006055b8000800e1000988e1000a90e1005d
:101050000b98e1000b003d000000540081805c0013
:1010600002015d0083815d001c0020000820e1007a
:1010700009a8e1000ab0e1000bb8e1000b003d0057
:10108000060037000006eb00e00f5200e08f5a0028
:10109000e00f5b00e08f5b0004003d0004025400a1
:1010a00085825c0006035d0087835d00a1ff070069
:1010b0008005780001057800820478000304780038
:1010c0000b0278008a027800090378008803780010
:1010d000e00f5600060032006000b8006011b80052
:1010e0000402500085825800060359008783590086
:1010f0000400be000601be004f0678004f05be008a
:101100004f04be0000000600889fbe008a9fbe00fc
:101110008c1f78000006eb00e00f5000e08f5800b5
:10112000e00f5900e08f590007003d006044b8000f
:101130006055b8000000540081805c0002015d0031
:1011400083815d001c002000e00f5200e08f5a00f8
:10115000e00f5b00e08f5b0007003d006044b800db
:101160006055b8000402540085825c0006035d00ef
:1011700087835d000c00a200200007000203be0070
:101180000002be00e00f5600060032006000b8000a
:101190006011b8000402500085825800060359000f
:1011a000878359000400be000601be004f06780088
:1011b0004f05be004f04be00000006006022b800cc
:1011c000060220000000d0008180d2000482d200fc
:1011d0008582d2000000a0000202520083825a00e1
:1011e000030031000202420083824a000000a10095
:1011f0000603e900f3ff3a0000000600889fbe00e6
:101200008a9fbe008c9fbe000404b8000506b8008b
:101210008904460060854e000606b8000a054600af
:10122000e0854e000706b8008b054600040eb800a6
:10123000890446000a854e00e0854d00050eb80081
:101240000a0546008b854e00060eb8008b05460049
:101250000416b8000a0546008b854e000516b80036
:101260008b054600041eb8008b0546000800be0032
:101270000a01be004f06be004f05be004f04be006f
:101280000000060003c2b3000001780002007800ed
:10129000b040780083cf5000fbff3200e9cf500010
:1012a000f9ff3200d3c2b30083cf500003003a00ed
:1012b0000001780013c0b300050037008041eb0047
:1012c000b4c2b30084cf500001003a00000178009e
:1012d0000000eb00020037006a00b9000000420085
:1012e0003202fb000403b100e90f5200faff36009e
:1012f000e0cf5100010032000000ea0000000600cb
:10130000889fbe008a9fbe0001c2b30030447800af
:1013100080047800814f5400fcff3200e94f5400f4
:10132000faff3200d0c2b300804f540003003a00ed
:10133000394478001ac0b300050037000045eb00bf
:10134000b0c2b300804f540001003a003944780025
:101350006022b8000bcdb3000b003700a2002000c4
:10136000030020000400be00d40007000001be00fe
:101370000b4244000482fb000500200004024100ef
:1013800085824900394478000880fb000003b100e1
:10139000e90f5000f1ff3600e04f55000200320027
:1013a00060021200e0821a000400be004f05be0079
:1013b0004f04be0000000600889fbe008a9fbe004a
:1013c0008c9fbe00800678008205780003067800b6
:1013d000010478000b0078008c007800cfc4de0098
:1013e00001003700820678000801be0073ff070085
:1013f0008001780001017800030078008200780005
:101400000d01e800e00f5000e08f5800f5ff3a00b2
:101410000049eb000801be000b0078008c0078004a
:10142000fdfd0700004578000801be000b007800b4
:101430008c00780061ff07000002be000403be00bc
:101440008605780007067800e94f55000100340052
:101450006745450000c3b30080564500e00f5200c9
:10146000e08f5a00ebff3a000d0078004f06be00f7
:101470004f05be004f04be0000000600881f780024
:1014800000047800e00f5100e08f590006003d0095
:1014900008027800d0c2b300005a78006001110041
:1014a000e08119000100370008027800040078008c
:1014b000c1ff0700080078004f0478000000060014
:1014c000e68747008e1f7800d0bf9f0066875700d1
:1014d000012f78000e0037005fba970014407800a3
:1014e000efb99700934078000201e900814f500066
:1014f000040032000080fb008180fb0001005000ee
:10150000060037000402e800d4bf9f00030fe80084
:10151000e00f5100f0ff3a00020078004f0778001a
:101520006f00b10000000600800178000200370063
:10153000b15978000201e900e00f5100fcff3a00c8
:101540000000060080017800020037008159780011
:101550000201e900e00f5100fcff3a000000060024
:10156000000178000200780000017800b2417800a4
:1015700081cf510003003200e0cf5100f9ff3a0063
:101580000000eb0000000600b041780031c15100be
:1015900002003a0082cf5100fbff3a000200fb003c
:1015a00000000600800178003141780082597800ff
:1015b000e04f5100fcff3a00000006008000780078
:1015c0000041eb00b14f1100fdff3a000080ea003e
:1015d000008040000000060080017800060037000f
:1015e0000201e900b14278008559780003027800d1
:1015f000e0cf52000600320003027800e00f5100f5
:10160000f7ff3a0002003700005aeb000201e90040
:10161000e00f5100fcff3a0000000600889fbe006a
:101620000004be000b00370009007800e3ff07004c
:10163000000178000800be000f000700e00f500016
:101640000a0032000800e8009900fb00c4ff070010
:1016500000047800e00f5400040032000040eb006a
:10166000984f1000f0ff3a000004eb0008007800eb
:101670004f04be00000006000b003700b0417800a8
:10168000e0cf5100030032000201e900b1cf510068
:10169000050032008381fb00144278000480fb00c7
:1016a000008051000000060001027800e00f5100a8
:1016b000f2ff3a000200780000000600020ab900ba
:1016c000001bb9000200b800810042008100430005
:0416d0000000060010
:020000040000fa
:1016d400666f00006f740000657200002e690000e0
:1016e4006e6300000068000065610000646500002e
:1016f400722e0000696e00006300000021440000a7
:1017040045460000000d00000a0000007478000047
:1017140074000000687400006d000000687400002c
:101724006d6c000000630000676900000078000031
:101734006d6c00000063000073730000006700001c
:1017440069660000007000006e670000006a000017
:1017540070670000006300006c6100000077000007
:10176400617600000000000000000000000000009e
:10177400888b00008c8b0000908b0000958b000000
:10178400998b00009d8b0000a18b0000a58b0000ad
:10179400a98b0000ad8b0000b18b0000b58b00005d
:1017a40074650000787400002f7000006c61000004
:1017b400696e00000074000065780000742f00005a
:1017c400687400006d6c000000740000657800000f
:1017d400742f0000786d00006c0000007465000038
:1017e400787400002f630000737300000069000028
:1017f4006d610000676500002f67000069660000e6
:10180400006900006d610000676500002f70000032
:101814006e670000006900006d61000067650000ec
:101824002f6a00007065000067000000617000000e
:10183400706c00006963000061740000696f00004f
:101844006e2f00006a610000766100002d760000b2
:101854006d00000061750000646900006f2f0000d6
:10186400782d00007761000076650000000000001c
:10187400d28b0000dd8b0000dd8b0000dd8b0000cf
:10188400e78b0000f08b0000f98b0000038c000054
:101894000d8c0000188c00002c8c0000398c00008a
:1018a40048540000545000002f3100002e31000035
:1018b4002032000030300000204f00004b0d0000ab
:1018c4000a4300006f6e00006e6500006374000040
:1018d400696f00006e3a0000206300006c6f000026
:1018e400736500000d0a0000004800005454000015
:1018f400502f0000312e0000312000003430000051
:1019040030200000426100006420000052650000a5
:101914007175000065730000740d00000a43000037
:101924006f6e00006e65000063740000696f000054
:101934006e3a0000206300006c6f000073650000c5
:101944000d0a00000d0a00003430000030200000b1
:1019540042610000642000005265000071750000bf
:1019640065730000743a000020630000616e00009b
:101974002774000020680000616e0000646c0000a1
:1019840065200000436f00006e740000656e000067
:10199400742d00004c6500006e6700007468000040
:1019a4000d0a00000048000054540000502f0000ad
:1019b400312e0000312000003430000031200000be
:1019c400556e000061750000746800006f720000bd
:1019d400697a0000656400000d0a00005757000092
:1019e400572d00004175000074680000656e00000a
:1019f4007469000063610000746500003a2000000f
:101a040042610000736900006320000072650000f9
:101a1400616c00006d3d000022500000726f0000f8
:101a2400746500006374000065640000220d00000a
:101a34000a4300006f6e00006e65000063740000ce
:101a4400696f00006e3a0000206300006c6f0000b4
:101a5400736500000d0a00000d0a00003430000018
:101a640031200000556e00006175000074680000ac
:101a74006f720000697a0000656400003a2000007b
:101a84005061000073730000776f000072640000ff
:101a94002072000065710000756900007265000025
:101aa400640d00000a000000485400005450000077
:101ab4002f3100002e3100002034000030340000ab
:101ac400204e00006f740000206600006f75000057
:101ad4006e6400000d0a0000436f00006e6e00008b
:101ae40065630000746900006f6e00003a20000016
:101af400636c00006f730000650d00000a43000072
:101b04006f6e0000746500006e7400002d540000b8
:101b140079700000653a00002074000065780000c8
:101b2400742f0000687400006d6c00000d0a000042
:101b34000d0a000034300000343a00002046000052
:101b4400696c0000652000006e6f000074200000c6
:101b5400666f0000756e0000643c00006272000055
:101b64003e55000073650000203c00006120000029
:101b740068720000656600003d2200002f6d0000c1
:101b84007066000073750000706c00006f610000e7
:101b9400642200003e4d0000504600005320000027
:101ba400557000006c6f0000616400003c2f000061
:101bb400613e0000207400006f200000707200007d
:101bc4006f670000726100006d20000077650000ff
:101bd400622000007061000067650000730d000062
:101be4000a00000048540000545000002f31000047
:101bf4002e31000020340000313400002052000057
:101c04006571000075650000737400002d550000b7
:101c140052490000205400006f6f0000204c000067
:101c24006f6e0000670d00000a4300006f6e000035
:101c34006e65000063740000696f00006e3a000076
:101c4400206300006c6f0000736500000d0a000043
:101c54000d0a0000343100003420000052650000f9
:101c64007175000065730000742d0000555200006a
:101c740049200000546f00006f2000004c6f0000ea
:101c84006e6700003a20000042750000666600009e
:101c940065720000206f0000766500007266000027
:101ca4006c6f00007720000064650000746500001c
:101cb40063740000656400000d0a00000048000021
:101cc40054540000502f0000312e00003120000039
:101cd4003530000030200000496e000074650000bb
:101ce400726e0000616c00002053000065720000f9
:101cf400766500007220000045720000726f0000db
:101d0400720d00000a4300006f6e00006e65000053
:101d140063740000696f00006e3a000020630000e5
:101d24006c6f0000736500000d0a00000d0a0000ce
:101d34003530000030200000496e0000746500005a
:101d4400726e0000616c0000205300006572000098
:101d5400766500007220000045720000726f00007a
:101d6400723a0000204500007870000065630000ae
:101d74007465000064200000646100007461000068
:101d8400206e00006f740000207000007265000077
:101d9400736500006e7400000d0a00000048000026
:101da40054540000502f0000312e00003120000058
:101db40035300000312000004e6f00007420000018
:101dc400496d0000706c0000656d0000656e0000d8
:101dd40074650000640d00000a4300006f6e00008b
:101de4006e65000063740000696f00006e3a0000c5
:101df400206300006c6f0000736500000d0a000092
:101e04000d0a000035300000312000004e6f000044
:101e140074200000496d0000706c0000656d0000c6
:101e2400656e000074650000643a0000204f0000f5
:101e34006e6c00007920000047450000542000002b
:101e4400616e000064200000504f000053540000f5
:101e54002073000075700000706f00007274000041
:101e6400656400000d0a000000480000545400009e
:101e7400502f0000312e00003120000032300000cd
:101e8400302000004f4b00000d0a0000436f00009b
:101e94006e6e000065630000746900006f6e0000e0
:101ea4003a200000636c00006f730000650d0000b1
:101eb4000a4300006f6e0000746500006e74000039
:101ec4002d54000079700000653a00002074000071
:101ed40065780000742f0000687400006d6c0000c9
:101ee4000d0a00000d0a00003c680000746d00003b
:101ef4006c3e00003c6200006f640000792000002a
:101f040073740000796c0000653d0000226d0000d0
:101f140061720000676900006e3a00003130000011
:101f240030700000782200003e3c0000666f000024
:101f3400726d0000206d000065740000686f000081
:101f4400643d0000706f00007374000020610000a5
:101f540063740000696f00006e3d0000222f0000d2
:101f64006d70000066730000757000006c6f0000f7
:101f74006164000022200000656e000063740000ac
:101f840079700000653d0000226d0000756c000052
:101f94007469000070610000727400002f66000014
:101fa4006f7200006d2d0000646100007461000018
:101fb400223e00003c6200003e4d000050460000fe
:101fc40053200000496d0000616700006520000097
:101fd400557000006c6f0000616400003c2f00002d
:101fe400623e00003c7000003e3c0000696e000050
:101ff40070750000742000007479000070650000a2
:102004003d660000696c0000652000006e61000000
:102014006d6500003d69000020730000697a0000ce
:10202400653d0000343000003e200000266e0000b4
:1020340062730000703b0000203c0000696e0000e9
:102044007075000074200000747900007065000051
:102054003d730000756200006d690000742000008b
:10206400766100006c750000653d0000225500009b
:10207400706c00006f610000642200003e3c0000b0
:102084002f6600006f7200006d3e00003c2f0000c0
:10209400626f0000647900003e3c00002f6800007d
:1020a400746d00006c3e00000048000054540000b1
:1020b400502f0000312e000031200000323000008b
:1020c400302000004f4b00000d0a0000436f000059
:1020d4006e6e000065630000746900006f6e00009e
:1020e4003a200000636c00006f730000650d00006f
:1020f4000a4300006f6e0000746500006e740000f7
:102104002d54000079700000653a0000207400002e
:1021140065780000742f0000687400006d6c000086
:102124000d0a00000d0a00003c680000746d0000f8
:102134006c3e00003c6200006f64000079200000e7
:1021440073740000796c0000653d0000226d00008e
:1021540061720000676900006e3a000031300000cf
:1021640030700000782200003e3c0000623e000017
:102174004d500000465300002055000070640000dc
:102184006174000065200000537500006363000063
:102194006573000073660000756c00003c2f00003e
:1021a400623e00003c7000003e3c000061200000e4
:1021b40068720000656600003d2200002f220000c6
:1021c4003e53000069740000652000006d6100004a
:1021d400696e00002070000061670000653c00002b
:1021e4002f6100003e3c00002f6200006f6400007d
:1021f400793e00003c2f0000687400006d6c000004
:102204003e00000048540000545000002f310000ec
:102214002e3100002035000030300000204900003d
:102224006e740000657200006e6100006c20000096
:1022340053650000727600006572000020450000be
:10224400727200006f7200000d0a0000436f0000fc
:102254006e6e000065630000746900006f6e00001c
:102264003a200000636c00006f730000650d0000ed
:102274000a4300006f6e0000746500006e74000075
:102284002d54000079700000653a000020740000ad
:1022940065780000742f0000687400006d6c000005
:1022a4000d0a00000d0a00003c680000746d000077
:1022b4006c3e00003c6200006f6400007920000066
:1022c40073740000796c0000653d0000226d00000d
:1022d40061720000676900006e3a0000313000004e
:1022e40030700000782200003e3c0000623e000096
:1022f4004d50000046530000204900006d6100006d
:1023040067650000204300006f72000072750000d2
:1023140070740000206f00007220000057720000eb
:102324006f6e0000672000005665000072730000a5
:10233400696f00006e3c00002f6200003e3c00000c
:10234400703e00003c6100002068000072650000df
:10235400663d0000222f00006d70000066730000cf
:10236400757000006c6f000061640000223e000084
:102374005472000079200000616700006169000068
:102384006e3f00003c2f0000613e00003c2f000027
:10239400626f0000647900003e3c00002f6800007a
:1023a400746d00006c3e00000048000054540000ae
:1023b400502f0000312e0000312000003330000087
:1023c40032200000466f0000756e0000640d0000ae
:1023d4000a4300006f6e00006e6500006374000025
:1023e400696f00006e3a0000206300006c6f00000b
:1023f400736500000d0a00004c6f0000636100006b
:10240400746900006f6e00003a200000004800006c
:1024140054540000502f0000312e000031200000e1
:102424003430000033200000466f00007262000068
:1024340069640000646500006e0d00000a4300003a
:102444006f6e00006e65000063740000696f000029
:102454006e3a0000206300006c6f0000736500009a
:102464000d0a00000d0a0000343000003320000083
:10247400466f000072620000696400006465000039
:102484006e3a000020530000534c0000205200001c
:102494006571000075690000726500006420000029
:1024a4002d200000757300006520000048540000d2
:1024b40054500000530d00000a000000528c00002c
:1024c400528c0000778c0000d58c0000568d0000e3
:1024d400f48d0000618e0000d18e0000378f000063
:1024e400398c00005790000004910000d79100003f
:1024f40009920000436f00006f6b000069650000e3
:102504003a00000041750000746800006f7200001a
:10251400697a000061740000696f00006e3a00007f
:10252400004300006f6e0000746500006e740000cc
:102534002d4c0000656e000067740000683a0000ce
:10254400000000007c92000084920000939200003e
:102554004745000054000000504f00005354000051
:10256400006d00007066000073750000706c000060
:102574006f61000064000000696e00006465000083
:10258400782e0000687400006d0000000d0a000041
:102594000d0a0000333000003420000052650000b2
:1025a4006469000072650000637400003a20000052
:1025b400004300006f6e0000746500006e7400003c
:1025c4002d54000079700000653a000020000000de
:1025d400436f00006e740000656e0000742d0000ef
:1025e400456e0000636f0000646900006e670000c0
:1025f4003a200000677a0000697000000d0a0000ac
:102604000043000061630000686500002d43000082
:102614006f6e0000747200006f6c00003a200000be
:10262400006e00006f2d000063610000636800000d
:10263400650000006d610000782d000061670000f6
:10264400653d0000003600003030000000530000fb
:10265400657400002d4300006f6f00006b6900007b
:10266400653a0000200000000d0a00000d0a000079
:10267400000d00000a0d00000a4d00005046000045
:102684005302000001000000707200006f7400002b
:102694006563000074000000736e00006d7000003c
:1026a40000610000646d0000696e0000006d0000b0
:1026b40069630000726f00006368000069700000c5
:1026c400006600006f7200006d7300002e68000049
:1026d400746d0000006c00006564000034000000ac
:1026e4006c65000064330000006c00006564000049
:1026f400320000006c6500006431000000630000db
:102704006f6f00006b690000657300002e680000a5
:10271400746d0000006c000065640000732e0000fe
:1027240063670000690000006c650000640000003d
:10273400757000006c6f0000616400002e6800007a
:10274400746d000000700000726f0000746500007a
:10275400637400002f6300006f6e00006669000060
:10276400672e0000687400006d000000656d0000b5
:10277400616900006c2f0000696e00006465000050
:10278400782e0000687400006d0000006c63000087
:10279400640000002f6600006f7200006d7300007b
:1027a4002e680000746d00000069000070000000d5
:1027b4006777000000730000756200000064000089
:1027c4006e73000031000000646e0000733200007c
:1027d400006d000061630000006800006f7300007a
:1027e400740000006468000063700000002f0000a3
:1027f400707200006f74000065630000742f0000a5
:1028040072650000626f00006f7400002e680000a3
:10281400746d00003f0000002f700000726f000014
:1028240074650000637400002f6300006f6e000085
:1028340066690000672e0000687400006d000000e7
:102844000d0a0000000d00000a0d00000a0000003f
:102854004d690000637200006f6300006869000046
:102864007020000054430000502f00004950000025
:102874002053000074610000636b000020530000cb
:10288400746100007475000073200000557000002e
:10289400646100007465000000220000534d0000d4
:1028a4005450000020530000657200007669000057
:1028b40063650000222000003c6d00006368000096
:1028c400706200006f6100007264000040700000dc
:1028d400696300007361000072650000676f0000a7
:1028e4006f6400002e6300006f6d00003e00000066
:1028f4004d4900004d4500002d7600006572000032
:10290400736900006f6e00003a200000312e000051
:10291400300d00000a4300006f6e00007465000073
:102924006e7400002d74000079700000653a000098
:10293400206d0000756c0000746900007061000077
:10294400727400002f6d0000697800006564000057
:102954003b200000626f0000756e0000646100009f
:10296400727900003d220000667200006f6e000064
:102974007469000065720000220d00000a00000066
:10298400736500007276000065720000007000003c
:102994006f7200007400000075730000657200001f
:1029a400007000006173000073000000746f000089
:1029b400006d0000736700000054000068690000a7
:1029c400732000006973000020610000206d000086
:1029d400756c0000746900002d70000061720000c5
:1029e400742000006d6500007373000061670000cf
:1029f40065200000696e0000204d0000494d000074
:102a040045200000666f0000726d000061740000d4
:102a14002e0d00000a0000002d2d0000667200003b
:102a24006f6e000074690000657200000d0a0000fa
:102a3400436f00006e740000656e0000742d00008a
:102a440074790000706500003a200000746500008d
:102a5400787400002f7000006c610000696e000043
:102a64000d0a00000d0a0000000d00000a2d0000f0
:102a74002d660000726f00006e740000696500002e
:102a8400720d00000a4300006f6e000074650000c0
:102a94006e7400002d74000079700000653a000027
:102aa4002074000065780000742f00006373000038
:102ab400760d00000a4300006f6e0000746500008c
:102ac4006e7400002d44000069730000706f0000f4
:102ad40073690000746900006f6e00003a20000002
:102ae4006174000074610000636800006d6500009b
:102af4006e7400003b200000666900006c650000f5
:102b04006e6100006d6500003d22000073740000da
:102b140061740000757300002e630000737600007a
:102b2400220d00000a0d00000a00000053590000a5
:102b340053540000454d0000205300005441000050
:102b440054550000530d00000a00000042750000b7
:102b5400747400006f6e0000733a00002c000000d3
:102b64004c450000447300003a2c00000050000063
:102b74006f7400003a2c0000002d00002d66000048
:102b8400726f00006e74000069650000722d000011
:102b94002d0d00000a0000002f6500006d6100008b
:102ba400696c00002f6900006e6400006578000005
:102bb4002e680000746d0000005300006570000072
:102bc400203100003020000032300000313200009b
:102bd40020300000303a0000303800003a30000065
:102be40030000000763500002e3400003200000072
:102bf40075700000006400006e0000005345000082
:102c04004c4500004354000045440000003c0000d3
:102c140062720000202f00003e000000266e0000bb
:102c240062730000703b0000006e0000616d0000e4
:102c340065000000486500006c6c00006f2c00000b
:102c4400200000006e6f0000742000007365000017
:102c5400740000003c6200003e550000706c0000ef
:102c64006f610000642000006120000046690000dc
:102c74006c6500003c2f0000623e0000003c000038
:102c8400623e0000557000006c6f0000616400003b
:102c94006564000020460000696c000065270000a0
:102ca400732000004d4400003520000077610000cf
:102cb400733a00003c2f0000623e00003c620000ba
:102cc400722000002f3e00000063000068650000d1
:102cd400636b000065640000006600006169000029
:102ce4006c00000054680000652000004479000076
:102cf4006e6100006d69000063200000444e000016
:102d040053200000436c0000696500006e740000ed
:102d140020690000732000006e6f00007420000022
:102d2400656e0000616200006c650000642e0000a6
:102d3400006e00006f6e000065000000626c000011
:102d44006f6300006b0000000d0a00000d0a000014
:102d54000d4d000069630000726f0000636800009d
:102d64006970000020540000435000002f49000007
:102d740050200000436f00006e6600006967000089
:102d840020410000707000006c6900006361000065
:102d9400746900006f6e0000202800007635000082
:102da4002e340000322c0000205300006570000017
:102db40020310000302000003230000031320000a9
:102dc400290d00000a0d00000a000000093100006e
:102dd4003a20000043680000616e0000676500004f
:102de4002073000065720000696100006c2000001f
:102df4006e7500006d620000657200003a09000003
:102e0400090000000d0a0000093200003a20000009
:102e140043680000616e00006765000020680000e0
:102e24006f730000742000006e6100006d65000087
:102e34003a09000009090000000d00000a09000019
:102e4400333a000020430000686100006e67000010
:102e54006520000073740000617400006963000061
:102e640020490000502000006164000064720000ea
:102e740065730000733a000009090000000d0000aa
:102e84000a090000343a0000204300006861000091
:102e94006e67000065200000737400006174000018
:102ea400696300002067000061740000657700001a
:102eb4006179000020610000646400007265000014
:102ec400737300003a090000000d00000a090000b5
:102ed400353a000020430000686100006e6700007e
:102ee40065200000737400006174000069630000d1
:102ef40020730000756200006e65000074200000fd
:102f04006d610000736b00003a09000009000000c5
:102f14000d0a0000093600003a2000004368000052
:102f2400616e00006765000020730000746100009a
:102f3400746900006320000070720000696d000075
:102f44006172000079200000444e0000532000000c
:102f54007365000072760000657200003a09000093
:102f6400000d00000a090000373a00002043000069
:102f7400686100006e670000652000007374000043
:102f84006174000069630000207300006563000041
:102f94006f6e00006461000072790000204400003c
:102fa4004e53000020730000657200007665000037
:102fb400723a0000090000000d0a00000938000000
:102fc4003a2000000044000069730000004500003e
:102fd4006e000000616200006c6500002044000087
:102fe4004843000050200000262000004950000003
:102ff400204700006c650000616e0000696e0000ef
:10300400673a0000090900004448000043500000ea
:1030140020690000732000006375000072720000d4
:10302400656e0000746c00007920000000650000eb
:103034006e610000626c00006564000000640000c2
:1030440069730000616200006c65000064000000a8
:103054000d0a0000093900003a200000446f000006
:10306400776e00006c6f000061640000204d00006a
:103074005046000053200000696d000061670000a5
:10308400652e0000000d00000a090000303a00001f
:103094002053000061760000652000002620000017
:1030a40051750000697400002e0000000d0a000034
:1030b400456e00007465000072200000612000006d
:1030c4006d6500006e75000020630000686f0000ed
:1030d40069630000653a0000200000000d0a00004a
:1030e400004e000065770000207300006574000046
:1030f400746900006e6700003a2000000049000077
:103104006e760000616c00006964000020690000b4
:103114006e700000757400002e0d00000a0000009f
:103124005365000074740000696e0000677300004a
:103134002073000061760000656400002e0d00001d
:103144000a0000001b5b0000324a00001b5b000009
:10315400333100006d1b00005b3100006d4d000039
:1031640069630000726f000063680000697000000a
:1031740020540000656c00006e650000742000009f
:103184005365000072760000657200002031000073
:103194002e3100001b5b0000306d00000d0a0000a2
:1031a400286600006f720000207400006869000047
:1031b40073200000646500006d6f00002c20000087
:1031c400747900007065000020270000616400002d
:1031d4006d6900006e270000206600006f72000019
:1031e4002074000068650000206c00006f67000018
:1031f400696e0000206100006e640000202700005a
:103204006d690000637200006f630000686900006c
:1032140070270000206600006f7200002074000018
:10322400686500002070000061730000737700007f
:103234006f720000642e0000290d00000a4c00008b
:103244006f670000696e00003a2000000050000023
:1032540061730000737700006f720000643a00002d
:1032640020ff0000fd2d0000000d00000a410000b9
:103274006363000065730000732000006465000050
:103284006e690000656400000d0a00000d0a00006c
:10329400000d00000a4c00006f6700006765000025
:1032a40064200000696e0000207300007563000054
:1032b4006365000073730000667500006c6c0000a9
:1032c400790d00000a0d00000a0d00000a500000ec
:1032d400726500007373000020270000712700004e
:1032e400207400006f2000007175000069740000f4
:1032f4000d0a0000000d00000a5300004e540000a7
:1033040050200000546900006d6500003a20000060
:103314002020000020280000646900007361000080
:10332400626c000065640000290d00000a41000081
:103334006e6100006c6f0000673a000020200000fe
:103344002020000020200000202000002020000079
:10335400202000002031000030320000330d000036
:103364000a42000075740000746f00006e73000060
:103374003a2000002020000020200000202000002f
:103384002020000033200000322000003120000003
:10339400300d00000a4c000045440000733a000060
:1033a40020200000202000003720000036200000ec
:1033b40035200000342000003320000032200000bb
:1033c40031200000300000002020000020200000f8
:1033d400202000002020000020200000000d00001c
:1033e4000a0d00000a4700006f6f000064620000cd
:1033f40079650000210d00000a0000000d0a00009c
:10340400546f00006f2000006d75000063680000b9
:103414002064000061740000612e00000d0a0000a9
:1034240000610000646d0000696e0000005400003b
:103434006f6f0000206d00007563000068200000bd
:1034440064610000746100002e0d00000a00000099
:103454006d690000637200006f630000686900001a
:10346400700000001b5b0000316d0000001b0000b9
:103474005b310000303b0000313500006600000085
:103484001b5b0000313100003b320000316600005c
:10349400001b00005b310000323b000031380000ab
:1034a400660000001b5b0000313300003b3100006c
:1034b40030660000001b00005b310000343b00005c
:1034c4003166000000000000070c00001116000027
:1034d400070c000011160000070c00001116000074
:1034e400070c000011160000050900000e1400006e
:1034f400050900000e140000050900000e14000068
:10350400050900000e140000040b00001017000051
:10351400040b000010170000040b0000101700003b
:10352400040b000010170000060a00000f1500002d
:10353400060a00000f150000060a00000f1500001f
:10354400060a00000f15000078a400006ad70000e6
:1035540056b70000c7e80000db700000202400001c
:10356400eece0000bdc10000af0f00007cf50000ee
:103574002ac60000874700001346000030a8000058
:103584000195000046fd0000d89800008069000005
:10359400aff70000448b0000b15b0000ffff0000a8
:1035a400bed700005c89000022110000906b00006f
:1035b4009371000098fd00008e43000079a600007e
:1035c40021080000b4490000622500001ef6000036
:1035d40040b3000040c00000515a00005e260000c5
:1035e400aac70000b6e900005d1000002fd6000055
:1035f400531400004402000081e60000a1d800003a
:10360400c8fb0000d3e70000e6cd0000e121000084
:10361400d607000037c30000870d0000d5f4000072
:10362400ed1400005a45000005e90000e3a900007c
:10363400f8a30000effc0000d90200006f6700004f
:103644008a4c00002a8d000042390000faff000075
:1036540081f6000071870000226100009d6d00006a
:103664000c380000e5fd000044ea0000bea40000a0
:10367400a9cf0000de4b0000604b0000bbf6000049
:1036840070bc0000bfbe0000c67e00009b28000086
:10369400fa270000a1ea000085300000efd4000002
:1036a400051d00008804000039d00000d4d90000b2
:1036b400e5990000dbe60000f87c0000a21f000092
:1036c40065560000acc400004422000029f4000048
:1036d40097ff00002a430000a723000094ab0000da
:1036e40039a0000093fc0000c35900005b65000092
:1036f40092cc00000c8f00007df40000efff00006e
:10370400d15d0000848500004f7e0000a86f00009a
:10371400e0e600002cfe00001443000001a30000ba
:10372400a1110000084e0000827e000053f7000043
:1037340035f200003abd0000bbd20000d72a0000d9
:1037440091d3000086eb000077770000772e00000d
:10375400676f00006f6700006c6500002e63000057
:103764006f6d0000004300006f7500006c64000082
:10377400206e00006f74000020720000657300006a
:103784006f6c000076650000205300006572000035
:1037940076650000724e0000616d0000655b0000fc
:1037a4005d200000746f00002049000050200000dc
:1037b400616400006472000065730000732e0000f1
:1037c4000d0a0000000d00000a0d00000a4300006d
:1037d4006f6e00006e65000063740000696e000087
:1037e4006720000075730000696e00006720000008
:1037f40042650000726b0000656c00006579000092
:10380400205300006f6300006b65000074730000b8
:1038140020540000435000002041000050490000a3
:103824002e2e00002e0d00000a00000020200000b3
:10383400204e00006f740000653a00002074000000
:103844006869000073200000646500006d6f00006b
:1038540020770000696c00006c200000646f000099
:10386400206e00006f740000686900006e6700003d
:103874002069000066200000616e000020750000d1
:103884006e640000657200006c790000696e0000cf
:103894006720000054430000505f000050550000b2
:1038a400525000004f530000455f000042450000a5
:1038b400524b0000454c0000455900005f43000096
:1038c4004c490000454e000054200000747900006b
:1038d40070650000200d00000a2000002020000078
:1038e400736f0000636b00006574000020690000c2
:1038f40073200000756e00006176000061690000ad
:103904006c610000626c0000652c00002061000006
:103914007320000064650000636c000061720000a5
:1039240065640000206200007920000074680000d3
:103934006520000054430000505300006f630000f2
:103944006b650000744900006e6900007469000032
:10395400616c0000697a0000657200005b5d000024
:10396400206100007272000061790000206900008b
:103974006e2000000d0a00002020000020540000ea
:103984004350000049500000436f00006e66000081
:10399400696700002e6800002e0d00000a0d00006b
:1039a4000a000000544300005053000074610000fa
:1039b400636b000020760000352e000034320000d6
:1039c40020200000202000002020000020200000f3
:1039d40020200000202000002020000020200000e3
:1039e40020200000000d00000a0d00000a42000023
:1039f40055540000544f00004e3000002068000071
:103a0400656c000064200000666f000072200000f6
:103a14006d6f000072650000207400006861000092
:103a24006e2000003420000073650000636f000006
:103a34006e640000732e0000202000004465000026
:103a440066610000756c000074200000736500005e
:103a540074740000696e0000677300002072000037
:103a640065730000746f000072650000642e00002e
:103a74000d0a00000d0a0000000d00000a4e0000af
:103a840065770000204900005020000041640000d8
:103a94006472000065730000733a000020000000a7
:103aa4000d0a00000000000004a300000000000054
:103ab400004d000043480000504200004f41000008
:103ac40052440000000000002f73000065610000f4
:103ad40072630000683f0000617300005f710000c2
:103ae4003d4d000069630000726f000063680000d0
:103af4006970000026610000735f000073690000b4
:103b04007465000073650000617200006368000062
:103b14003d6d000069630000726f0000636800007f
:103b2400697000002e6300006f6d0000000d00003e
:103b34000a0d00000a4300006f6e00006e6500006d
:103b440063740000696e0000672000007573000054
:103b5400696e0000672000004d6900006372000078
:103b64006f63000068690000702000005443000087
:103b74005020000041500000492e00002e2e00006d
:103b84000d0a00000047000045540000200000001a
:103b94002048000054540000502f0000312e000033
:103ba400300d00000a4800006f730000743a0000f2
:103bb400200000000d0a0000436f00006e6e00003c
:103bc40065630000746900006f6e00003a20000015
:103bd400636c00006f730000650d00000a0d0000a7
:103be4000a000000484500004c4f0000204d000032
:103bf40043480000504200004f410000524400007e
:103c04000d0a000000450000484c00004f20000051
:103c14004d43000048500000424f00004152000054
:103c2400440d00000a000000415500005448000003
:103c3400204c00004f470000494e00000d0a0000d0
:103c4400000d00000a0000004d410000494c000036
:103c540020460000524f00004d3a00003c00000096
:103c64003e0d00000a0000005243000050540000c2
:103c7400205400004f3a00003c0000004441000082
:103c8400544100000d0a000000460000726f00005d
:103c94006d3a0000200000000d0a0000546f00007f
:103ca4003a200000000d00000a430000433a0000df
:103cb400200000000d0a000053750000626a000035
:103cc40065630000743a0000200000000d0a000043
:103cd4002e0d00000a0000000d0a00002e00000056
:103ce40051550000495400000d0a00000000000076
:103cf4003a20000057650000206100007265000052
:103d04002063000075720000726500006e7400008c
:103d14006c790000206100006368000069650000a0
:103d2400766900006e67000020000000202000007b
:103d3400202000002020000020000000303000007f
:103d44002062000079740000657300002f73000086
:103d5400656300006f6e000064200000545800008a
:103d640020740000687200006f750000676800002e
:103d740070750000742e00000d0a00000020000081
:103d84006279000074650000732f00007365000001
:103d9400636f00006e6400000d0a00000000000064
:103da4006d610000696c000000220000534d0000aa
:103db4005450000020530000657200007669000032
:103dc40063650000222000003c6d00006368000071
:103dd400706200006f6100007264000040700000b7
:103de400696300007361000072650000676f000082
:103df4006f6400002e6300006f6d00003e00000041
:103e0400486500006c6c00006f200000776f0000b4
:103e1400726c00006421000020200000534d00005b
:103e2400545000002054000065730000742e0000fc
:103e34000000000077770000312e00006d6900005b
:103e4400637200006f63000068690000702e000058
:103e5400636f00006d000000506900006e67000091
:103e640020740000696d000065640000206f00008c
:103e74007574000000430000616e000027740000a8
:103e840020720000657300006f6c0000766500000e
:103e9400204900005000000052650000706c0000d2
:103ea400793a0000200000006d730000000000005b
:103eb400000000007d00000064000000010000001c
:103ec400140000001400000002000000c8000000fc
:103ed4009600000005000000c8000000010000007a
:103ee40007000000000100000001000008000000bd
:103ef400c8000000c800000008000000c80000005e
:103f0400c800000009000000c8000000c80000004c
:103f14000a00000019000000140000000d0a00004f
:103f240044480000435000002f5000006f77000009
:103f34006572000020650000766500006e74000064
:103f4400206f00006363000075720000726500005a
:103f540064000000426f00006f7400006c6f00008a
:103f64006164000065720000205200006573000067
:103f74006574000000000000706f00006f6c0000aa
:103f84002e6e0000747000002e6f00007267000037
:103f940000000000706f00006f6c00002e6e0000c7
:103fa400747000002e6f00007267000000000000b3
:103fb4004d500000465300000201000000000000c4
:020000040000fa
:103fc4000200fa00004f780061fc20009140780064
:103fd4001e40780080cf50002100320061fc200098
:103fe40091407800e0cfb30080cf50000a00320047
:103ff400c6cfbf000080fb007e00b90080007800bf
:104004000080200000804000e20120002197200071
:10401400940a0200000000001e407800c6efb700ba
:104024009e407800e0cfb30080cf50000e003200f5
:104034009e4078000180fb007e00b900800078007b
:104044000080200000804000e20120008000780011
:1040540020972000940a02000000000003003700ab
:104064000000000001003700000000000080fa009a
:10407400000006000000fa0071fc20009140780066
:10408400c6cfbf0080cf50002700320071fc200053
:1040940091407800e0cfb30080cf5000150032008b
:1040a400e2902000c7cfbf000080fb007e00b90073
:1040b40000007800fc0040000080200000804000e8
:1040c40090427800c7cfbf000080fb007e00b9009b
:1040d40080007800008020000080400010007800fc
:1040e4008002b1008402200013c0b3008540780030
:1040f400ed110700c6cfbf00c7efb7008ec9bf00e0
:10410400914b80008102b100e590200084022000e0
:10411400804178000101780011c0b30005007800e7
:10412400e111070001003700000000000080fa00e0
:10413400000006000c00fa00c0fb200010079800e5
:10414400217e80000000eb00808f500008003a00c0
:1041540096aa02000000000080007800f07f200092
:10416400808060000040200000804000207e8800a5
:10417400c20320008000eb0060932000a20a02002a
:10418400000000000040eb00404798000040eb00b6
:10419400004f78004e0037001e40780088ff07006b
:1041a4009e4078000180fb006600b9008000780022
:1041b400a0f52900008040009040900051479800ed
:1041c4009e4078000180fb006600b9000000780082
:1041d4008080e800a0f5290000804000900078006d
:1041e400310798009e4078000180fb006600b9000a
:1041f40000007800e4004000a0f5290000804000a1
:1042040090007800410798005e4090008080fb0099
:104214000000eb00808f5000010032002b003700bb
:104224001e00900050079800be0090004e009000c1
:10423400808040001e00900000804000a002b0007a
:10424400100798009e00900080ef2100808f50009e
:10425400fcff3e00de409000010078008ee9b700cc
:104264005e0090008002b000904b8800914b80006b
:104274003e009000008040000000e800a04b880051
:10428400a14b80004e00900000804000b04b88009d
:10429400d0002000404c88008a69a90075ff0700ff
:1042a4009e4078000180fb006600b9008000780021
:1042b400a0f52900008040001040780035e9b700df
:1042c400730b07001e4fe80001003700ffff3700a3
:1042d4009e40780080c0b30080cf5000aeff36000f
:1042e4000080fa00000006000c00fa001007980095
:1042f400210798006247980043079800244f9800cc
:104304000040eb00004f78009a0037001e40780010
:104314002bff0700414c8000d0002000808f50000c
:1043240090003a0053ff0700519320009140780019
:104334002e48900080cf50008c003a00802120004d
:1043440090498800ee4090000040eb0080cf500080
:1043540008003a004e009000f04888008a69a800de
:1043640040002000404c8800ce019000634c88003f
:104374007a003700217e8000f03f2000808f5000bb
:1043840004003600217e800080382100808f500098
:104394000200360000402000207e8800207e80003d
:1043a400f04888000000e800207e88004e0090005d
:1043b400e04888009a10020001000000004c8800c8
:1043c400114c88008a89a8006e4090000080fb0090
:1043d4006101b9000080eb008080eb000200400026
:1043e400838048003200200003002000820f500028
:1043f400838f580059003e0000600100030037001d
:1044040002003700160037002c0037001e00900011
:10441400ae00900020498800314988006e40900029
:104424000014a2000080fb000000e9004f00de0041
:10443400004078000080fb00610060004200dd0065
:1044440082498000b1ff2f0081006100008070006c
:10445400804988000000eb00404c88003f00370092
:104464000e80e800900090000e80e80010007800b4
:10447400808040004e00900080804000f048800022
:1044840000806800604c88001e009000ae00900020
:1044940020498800314988000040eb0034e9b70026
:1044a400d003200001002000704888008148880063
:1044b40020002000404c8800280037001e00900097
:1044c400ae00900000007800800078002140900049
:1044d4000081fb00314090000080fb004800dd00bb
:1044e40002007000000178001e009000ae009000f1
:1044f40000007800904178008380fb001040900019
:104504000080fb004800dd000100700080004100d5
:104514004e00900080804000f048800000806800d9
:10452400604c88001e009000ae00900000007800ef
:10453400a20020008000780040922000940a02002b
:104544000000000050002000404c880011c0b3005f
:1045540020c0b30056070700000000001e4078008a
:1045640009003700000000000100370000000000cf
:104574001e4fe8009e40780080c0b30080cf5000fa
:1045840062ff3600e0cfb3000080fa0000000600ae
:104594000200fa00004f78009e40780080c0b3000b
:1045a40080cf500002003600100020000c003700bd
:1045b4001e40780082fe0700514c8000000021005c
:1045c400808060000000eb00808f50000300320008
:1045d4008b89a90010002000010037000000eb00c7
:1045e4000080fa00000006000200fa00004f780084
:1045f4009e40780080c0b30080cf50000200360097
:104604000000eb00080037001e4078006cfe070035
:10461400424c80001000200071002000810f5100e6
:10462400010032000000eb000080fa0000000600e8
:104634000200fa00004f78009e40780080c0b3006a
:1046440080cf50004a003e001e4078005cfe070008
:10465400e04b8000f04b8800404c800001002000bb
:10466400e200200003002000820f5000838f5800d6
:1046740039003e0000600100120037000d003700d1
:10468400100037000f003700330037000d003700eb
:104694000e0037000d0037002f0037002e003700c2
:1046a4002d003700190037002b0037002a0037008f
:1046b4002600370072c6020000000000740a0700da
:1046c4002c003700720a07002a00370011c0b3001b
:1046d40010c1b300f6060700014980000000eb009a
:1046e400808f500005003200c14b8000d04880000c
:1046f400808f5000f5ff3a000100370000000000f1
:1047040080002000404c88001a00370011c0b3001c
:1047140010c1b300e6060700014980000000eb0069
:10472400808f500005003200c14b8000d0488000cb
:10473400808f5000f5ff3a000100370000000000b0
:10474400c0002000404c88000a003700d000200040
:10475400404c8800070037008040eb0040c1b300a4
:10476400d30607004a0a07000000000001003700d2
:10477400000000000080fa00000006000200fa00b9
:10478400004f78009e40780080c0b30080cf500076
:1047940006003e001e40780009fe07008a69a90051
:1047a4001e407800a2ff070001003700000000004f
:1047b4000080fa00000006000200fa00004f7800b2
:1047c4009e40780080c0b30080cf500002003600c5
:1047d4000000eb000b0037001e407800f8fd0700d6
:1047e40024fe0700a200200041922000009920002e
:1047f400940a020000000000e0488000d04c8800c9
:10480400009920000080fa00000006000200fa006f
:10481400004f78009e40780080c0b30080cf5000e5
:104824000b003e001e407800e5fd070011fe070066
:10483400c14b8000d0488000808f500005003200ba
:1048440011c0b30000c1b30099060700010037008e
:10485400000000000080fa00000006000400fa00d6
:1048640020479800ae40900080c0b30080cf500035
:10487400020036000000eb001f0037002e409000bd
:10488400cffd0700404c8000004f78009e40780028
:1048940070c0b30080cf5000060032009e40780004
:1048a400b0c0b30080cf5000020032000000eb0023
:1048b40011003700c14b8000d04b8000808f500026
:1048c40009003900a14b8000904b8000808050008b
:1048d400d24b8000c04b800000005100008040009b
:1048e4000000e90004003700d14b8000c04b800079
:1048f400008050000000e9000080fa00000006007b
:104904000400fa002047980031479800ae40900018
:1049140080c0b30080cf5000020036000000eb00de
:10492400470037002e409000a5fd07002e40900060
:10493400caff0700000f78009e0078000000eb001b
:10494400808f500002003a000000eb003c0037006a
:104954009e00780010002000808f500002003a0072
:104964002e409000a9ff0700514c80000010200049
:10497400808060000000eb00808f50000a003a0045
:10498400a14b8000904b8000008050008000d1003b
:104994001e007800808f5000030039002e409000e4
:1049a4009aff07008b09a800e30047008ec9bf00e7
:1049b400c54b80001400200013c0b300010178002f
:1049c4008040780005007800b70f0700c04b8000d6
:1049d4000000e800c04b8800c14b8000a04b800061
:1049e400808f500002003900904b8000c04b88003b
:1049f4009e00780010002000808f500003003a00d1
:104a04002e40900081ff07000c003700514c8000bd
:104a140000022000808060000000eb00808f5000c6
:104a240006003a008aa9a800a610020001000000ae
:104a34000000780069004000204c8800100020002d
:104a44000080fa00000006000c00fa00604798009d
:104a540041079800520798000000eb0010079800e7
:104a6400ee40900080c0b30080cf500002003600ba
:104a74000000eb00600037006e40900050fd07001e
:104a84006e40900075ff070020079800ae0090006c
:104a94000000eb00808f500004003a006e4090004c
:104aa4005aff07000000eb00530037002e0090006f
:104ab400000f7800ae0090005e009000808f5000e0
:104ac400020036005e009000000f7800514c800018
:104ad40000102000808060000000eb00808f5000f8
:104ae4000a003a00a14b8000904b800000805000e7
:104af4008000d1002e009000808f50000300390008
:104b04006e40900041ff07008b09a800c04b800055
:104b14009e004000a04b8000808f5000150039009b
:104b2400a14b8000c04b800000805000100798000b
:104b3400ce0090008ec9bf00c54b80001e029000bd
:104b440013c0b300010178008040780005007800ac
:104b5400550f0700ce0090001e009000008040001a
:104b6400400798001e0090001e0f1000904b80001c
:104b7400c04b8800ce0090008ec9bf00c54b80009a
:104b84001e02780013c0b300010178008040780051
:104b940005007800440f0700c04b80001e00400051
:104ba400c04b8800ae0090005e009000808f5000e3
:104bb40003003e006e40900014ff07000c00370015
:104bc400514c800000022000808060000000eb0057
:104bd400808f500006003a008aa9a800a61002009f
:104be400010000000000780069004000204c8800ab
:104bf4001e0090001e0040000080fa000000060025
:104c04000400fa00004f7800110798001e0090007d
:104c1400de0a020000000000000178009e009000ff
:104c24001e40780088ff07009e009000008040002e
:104c34000080fa00000006000600fa0040479800d1
:104c4400ce40900080c0b30080cf500002003600f8
:104c54000000eb000b0037004e409000d8fc07002a
:104c6400a14b8000904b800000805000000fe900b1
:104c74004e409000f9fe0700100798001e009000b7
:104c84001e0010000080fa00000006000200fa0076
:104c9400004f78001e4078000c0007008000eb00f5
:104ca400810f5000070032001e407800c4fc07004a
:104cb400e04b8000f04b880011c0b30000c1b3008a
:104cc4007b0507000080fa00000006000200fa00dd
:104cd400004f78009e40780080c0b30080cf500021
:104ce400020036000000eb00120037001e4078007e
:104cf400b3fc0700e14b8000f04b8000808f500034
:104d040004003900e14b8000f04b8000008050002b
:104d140008003700b14b8000f04b800080805000c9
:104d2400e24b8000a04b8000000051000080400056
:104d34000000e8000080fa00000006000600fa0007
:104d440020479800210798002e409000dfff0700bd
:104d5400000f78009e0078000000eb00808f500068
:104d640002003a000000eb002b0037002e409000b8
:104d740093fc0700ae0090000000eb00808f500011
:104d8400090032008ec9bf00f14b8000ae029000d2
:104d940014002000804178000101780011c0b300a4
:104da40005007800c00e0700f04b80000000e8000a
:104db400f04b8800f14b8000b04b8000808f500096
:104dc40002003600a04b8000f04b88009e00780063
:104dd40010002000808f500002003a008b49a80088
:104de4000c003700514c80000002200080806000dd
:104df4000000eb00808f500006003a008aa9a8004a
:104e0400a610020001000000000078000003b000ba
:104e1400204c8800100020000080fa0000000600ea
:104e24000a00fa00404798003107980042079800aa
:104e34000000eb00000f78004e409000a3ff070035
:104e4400100798009e0090000000eb00808f500037
:104e540002003a000000eb00500037004e40900082
:104e640057fc0700ce0090001e009000808f500079
:104e7400020036001e00900040079800f14b8000ad
:104e84004e00900080804000b04b8000808f500026
:104e940019003600b14b8000f04b800000805000b8
:104ea400000fe800be0090000000eb00808f50006f
:104eb4000c0032008ec9bf00f14b8000be0290008e
:104ec4001e027800804178000101780011c0b3000f
:104ed40005007800740e07003e0090001e0040009c
:104ee400300798004e0090001e00500040079800c4
:104ef400a04b8000f04b8800be0090000000eb0047
:104f0400808f5000090032008ec9bf00f14b800031
:104f1400be0290004e0290008041780001017800aa
:104f240011c0b300050078005f0e0700f14b80004c
:104f34004e00900000804000f04b88004e0090002e
:104f44001e004000400798009e0090004e00900014
:104f5400808050004e009000808f500002003e0080
:104f64008b49a8000c003700514c8000000220003f
:104f7400808060000000eb00808f500006003a0043
:104f84008aa9a800a6100200010000000000780011
:104f94000003b000204c88004e0090000080fa000e
:104fa400000006000600fa0040479800ce4090003a
:104fb40080c0b30080cf5000020036000000eb0038
:104fc4000a0037004e409000fdfb0700b14b800003
:104fd400a04b8000008f50004e4090003bff070024
:104fe400100798001e0090001e0010000080fa00b8
:104ff400000006000e00fa00604798004107980080
:105004005207980063079800ee40900080c0b300f8
:1050140080cf500004003e00de0090000000eb0052
:10502400808f500002003a000000eb00430037007c
:105034006e409000e2fb07006e40900023ff0700e3
:1050440010079800ee0090005e0090008080400001
:105054001e009000808f5000040036009e009000d7
:105064006e0090000080500050079800f14b8000c3
:105074006e009000008f4000b14b80001e0078004d
:10508400808f500005003100b14b8000a04b8000a0
:10509400008050000080ea001e0f4000b04b8000ea
:1050a4001e0050000000e80020079800de00900079
:1050b4002e009000808f500009003e008ec9bf0072
:1050c400ce0290005e029000804178001e017800bc
:1050d40011c0b30005007800f30d07001600370077
:1050e4008ec9bf00ce0290002e029000804178004d
:1050f4001e01780011c0b30005007800ea0d070016
:10510400de0090002e009000008150008ec9bf0088
:10511400a14b80004e029000ae0190008302420039
:1051240002027800804178000101780011c0b300c8
:1051340005007800dc0d07005e0090000080fa0096
:10514400000006000600fa00204798002107980096
:10515400ae019000120020008e0078002e409000d6
:10516400a4ff07001e4078000080fa00000006003b
:105174003e00fa0020779800211f9800321f980003
:10518400431f9800541f9800651f9800ae7090004c
:1051940080c0b30080cf500004003e00be189000d1
:1051a4000000eb00808f500002003a000000eb008a
:1051b400330137002e70900081fb07002e709000a1
:1051c400c2fe0700ce18900001005000100798009e
:1051d4009e0090003e189000808f50000200310025
:1051e4000080eb0026013700de1890000000eb0081
:1051f400808f5000060032009e0090005e189000e0
:10520400808f5000020036005e189000100798004e
:10521400f14b80004e189000008040003007980049
:10522400b14b80003e009000808f50000700310099
:10523400b14b8000a04b8000008050000080ea0049
:10524400be0090000080400030079800be0090002f
:10525400010f7800b14b80003e00900000805000a8
:105264000000e800200798004e18900030079800ce
:10527400be189000710798002e189000000f980037
:105284002e18900090407800114f98002e1890002e
:105294000000e800201f98000000eb006007980061
:1052a400ee1890000000eb00808f50000c003200dc
:1052b4009e48900000c6b30080cf5000080036001e
:1052c4009e489000a0c7b30080cf500004003e0069
:1052d4009e48900000ceb30000c04000104f9800dc
:1052e40000c2b300204f98002e4890008080fb003d
:1052f4002e009000808f5000020036002e00900097
:10530400204f98002e4890008080fb001e009000e3
:10531400808f5000020036001e009000204f98003d
:105324002e4890008080fb008ec9bf00f202470027
:1053340001027800804178001e01780011c0b3009a
:1053440005007800580d07002e4890000080fb00ef
:105354001e0f40002e4890000080fb00ae0090001d
:105364000080500020079800ae0090000000eb0081
:10537400808f500004003a00a04b8000000f78009a
:105384000080eb0020079800ee1890000000eb006e
:10539400808f50006f0032000040eb00004f9800f7
:1053a400670037000e4890000080fb00f2004700c1
:1053b400008040009040780000c6b30080cf5000c9
:1053c400140036000e4890000080fb00f2004700f5
:1053d4000080400090407800a0c7b30080cf500008
:1053e4000c003e000e4890000081fb000e48900027
:1053f4000080fb00f20047000080400090407800ed
:1054040000ceb30000c04000f2004700828040009c
:10541400804878000e4890000080fb00f2004700ae
:1054240000804000904078001e48900080cf5000db
:1054340024003a003e1890000000e900301f980054
:10544400be1890000000eb00808f500008003a0066
:10545400be0090007e009000808050000e489000b6
:105464000080fb00008040000000e800840037005a
:105474002e18900090407800114f98002e1890003c
:105484000000e800201f980010002000600798002a
:105494009e48900000c6b30080cf5000250036001f
:1054a4009e489000a0c7b30080cf500021003e006a
:1054b4009e48900000ceb30000c04000104f9800fa
:1054c4001c0037007e009000301f9800ee00900012
:1054d4000000eb00808f5000160032008e08900010
:1054e400211f98002e18900090407800114f9800ca
:1054f4002e1890000000e800201f98009e4890009d
:1055040000c6b30080cf5000080036009e489000cb
:10551400a0c7b30080cf500004003e009e48900016
:1055240000ceb30000c04000104f98000000eb0014
:10553400600798000e4890000040e800004f980073
:105544008e4890002e48900080cf500095ff39007f
:105554003a0037000040eb00004f9800330037005a
:105564000e4890000080fb00f200470000804000dd
:10557400904078001e48900080cf500018003a00f8
:105584003e1890000000e900301f9800be189000fb
:105594000000eb00808f500008003a00be0090002d
:1055a4007e009000808050000e4890000080fb0038
:1055b400008040000000e800310037002e18900001
:1055c40090407800114f98002e1890000000e800d9
:1055d400201f98001000200060079800100037007a
:1055e4007e009000301f9800ee0090000000eb0059
:1055f400808f50000a0032008e089000211f98000e
:105604002e18900090407800114f98002e189000aa
:105614000000e800201f98000000eb0060079800dd
:105624000e4890000040e800004f98008e4890001b
:105634002e48900080cf5000c9ff39002e489000ba
:105644000080fb009e00900000805000100798002e
:105654009e0090003e189000808f500002003100a0
:105664000080eb00060037002e4890000080fb000d
:10567400be009000008040003007980018ff3700fb
:105684000080fa00000006000800fa00004f7800cd
:1056940011479800120798002307980034079800d0
:1056a4000e00e800be0290002e0290009e019000c1
:1056b40012002000800078001e407800acfe070035
:1056c4000080fa00000006000e00fa00881f78002f
:1056d4000040eb00004f7800500237001e40780075
:1056e40037fa07000040eb00604798000000eb0029
:1056f400100798000000eb0020079800514c800030
:1057040000202000808060000000eb00808f5000ab
:1057140006003a00514c8000004020008080600068
:105724000000eb00808f50000c0032007e860200e7
:10573400000000008000eb00810f500007003200e1
:1057440000c1b30060479800504c80004a00de005e
:10575400614060000080fb0010079800514c8000fd
:1057640000022000808060000000eb00808f500069
:105774000b003200284c8000a6100200010000003b
:105784000000780000005400800078000000eb0066
:10579400808f500002003c0000c1b30060479800b5
:1057a400514c800000042000808060000000eb0069
:1057b400808f50000b003200384c8000a61002008d
:1057c4000100000000007800000054008000780010
:1057d4000000eb00808f500002003c0000c1b300c9
:1057e40060479800414c8000b0002000808f50003a
:1057f4000d003a00384c8000a610020001000000a1
:105804000000780000005400800078000000eb00e5
:10581400808f500004003c0010c1b3006047980022
:10582400c0002000404c8800414c80004000200013
:10583400808f500065003a000000eb00400798009c
:105844005c0037004e0090007400b900000078003e
:10585400f000400060932000008040009000780039
:105864000000eb00808f5000570032004e00900083
:105874007400b90000007800f0004000609320003c
:105884000080400090007800604c8000808f5000c1
:1058940045003a00f7f907004e0090007400b90083
:1058a400800078006093200000804000a200200067
:1058b4008000780040922000940a0200000000005a
:1058c4004e0090007400b90000007800ea00400027
:1058d400609320000080400010007800e0488800b9
:1058e4004e0090007400b90000007800ec00400005
:1058f40060932000008040001001be0010002000d2
:10590400010020000200400083804800b048880065
:10591400c1488800314980002049800080804000cf
:10592400e048800080804000f048800000806800eb
:10593400604c880020c1b3006047980060002000dc
:10594400404c8800ce009000c0fe2f000088b900b3
:105954000000780083022000808141004e00900006
:105964000000e8007400b900800078006093200013
:1059740000804000000178004e0090007400b900df
:1059840080007800609320000080400003027800cb
:1059940013c0b30011c0b300c30b07000000eb0039
:1059a400704b8800090037004e0090000000e800aa
:1059b40040079800ce00900020002000808f500007
:1059c400a0ff36000100370000000000ee40900008
:1059d4000040eb0080cf50000900320010c0b3003b
:1059e4001e0190008000eb00810f51000100320085
:1059f4000040eb00804078006e4090002c020700cd
:105a0400504c8000f00060000000eb00808f5000dc
:105a140032003a00414c800070002000808f50001a
:105a240076013a009a100200010000000001be0055
:105a3400004c8000114c800000005100818059000e
:105a44000001be006000b800800f5100818f590032
:105a54006c013500504c8000e700600060002000bd
:105a6400808f50000f003a00504c80004300de004d
:105a740061406000604798001e407800ecfa07001f
:105a84001e407800eafa0700ee4090000040eb0068
:105a940080cf50005d013a00e0002000404c8800b7
:105aa4005d01370073f9070021c0b30000c1b300e2
:105ab400ff0107009a100200010000000001be006f
:105ac4008096280091002000020040008380480056
:105ad400004c8800114c88004f0137009a100200d6
:105ae400010000000001be00004c8000114c800049
:105af40000005100818059000001be006000b80020
:105b0400800f5100818f59004201350059f9070077
:105b1400404c800001002000c2002000030020004f
:105b2400820f5000838f5800ef003e000060010098
:105b34000c003700250037005000370059003700ab
:105b4400eb003700800037008f003700a5003700d6
:105b5400b3003700c1003700c5003700a10037008b
:105b6400d20037005ac60200000000008000eb009b
:105b7400810f5000e000320010002000404c8800eb
:105b840080498000e40060000000eb00808f50003a
:105b9400070032002049800031498000000078006d
:105ba40011c0b3009cc6020000000000d9003700f9
:105bb40020498000314980000000780011c0b30002
:105bc4009cc6020000000000d20037006a004700b3
:105bd400cec60200000000008000eb00810f5000e0
:105be400c700320072c60200000000008000eb0013
:105bf400810f5000150032005e009000ee0090000e
:105c0400204988003149880020002000404c880049
:105c1400314980002049800080804000e0488000b5
:105c240080804000f048800000806800604c88005c
:105c34000040eb0034e9b700d0032000010020004d
:105c44007048880081488800b20037009a1002002a
:105c5400010000000001be00809628009100200091
:105c64000200400083804800004c8800114c8800ea
:105c74000000eb00404c8800a6003700a61002008c
:105c84000100000000007800204c880040922000b1
:105c940060e602000000000030002000404c880054
:105ca4009c00370081922000409220002ce70200e3
:105cb400000000008000eb00810f50001b003a0040
:105cc400a61002000100000080007800204c800033
:105cd40000815000704880008148800000007800f6
:105ce400800f5100880036004193200091407800d5
:105cf40050c0b30080cf500009003e0034c9bf003b
:105d04000040e80034e9b700704880008148800012
:105d14000000400081804800704888008148880065
:105d240020002000404c88007a00370020c0b300d7
:105d3400604798000000eb00100798005000200016
:105d4400404c88007300370020c0b30060479800bf
:105d54001000200010079800419320009140780023
:105d640030c0b30080cf50006900360040c0b3009b
:105d740034e9b70000242400f100200070488800b2
:105d840081488800630037004193200091407800e7
:105d940010c0b30080cf500005003e0020c1b30006
:105da4006047980010002000100798005900370041
:105db400504c8000e80060000000eb00808f500031
:105dc4000500320040c1b300604798001000200075
:105dd400200798004f00370020c0b30060479800a8
:105de4004c003700419320009140780040c0b3003c
:105df40080cf500005003e0000c1b300604798000a
:105e04001000200010079800420037008000200096
:105e1400404c880010c1b300604798003d00370033
:105e2400419320009140780040c0b30080cf5000df
:105e340005003e0010c1b300604798001000200028
:105e4400100798003300370040c1b3006047980042
:105e540010002000200798002e00370040c1b30036
:105e640060479800100020002007980029003700a0
:105e7400419320009140780040c0b30080cf50008f
:105e840005003e0000c1b3006047980010002000e8
:105e9400100798001f00370040c1b3006047980006
:105ea40010002000200798001a00370041932000ba
:105eb4009140780040c0b30080cf500005003e0000
:105ec40010c1b3006047980010002000100798002c
:105ed4001000370040c1b300604798001000200054
:105ee400200798000b00370000000000090037006d
:105ef4000000000007003700000000000500370024
:105f0400000000000300370000000000010037001b
:105f140000000000ee4090000040eb0080cf5000f5
:105f2400300032009e0090000000eb00808f500093
:105f34002900320034c9bf000040e80034e9b7004a
:105f44007048800081488000000040008180480043
:105f54007048880081488800d1488000d04b800078
:105f64000080500040079800d1488000d04b80004a
:105f7400808f500006003100a14b8000904b8000c0
:105f840000805000ce009000008040004007980040
:105f940092488000a34880004e0090000100200039
:105fa400000051008180590090488800a148880071
:105fb400014980004e0090000080400000498800a4
:105fc400d04b8000d04888008040eb006e409000a9
:105fd400b70007000300370011c0b3006e40900003
:105fe400b3000700ae0090000000eb00808f50006b
:105ff40009003200260407000700370000000000f3
:106004000500370000000000030037000000000016
:1060140001003700000000001e4fe8009e40780099
:1060240080c0b30080cf5000acfd36000000eb0010
:1060340040079800360037004e0090007400b90005
:1060440000007800f00040006093200000804000d1
:10605400900078000000eb00808f50003100320087
:10606400a610020001000000000178004e0090001c
:106074007400b90000007800f20040006093200032
:10608400008040001000780080005100c02d2000e6
:10609400808f50001b003600ce009000c0fe2f0001
:1060a4000088b9000000780083022000808141004c
:1060b4004e0090000000e8007400b90080007800f1
:1060c4006093200000804000000178004e009000a2
:1060d4007400b900800078006093200000804000c4
:1060e4000302780013c0b30011c0b300ee09070027
:1060f4000000eb00704b88004e0090000000e900a7
:10610400400798004e0090000000e8004007980007
:10611400ce00900020002000808f5000c6ff360083
:1061240001003700000000004f0478000080fa00ee
:10613400000006002c00fa00301798004117980060
:1061440052179800760247003e11900012407800e2
:106154008082fb00924190008381fb00c819dd001e
:106164008581710003007800a24190008381fb00c7
:10617400324190000281fb004811dd0003017100ef
:1061840082007800008abe0076004700ce1090009e
:106194001101be002200980033009800f600470069
:1061a4000040eb0080489800f600470060c0b30050
:1061b4009048980076004700de1190005300980044
:1061c4007600470050009000bab1020000000000c1
:1061d400f6004700d000980076004700c100200078
:1061e40032b20200000000000080ea00101798009c
:1061f4005e109000c48a020000000000201798007e
:106204009e1090002e109000808f500004003200e9
:1062140094860200000000001000200022003700d5
:106224000000eb00ae070200010000000e80e80051
:1062340041012000be8d0200000000000e80e80035
:10624400610307000e80e800600090004400de0057
:106254006f406000210020000100dd00744f5000f9
:106264009e4078000180fb00de109000008050000a
:1062740074005000501798000e80e800be10900083
:10628400230207008000eb00810f5000030032005e
:106294000e80e800de1090002c04070094860200b3
:1062a40000000000100020000080fa00000006003a
:1062b4002a00fa00006f9800116f98006df707002c
:1062c4000e6890000080fb00610060008040780050
:1062d4000040eb0080cf5000050032008b69a8001d
:1062e4008e689000e0cfb30000c06000006f98009b
:1062f4008aa9a9008ac9a9008ae9a9008b29a90049
:106304008b49a9008b09a900000000007e860200c9
:10631400000000008000eb00810f5000fbff320002
:106324000e6890000080fb00e60060000000eb00b7
:10633400808f5000030032000000eb00000f780053
:1063440088003700c14b8000d0488000808f500007
:1063540003003a000000eb00000f780070003700e3
:10636400c14b8000d0488000808f50001c00360054
:10637400c14b8000d0488000008f5000014980004c
:106384001e007800808f5000020031000049800018
:10639400000f7800914980001e007800808f500023
:1063a4000300310091498000010f78008b49a80057
:1063b4008ec9bf00d14880001e0278008041780059
:1063c400010178008040eb0010a02000360907008e
:1063d400d04880001e004000d0488800500037009c
:1063e400a14b8000d0488000808050007c00470092
:1063f400510098007c004700d0009000c04b800002
:1064040080804000904b8000008f50000149800044
:106414001e007800808f5000020031000249800085
:10642400020f7800914980001e007800808f500090
:106434000300310093498000030f78008b49a800c2
:106444007c004700d00090001e007800808f500030
:10645400030036007c0047009e007800510098003d
:106464007c004700500190008ec9bf00d1488000d5
:106474000202780080417800010178008040eb003e
:1064840010a02000080907007c004700500090007d
:106494009e0010007c004700510098007c004700db
:1064a400d00090000000eb00808f50000f003200fd
:1064b4007c004700500190008ec9bf00914b8000c2
:1064c400a44b8000d34880000302520013a0200094
:1064d40083024200020278008041780001017800c2
:1064e4008040eb0005007800ef080700d0488000ea
:1064f4001e004000d0488800d1488000a04b800096
:10650400808f500006003900d1488000924b8000f3
:10651400a04b80000000510000804000d04888005b
:10652400514c800000802000808060000000eb005f
:10653400808f50000b003200014980001e0078005b
:10654400808f500007003200914980001e007800bf
:10655400808f5000030032000e6890000004a000f9
:10656400006f98009e0078000000eb00808f5000c0
:1065740006003a000e6890000080fb00e300600013
:106584000000eb00808f50002200320000498000a0
:106594001e005000004988009e0078000000eb00b7
:1065a400808f5000030032000e6890000034a00079
:1065b400006f98001e6890000080fb00610060007e
:1065c400804078000040eb0080cf5000060032008d
:1065d4000040eb0034e9b70040422f0001002000e6
:1065e40070488800814888009a1002000100000069
:1065f4000001be0070488000814880000200400015
:1066040083804800004c8800114c88008a89a800c7
:106614003e0037001e6890000080fb00e20060002e
:106624000000eb00808f500016003200504c8000b8
:10663400674060000040e800674060000080fb00a5
:1066440067006000524c800081ff2f0081006100d0
:1066540000807000504c880092488000a34880005d
:106664000080eb008080eb00020040008380480043
:1066740090488800a148880010002000000f78008e
:1066840022003700504c8000f00060000000eb0056
:10669400808f50001d0032001e6890000080fb00b7
:1066a400e10060000000eb00808f50000e003a0013
:1066b40041932000914078000040eb0080cf5000cf
:1066c4000900320034c9bf000040e90034e9b700d2
:1066d40070488000814880008100d1000080d30090
:1066e40070488800814888009a1002000100000068
:1066f4000001be0070488000814880000200400014
:1067040083804800004c8800114c8800f1488000c8
:106714006400470001087800e148800064004700f5
:106724001100980090488000a1488000640147004f
:106734002001980031019800b0488000c1488000d1
:10674400640147004001980051019800640047002b
:1067540060019000f1ff2300810061006100980056
:10676400640047006001900001ff2f008100610078
:1067740061009800640047000e6990005248980038
:10678400640047008000eb001108980092488000e4
:10679400a34880001e007800010020000200400091
:1067a4008380480090488800a14888000e689000c3
:1067b4000080fb00e20060000000eb00808f5000ce
:1067c400230032000e6890000080fb00f00060009f
:1067d4000000eb00808f500004003a006401470081
:1067e4006000b80040019800510198008049800081
:1067f400e20060000000eb00808f50000b003200cc
:106804006400470020019000b00190000080eb007c
:106814008080eb0002004000838048006401470050
:106824002001980031019800090037009248800047
:10683400a348800010002000010020000200400056
:106844008380480090488800a14888003029a80027
:106854000e6890000080fb006100600080407800ba
:106864000040eb0080cf5000010032003009a80046
:10687400e14b8000f04b8000808f50000a0039000b
:10688400b14b8000a04b800080805000f24b800010
:10689400e04b80000000510080804000640047000d
:1068a4007100980006003700f14b8000e04b800037
:1068b400008050008000e9006400470071009800e7
:1068c400d286020000000000100798009e0090008d
:1068d400f0032000808f500003003e000000eb0016
:1068e40010079800030037001e0090000004b10058
:1068f4001007980064004700f00090001e0090000c
:10690400808f5000030036009e0090006400470012
:106914007100980064004700ab0107009e017800f5
:10692400748f41006400470060019000f1f02f0073
:1069340001016100010520008100710061009800df
:106944000e6890000080fb00e20060000000eb0095
:10695400808f5000170032001e007800640f400042
:1069640020c0b300005f980040c0b300105f9800df
:1069740020802100500f98006400470060009000c0
:106984004400de006f4060000040e8006f4060009b
:10699400e40047000080fb006f0060004400dd005d
:1069a400e1019000f2f02f0002816100000071000b
:1069b400e0009800fc01470002d320001241780057
:1069c4000282fb0012d32000124178000281fb00f6
:1069d4004811dd00040171000200780022d3200078
:1069e400124178000282fb0032d320001241780069
:1069f4000281fb004811dd0004017100820078006f
:106a04008089be007c004700224980003349800011
:106a14002200980033009800fc0047000040eb007f
:106a240080489800fc00470060c0b300904898007c
:106a34007c0047009e017800530098007c004700ca
:106a440050009000bab1020000000000fc004700b2
:106a5400d00098007c004700c100200032b2020040
:106a6400000000008080ea006400470001089800ec
:106a7400909d2000008a0200000000001e017800a2
:106a840061c0b3004092200004070200010000002e
:106a94006400470041012000f08e02000000000065
:106aa4000e6890000080fb00e20060000000eb0034
:106ab400808f50000400320078004700410020001d
:106ac400f08e020000000000d09e2000328a0200f6
:106ad400000000001e007800c48a020000000000cc
:106ae40010079800d09f2000008a020000000000d8
:106af4000e80e80021002000f08e0200000000005b
:106b04008e880200000000000080fa0000000600e9
:106b14000a00fa0030079800410798003e009000f0
:106b2400900090000000eb00808f500002003a00bb
:106b34000000eb0022013700e0cfb30010479800bb
:106b4400ce009000214090000081fb003140900075
:106b54000080fb004800dd00020070008000780027
:106b64004e009000904178000381fb00104090009b
:106b74000080fb004800dd000200700080804000bf
:106b84003e00900010007800808040003e0090009d
:106b94001000900000806800200798000040eb007f
:106ba400004f78003d0037001e40780004f50700d0
:106bb400414c8000d0002000808f50003100320012
:106bc400414c800040002000808f500008003a00b3
:106bd400614c80003e00900010009000808f5000b7
:106be4002a003a001e407800104798002a00370017
:106bf400614c80002e009000808f500025003a00e8
:106c04001cf507003e00900090009000f0488000c2
:106c1400808f500020003a003e00900090007800e1
:106c2400e0488000808f50001b003a004e01900025
:106c3400924178000382fb00924190008381fb0023
:106c4400c819dd008481710003007800a24190001e
:106c54008381fb00324190000281fb004811dd007a
:106c640003017100820078002249800033498000ca
:106c7400820f5000838f580007003a001000200054
:106c8400cf003700000000000300370000000000c0
:106c940001003700000000001e4fe8009e4078000d
:106ca40080c0b30080cf5000bfff36009e409000ec
:106cb400e0cfb30080cf5000180032001e40900097
:106cc400bff40700ebf407009e409000e0cfb30050
:106cd40080cf5000110032002e009000604c8800dc
:106ce400a2002000ce00900040922000940a0200ee
:106cf400000000003e00900010007800e04888008a
:106d04003e00900010009000f0488800904b8000f6
:106d1400d048880010002000a90037003e009000f1
:106d2400e000900000202000808060000000eb0064
:106d3400808f500002003a000000eb00a0003700f2
:106d4400714b80000000eb00808f50000200320085
:106d54000000eb009a0037000000eb0010079800d9
:106d64004b0037001e0090007400b900000078004a
:106d7400f000400060932000008040009000780004
:106d84000000eb00808f5000460032001e0090008f
:106d94007400b90000007800f00040006093200007
:106da40000804000900078003e00900010009000a9
:106db400808f50002e003a001e0090007400b9002d
:106dc40000007800ea00400060932000008040004a
:106dd400900078003e00900010007800808f5000f2
:106de40025003a001e0090007400b900800078006d
:106df40060932000008040001001be004e0290000d
:106e0400144078000083fb00944290008582fb00cc
:106e1400c82add008682720005007800a442900032
:106e24008582fb00344290000482fb004822dd008e
:106e34000502720084007800800f5100818f590090
:106e44000f003a00a61002000100000000017800c3
:106e54001e0090007400b900800078008094200027
:106e640000804000020878000000eb005400370066
:106e7400000000000300370000000000010037009c
:106e8400000000001e0090000000e80010079800b9
:106e94009e00900020002000808f5000b1ff36003b
:106ea40001003700000000000040eb00004f7800b4
:106eb4003e0037001e40780041f40700504c80002b
:106ec400e80060000000eb00808f500033003200c7
:106ed40068f40700f14880003e0090001000900024
:106ee400808f50002f003a001e0090007400b900fb
:106ef400800078006093200000804000a200200001
:106f0400ce009000940a0200000000003e009000b1
:106f1400100178001e0090007400b9008000780011
:106f24000094200000804000020878003e00900099
:106f3400b0009000200090001e0190007411b90070
:106f44008201780022942000028141000089be0061
:106f54003e009000100190001e0090007400b900e3
:106f640080007800609420000080400002087800cf
:106f7400a610020001000000000178001e0090002d
:106f84007400b900800078008094200000804000e4
:106f9400020878000000eb00090037000000000040
:106fa40001003700000000001e4fe8009e407800fa
:106fb40080c0b30080cf5000beff36000000eb005d
:106fc4000080fa00000006000200fa00000f7800ba
:106fd4001e00780010007800bab102000000000022
:106fe4009e007800800878001e0078001000900051
:106ff400bab10200000000009e00780090009800e2
:107004001e007800b000900020009000d4b102006f
:10701400000000001e017800200198003101980052
:107024001e007800d000900040009000d4b102000f
:10703400000000001e0178004001980051019800f2
:107044001e00780070009000bab102000000000039
:107054009e007800f00098001e0078000008900060
:10706400bab10200000000009e0078008008980079
:107074001e00780010089000bab102000000000061
:107084009e007800900898000080fa000000060036
:107094000000fa00881f7800f6f30700f04880002b
:1070a400604c8800904b8000c04b8800904b80005f
:1070b400d04b8800a04b8000e04b8800a04b8000a0
:1070c400f04b8800504c8000e80060000000eb00aa
:1070d400808f500002003200400020000100370081
:1070e400d0002000404c88008a09a9008a29a90000
:1070f4008a49a9008a89a9008aa9a9008ac9a9007c
:107104008ae9a9008b09a9008b29a9008b49a90048
:107114008b69a9008b89a8003009a9003029a9002e
:107124003069a9003089a900904b8000d0488800bc
:107134002891200026aa020000000000000c78001c
:107144002891200026aa02000000000010049800e4
:107154000080eb007049880010002000004988007e
:107164004f0478000080fa00000006000400fa00d2
:10717400881f7800c0002000ae0702000100000054
:107184008a8d020000000000004f78001e40780045
:107194008080fb00000f2000008060004280de0041
:1071a40000407800744f50009e4078000040eb008f
:1071b40080cf500002003a00802120006000370098
:1071c400710020000000eb00be8d020000000000f2
:1071d400470037008a8d0200000000001047980025
:1071e4009e4090000040eb0080cf50004a003200e7
:1071f4009e40900010c0b30080cf50003b0032008e
:107204009e40900020c0b30080cf500022003a007e
:107214009e40780020c0b30080cf5000400036006c
:107224000000eb00100798008a8d020000000000a7
:10723400104798009e40900040c0b30080cf50009b
:1072440009003a000e80e8000004e8008a8d02007c
:1072540000000000004c78000e84e8008a8d0200d3
:1072640000000000004c78009e0090007021200077
:10727400808f50002c0036009e009000405b200060
:10728400808f500002003600405b20002c00370045
:107294001e0090002a0037009e40780010c0b30002
:1072a40080cf5000220036008a8d020000000000ca
:1072b400104798001e4090009e40780080cf5000f8
:1072c4001d0039001e4090000080fb008000780003
:1072d4000000eb00be8d0200000000009e4078001c
:1072e4001e40900000cf5000010037000000000055
:1072f4009e4078000180fb000000ea004f00de00a1
:10730400804078001e4fe9000040eb0080cf500021
:10731400b0ff3a0009003700000000000700370002
:1073240000000000050037000000000003003700e3
:107334000000000001003700000000008021200050
:107344004f0478000080fa00000006002200fa00d2
:10735400700f9800011798007e089000d0489000a4
:10736400015798007e08900040019000d0019000e1
:1073740042079800530798007e089000200190006f
:10738400b0019000120f9800230f98008a09a900f9
:107394008a29a9008a49a900504c8000f0006000a5
:1073a4000000eb00808f500009003a009a100200a0
:1073b400010000000001be0080962800910020001a
:1073c4000200400083804800004c8800114c880073
:1073d400404c800041002000810f50000400320026
:1073e40051002000810f500030003200810037002e
:1073f4000e5090000080fb00e40060000000eb00f1
:10740400808f50000200320021ff07006304370020
:107414000e5090000080fb00f00060000000eb00c4
:10742400808f5000090032004e009000de00900072
:1074340090488800a14888008040eb0040c0b30019
:107444009bfb070012ff0700540437000e50900006
:107454000080fb00e20060000000eb00808f500021
:10746400100032001e099000ae09900010002000a8
:10747400010020000200400083804800b0488800da
:10748400c148880039ff07009049880011c0b30043
:1074940020c1b30086fb070060002000404c880038
:1074a4003e043700fafe07003c0437000e509000fb
:1074b4000080fb00e40060000000eb00808f5000bf
:1074c40023043a000e5090000080fb00f00060009e
:1074d4000000eb00808f50001700320092488000bb
:1074e400a34880004e009000de009000800f510001
:1074f400818f59001000320092488000a348800018
:10750400120f9800230f98004e009000de009000a8
:1075140090488800a148880011c0b30040c0b3005f
:1075240063fb07001e099000ae0990009248880092
:10753400a3488800190437000e5090000080fb0017
:10754400e20060000000eb00808f50000204320073
:107554001e099000ae0990001000200001002000d8
:107564000200400083804800b0488800c148880079
:107574007e0890007000900000498800fbfe070020
:10758400904988000e5090000080fb00f0006000dd
:107594000000eb00808f50001000320011c0b300d7
:1075a40000c1b30042fb070070002000404c88007b
:1075b4009a100200010000000001be00809628001d
:1075c400910020000200400083804800004c8800a5
:1075d400114c88008a89a900f003370011c0b30058
:1075e40020c1b30032fb070060002000404c88003b
:1075f400ea0337008e119000630798000e50900044
:107604000080fb0061006000804078000040eb00d7
:1076140080cf5000030032006e0090000000e800ac
:10762400600798000e5090000080fb00e2006000ac
:107634000000eb00808f5000030032006e009000c9
:107644000000e80060079800e14b8000f04b8000e8
:10765400808f500009003900b14b8000a04b80009e
:1076640080805000f24b8000e04b8000000051000d
:10767400008040003007980005003700f14b80007f
:10768400e04b8000008050000000e90030079800c3
:10769400b0488000c14880001e099000ae099000e7
:1076a4000000510081805900300f9800410f98006c
:1076b4003e089000500f98000000eb0070079800ff
:1076c400ee0090000000eb00808f50003900320083
:1076d400be0090000000eb00808f50004d0032008f
:1076e4003e099000ce0990006000b800800f510060
:1076f400818f59000a0035003e0090006101b800f6
:107704003e089000ce089000800f5100818f5900f0
:1077140003003600100020007007980015003700a1
:107724006e0090006101b8003e089000ce08900001
:1077340002014000838148006000b800800f5100be
:10774400818f59000b003400be0090006e00900041
:10775400008050006101b9003e089000ce089000fe
:10776400800f5100818f5900020035001000200065
:10777400700798003e0090006101b8003e08900038
:10778400ce089000800f5100818f590021003400f1
:10779400de0890006e009000808040000000eb0046
:1077a400808f50001b0034001000200070079800e8
:1077b400180037003e099000ce0990006000b80020
:1077c400800f5100818f590003003a0010002000ff
:1077d400700798000f0037003e099000ce09900012
:1077e4006000b800800f5100818f590009003500f6
:1077f4003e0090006101b8003e089000ce08900061
:10780400800f5100818f59000200360010002000c3
:1078140070079800fe0090000000eb00808f50007d
:107824000a003a000e5090000080fb00e400600063
:107834000000eb00808f500049033a0011c0b300f0
:1078440000c1b3009afa0700540337000e509000a9
:107854000080fb00e60060000000eb00808f500019
:10786400020032000afe07004c0337000e5090005d
:107874000080fb00f00060000000eb00808f5000ef
:1078840039033200404c80006101b800a0ff2f0092
:10789400f1ff2f00020040008380480062002000b6
:1078a40003002000820f5000838f58006f013e00b8
:1078b40000600100060037001e0037001d0037007d
:1078c4001c0037001b0037001a0037005a0137002c
:1078d40092488000a34880004e009000de00900093
:1078e400800f5100818f59001000320092488000af
:1078f400a3488000120f9800230f98004e009000b8
:10790400de00900090488800a148880011c0b300b0
:1079140040c0b30066fa07001e099000ae0990004b
:1079240092488800a34888001c0337007000200098
:10793400404c8800c14b8000d0488000008050003b
:1079440020079800ae0090000000eb00808f5000ec
:1079540006003d00a14b8000904b80000080500049
:10796400ae009000008040002007980092488000fc
:10797400a34880002e00900001002000001f410059
:10798400019749004e019000de0190001e00be00e8
:107994000000510081805900008fbe001e01be000e
:1079a4006000b800800f5100818f59001700340027
:1079b40080498000e10060000000eb00808f5000ef
:1079c400060032001e01be0010002000010020004d
:1079d400800f5100818f5900040032008040eb0079
:1079e40000c1b30032fa0700ec0237004e019000e8
:1079f400de0190000080eb008080eb00020040007c
:107a040083804800400798005107980092488000fe
:107a1400a3488000d1488000d04b800000805000f3
:107a2400cf80de00001f510001975900d14880002b
:107a3400d04b8000808f500006003100a14b8000a5
:107a4400904b800000805000010020001e1f100099
:107a54001e9718004e009000de0090001e1f50007c
:107a64001e9758001e01be006000b800800f510030
:107a7400818f590051003400a14b8000904b80004d
:107a8400008050006101b8001e00be00800f51004c
:107a9400818f5900490039003069a9003089a90053
:107aa4008b09a900d34b800023079800d14b800099
:107ab4001e00780000804000d04b8800d148800030
:107ac4002e009000808f500011003900d1488000b2
:107ad400d04b8000808f50002300310092488000fa
:107ae400a3488000d14b8000d04880000080500023
:107af4000100200002004000838048009048880074
:107b0400a1488800d04b8000d04888001600370078
:107b1400d1488000a24b8000904b800000005100af
:107b24000080400020079800d14b80002e00900078
:107b3400808f50000c00360092488000a3488000db
:107b4400d14b80002e0090000080500001002000e6
:107b5400020040008380480090488800a1488800c3
:107b6400d04b8000d0488800d14b8000a04b8000cf
:107b7400808f500006003900d14b8000924b80006a
:107b8400a04b80000000510000804000d04b8800d2
:107b9400d1488000a04b8000808f50003200390013
:107ba400d1488000924b8000a04b8000000051001f
:107bb40000804000d04888002b003700d14b800063
:107bc400d0488000808f5000270032008049800018
:107bd400e80060000000eb00808f500021003200bc
:107be40080498000f00060000000eb00808f5000ae
:107bf4001b00320092488000a3488000d1488000d6
:107c0400d04b800000805000cf80de000000510087
:107c14008180590090488800a1488800d14880009c
:107c2400d04b8000808f50000a00310092488000c1
:107c3400a3488000a14b8000904b8000008050003e
:107c4400cf80de00000051008180590090488800f8
:107c5400a1488800d04b8000d04888008b49a800f8
:107c64003089a8003069a800d14b8000c04b800047
:107c7400808f50001f003a00514c8000008020008b
:107c8400808060000000eb00808f50000b003a0001
:107c94009a100200010000000001be008096280036
:107ca400910020000200400083804800004c8800be
:107cb400114c88008a89a9000e0037009248800080
:107cc400a34880004e009000de009000800f510019
:107cd400818f590007003a0080498000e10060006c
:107ce4000000eb00808f5000020032008a89a90056
:107cf4008b69a9007e08900070019000ce0190006d
:107d040090488000a1488000000078000080510065
:107d140000004100600f9800014980000000eb0062
:107d2400808f500005003a00ee0890000000eb0040
:107d3400808f5000010032008b29a8006e0890004b
:107d440000498800414c800080002000808f500052
:107d540019003a0092488000a34880004e00900029
:107d6400de009000800f5100818f590041003a00dd
:107d740080498000e10060000000eb00808f50002b
:107d84003e0032009a100200010000000001be0013
:107d9400404b2c004100200002004000838048003a
:107da400004c8800114c88008a89a80090002000ab
:107db400404c880036003700414c80009000200081
:107dc400808f50000f003a000e5090000080fb009e
:107dd400e10060000000eb00808f500029003a00b1
:107de4004e019000de01900092488800a34888006c
:107df4008040eb0040c1b3002df90700a4fc07004c
:107e0400e6013700414c8000a0002000808f500024
:107e14001e003a0092488000a34880004e00900063
:107e2400de009000800f5100818f5900d0013a008c
:107e340097fc0700d901370092488000a3488000ce
:107e4400100020000100200002014000838148004e
:107e54004e009000de009000800f5100818f590089
:107e6400c5013a008afc0700cc013700000000007d
:107e74000700370000000000050037000000000084
:107e8400030037000000000001003700000000007c
:107e94000e5090008080fb00000220008080600073
:107ea4000000eb00808f5000b5013a00414c800087
:107eb400b0002000808f5000b3013200414c80009c
:107ec400a0002000808f5000b1013200414c80009e
:107ed400c0002000808f5000af0132008e1090004f
:107ee4000000eb00808f500022013200de08900079
:107ef4000000eb00808f500080003c007e08900062
:107f0400600090004400de006f4060000080fb00d1
:107f14004200dd00800078005e0890000080500080
:107f2400ae070200010000008e1090005e08900071
:107f340000804000001798008e1090003e009000d2
:107f4400808f500002003600be0190000317980095
:107f5400b2488000c34880000e1090000100200049
:107f64000200400083804800b0488800c14888006f
:107f7400e14b80000e10900080804000b04b8000e8
:107f8400808f50001f003600b14b8000e04b800012
:107f9400008050000000e800200798008ec9bf0050
:107fa400e54b80002e0290008041eb000081eb0045
:107fb40080407800050078003b0207008e10900096
:107fc4002e009000808050008ec9bf00a54b800019
:107fd400010278008041eb000081eb0080407800d2
:107fe4000500780030020700a14b80000e119000bc
:107ff4002e0090000000510000804000e04b8800fb
:108004000c0037008ec9bf00e54b80000e129000b3
:108014008041eb000081eb0080407800050078008f
:1080240021020700e14b80000e1090000080400008
:10803400e04b8800714980000080eb00808f500085
:10804400cc00320070498000800078000e1090004f
:1080540000805000704988001149800070498000f8
:108064000080400020079800ae0090000000eb0064
:10807400808f500003003d000080eb0070498800b1
:10808400bc003700714980000000eb00808f500075
:10809400b8003c00b2488000c34880002e00900025
:1080a400010020000200400083804800b04888009e
:1080b400c1488800e14b80002e0090000080400001
:1080c400e04b8800e14b8000b04b8000808f500073
:1080d40007003600e14b8000b24b8000a04b8000cb
:1080e400000051000080ea0000804000e04b88005e
:1080f4000080eb00704988009e003700de08900085
:108104000000eb00808f50009a0034008e10900025
:108114005e089000808040003e009000808f5000f8
:1081240004003600be0090005e08900000805000fd
:10813400001798007e089000600090004400de0064
:108144006f4060000080fb004200dd00ae070200cb
:1081540001000000e14b80005e0890008080400038
:108164000e10900080804000b04b8000808f500043
:1081740032003600b14b8000e04b8000808050001c
:108184005e0890000000ea00008040000000e80063
:1081940020079800ae0090000000eb00808f500094
:1081a400160035008ec9bf00e24b8000de08900047
:1081b400810241002e0290008041eb000081eb001f
:1081c4008040780005007800b70107008e10900009
:1081d4002e009000808050008ec9bf00a54b800007
:1081e400010278008041eb000081eb0080407800c0
:1081f40005007800ac0107001a0037008ec9bf00e3
:10820400e24b8000de08900001014100b34b800086
:10821400a14b8000818051008180ea0081024100ed
:108224000e1290008041eb000081eb00804078004a
:10823400050078009c0107000a0037008ec9bf00c2
:10824400e24b8000de089000810241000e12900093
:108254008041eb000081eb0080407800050078004d
:1082640091010700714980000080eb00808f50006d
:1082740005003a005e089000704988000e109000d6
:10828400104988003b003700704980008000780066
:108294005e089000808f50001c003600de089000bd
:1082a4000e1090008080400070498000000178002a
:1082b4001049800000004100808f500006003e00fd
:1082c400de0890000e10900080804000704980000d
:1082d400808f5000030031008e10900011498800f7
:1082e4000700370070498000800078001049800042
:1082f400808040005e089000008050001049880093
:108304005e089000704988001a003700de0890006b
:108314000e109000808040007049800000017800b9
:108324001049800000004100808f50001100360089
:1083340070498000800078001049800080804000ef
:108344005e089000808f50000a00390011498000b7
:108354005e0990000e1090000001410070498000f9
:1083640000015100104980000000510000804000cd
:1083740010498800ee0090000000eb00808f500050
:108384001e003200414c800070002000808f50009d
:1083940002003200e04b8000f04b8800514c80001a
:1083a40000082000808060000000eb00808f5000f7
:1083b4000500320011c0b30000c1b300bcf70700d0
:1083c4002cef07000d0037008ae9a800514c80000b
:1083d40000042000808060000000eb00808f5000cb
:1083e40006003a008ac9a800a61002000100000095
:1083f4000000780078004000304c88000e50900057
:108404000080fb0061006000804078000040eb00c9
:1084140080cf500061003200b2488000c348800021
:108424001000200001002000020140008381480068
:108434006e0090006102b8001e089000ae08900023
:108444000400400085804800800f5100818f59004e
:1084540052003a00b2488000c34880001000200057
:10846400010020000200400083804800b0488800da
:10847400c1488800404c80006101b800a0ff2f0073
:10848400f1ff2f00020040008380480032002000ea
:1084940003002000820f5000838f580027003e0005
:1084a4000060010003003700080037000f003700a8
:1084b4001d003700c0002000404c880011c0b300ec
:1084c40010c1b3007af7070034003700b000200071
:1084d400404c8800a6100200010000000000780053
:1084e4000003b000304c880015003700924880002b
:1084f400a34880004e009000de009000800f5100e1
:10850400818f590005003a008040eb0000c1b300a0
:1085140067f70700defa070020003700a0002000fc
:10852400404c8800060037008040eb0000c1b300d7
:108534005ff70700d6fa07001800370000000000b4
:1085440011c0b30000c1b30059f70700130037008e
:108554000000000011003700000000000f00370089
:10856400000000000d003700000000000b00370081
:108574000000000009003700000000000700370079
:108584000000000005003700000000000300370071
:108594000000000001003700000000000080fa0025
:1085a400000006000e00fa0060479800410798009a
:1085b40052079800434f9800ee40900080c0b300eb
:1085c40080cf5000020036000000eb00b4003700fa
:1085d4006e4090007aee0700ce0090000000eb00a1
:1085e400808f500002003a001000200040079800dd
:1085f400b14b8000904b8000008050000000e900e7
:1086040020079800ce0090005e009000808040001b
:108614002e009000808f5000020036000000eb0016
:108624009f00370093ee07004e4890000080fb0047
:10863400e30060000000eb00808f500003003a006c
:108644004e4890003040b300404f98005e009000c8
:1086540010079800ce0090005e009000008040005b
:10866400ae00900000805000200798004e48900013
:108674000080fb00e20060000000eb00808f5000ef
:10868400110032004e4890000080fb006100600041
:10869400804078000040eb0080cf5000060032009c
:1086a4002e0090000000d1009e0090000080400049
:1086b40010079800040037009e0090002e009000e0
:1086c4000080400010079800914b80001e0090002d
:1086d400008040000000e80020079800e04b800084
:1086e400000f7800714980000080eb00808f5000fb
:1086f4000e0032007049800080007800104980002c
:10870400008040001e0f4000b14b80001e00780026
:10871400808f500005003100b14b8000a04b8000d9
:10872400008050000080ea001e0f4000f14b8000e2
:108734001e007800808f500011003100f14b800042
:108744002e009000808f5000260031004e4890008b
:108754000080fb00e40060000000eb00808f50000c
:10876400020032000000eb004d0037002e009000a4
:10877400f04b88002e009000e04b88001900370071
:10878400f14b80001e007800808f500011003600ed
:10879400a14b80002e009000808f5000110031000a
:1087a4004e4890000080fb00e40060000000eb00f5
:1087b400808f5000020032000000eb0038003700c8
:1087c4002e009000f04b88002e009000e04b8800b3
:1087d400040037002e009000f04b88002e0090001b
:1087e400e04b8800f14b80001e007800808f500021
:1087f4001b0036004e4890000080fb00e40060003f
:108804000000eb00808f500015003200a04b800068
:108814009e011000e198200091407800a24b800056
:108824008ec9bf000302780081417800804078003f
:108834002e0090001c000700e14b8000f04b8000ec
:10884400808f500006003100e14b8000a04b800077
:108854002e0190000000510000804000e04b880091
:108864002e009000a04b8800904b8000d0488800d8
:10887400904b8000d04b8800904b8000c04b880008
:10888400414c800070002000808f500003003a00ab
:1088940011c0b30000c1b30085f60700100020002a
:1088a4000080fa00000006000a00fa00000f7800b9
:1088b40021479800220798006347980044079800ce
:1088c4006e4090000080fb008000eb00810f5000a0
:1088d4001e00320011002000810f500040003a00b9
:1088e4002e4090000080fb008000eb00810f5000c0
:1088f4000900320011002000810f500035003a00b9
:10890400ae0090001e0078004e019000940a020010
:10891400000000000c0037009e0078000080eb008f
:10892400808f5000030032001e007800008a02008d
:10893400000000002e009000ce009000f08e020097
:108944000000000000000000250037002e409000c9
:108954000080fb008000eb00810f50000f0032000c
:1089640011002000810f50001c003a00ae0090005e
:108974000080eb00808f5000030032002e00900036
:10898400328a0200000000001e007800ce00900031
:10899400be8d0200000000000c0037004e01900064
:1089a400ae0090001e007800788b020000000000ea
:1089b40000000000748d0200000000008000eb0045
:1089c400810f5000fbff3200000000000000000097
:1089d4000300370000000000010037000000000021
:1089e4000080fa00000006000400fa00008fbe00b8
:1089f4000080eb008080eb003e014000ae81480027
:108a04000200be008204200003002000820f5000f8
:108a1400838f58001c013e000060010048003700ad
:108a24004a0037004c0037004e0037004f00370033
:108a34005100370054003700570037005a00370000
:108a44005d003700600037006300370066003700c0
:108a5400680037006c00370070003700740037007e
:108a6400780037007c00370080003700840037002e
:108a7400880037008a0037008d00370090003700e7
:108a84009300370096003700990037009b003700a9
:108a94009d0037009f003700a1003700a300370076
:108aa400a5003700a7003700a9003700ab00370046
:108ab400ad003700af003700b1003700b300370016
:108ac400b5003700b7003700b9003700bb003700e6
:108ad400bd003700bf003700c2003700c5003700b3
:108ae400e9003700c7003700e7003700e600370029
:108af400e5003700e4003700e3003700e200370008
:108b0400e1003700e0003700df003700de00370007
:108b1400dd003700dc003700db003700da00370007
:108b2400bb003700be003700c1003700c400370067
:108b3400c7003700ca003700cd003700cf00370028
:108b44007670020000000000da003700a0b62800aa
:108b5400c10c0700d7003700b87002000000000005
:108b6400d4003700d5000700d20037001c6d020086
:108b740000000000cf00370070002000f06d0200fc
:108b840000000000cb00370060002000f06d020000
:108b940000000000c700370050002000f06d020004
:108ba40000000000c300370040002000f06d020008
:108bb40000000000bf00370030002000f06d02000c
:108bc40000000000bb00370020002000f06d020010
:108bd40000000000b700370010002000f06d020014
:108be40000000000b30037008c6f0200000000009a
:108bf400b00037001100200040002000a26e0200e7
:108c040000000000ab0037008000eb0040002000b3
:108c1400a26e020000000000a60037001100200030
:108c240030002000a26e020000000000a100370006
:108c34008000eb0030002000a26e02000000000063
:108c44009c0037001100200020002000a26e0200ca
:108c540000000000970037008000eb002000200097
:108c6400a26e0200000000009200370011002000f4
:108c740010002000a26e0200000000008d003700ea
:108c84008000eb0010002000a26e02000000000033
:108c940088003700606d0200000000008500370086
:108ca4000000eb00f06d02000000000081003700be
:108cb4000000eb007a6d0200000000007d00370028
:108cc400100020007a6d02000000000079003700d7
:108cd400200020007a6d02000000000075003700bb
:108ce400300020007a6d020000000000710037009f
:108cf400646f0200000000006e003700fc70020088
:108d0400000000006b003700dc740200000000006b
:108d1400680037004c740200000000006500370052
:108d24006674020000000000620037003274020022
:108d3400000000005f0037003874020000000000eb
:108d44005c0037003e740200000000005900370048
:108d54001875020000000000560037005873020026
:108d640000000000530037003c72020000000000c5
:108d74005000370056720200000000004d0037001a
:108d84007c720200000000004a003700a872020052
:108d94000000000047003700d47202000000000009
:108da4004400370000730200000000004100370057
:108db4002c730200000000003e0037001074020013
:108dc400000000003b00370018740200000000009f
:108dd400380037000000eb0044740200000000007b
:108de400340037001000200044740200000000002a
:108df400300037002000200044740200000000000e
:108e04002c00370050b72800130c07002900370046
:108e14000000eb0000740200000000002500370091
:108e24001000200000740200000000002100370040
:108e34002000200000740200000000001d00370024
:108e44000000eb0008740200000000001900370065
:108e54001000200008740200000000001500370014
:108e640020002000087402000000000011003700f8
:108e7400a8740200000000000e003700c274020053
:108e8400000000000b00370001b82800f2cabf0040
:108e94000080fb00a2ae20004200dd000080e8005c
:108ea4000000410010407800420020002625020006
:108eb400000000000080fa00000006000000fa0034
:108ec400f2cabf000080fb00a1ae20004200dd001a
:108ed4000080e8000080400010407800e1c7b30043
:108ee40082240200000000000080fa000000060056
:108ef4000200fa00881f78000040eb00f2eab70095
:108f04002c003700f2cabf000080fb00a1ae200095
:108f14004200dd00008040008000eb000108780082
:108f2400f2cabf000084fb0084c0b3000305200024
:108f34000041eb006000b800762102000000000050
:108f4400a2ae2000c240dd00810041008180e80023
:108f54008048780000c0eb007ceab70000c0eb005a
:108f64007deab700f2cabf008080fb002008200021
:108f74000088b9008000780080ef21000080400064
:108f8400008a020000000000000f780080a6200084
:108f940021082000f08e0200000000001e0078006e
:108fa400008a020000000000f2cabf000040e8008e
:108fb400f2eab70021af20009140780010c0b3005e
:108fc40080cf5000cfff36000040eb00f2eab7003c
:108fd4004f0478000080fa00000006000200fa0046
:108fe4000040eb00004f78005a0037009e407800a4
:108ff4000180fb00a1ae20004200dd000080e800fb
:109004000080400090407800e0cfb30080cf500053
:109014004e0032009e4078000180fb00a1ae20008b
:109024004200dd000080e80000804000104078002d
:10903400ca220200000000008000eb00810f5000f3
:10904400290032001e40780048000700f2cabf0021
:109054000080fb00a1ae20004200dd000080400043
:109064008000eb0001087800c1a72000914078003f
:1090740000c0eb0080cf5000050032007ccabf0066
:10908400e6a002000000000000c0eb007ceab7008c
:10909400d1a720009140780000c0eb0080cf5000a1
:1090a400050032007dcabf00e6a0020000000000f7
:1090b40000c0eb007deab700f2cabf000080fb00ed
:1090c400a1ae20004200dd000080e80000804000e6
:1090d4001040780043c0b3000001eb0011002000f1
:1090e400d4420200000000009e4078000180fb0092
:1090f400a1ae20004200dd00008040009000780016
:109104000000eb00808f50000c003a009e40780075
:109114000180fb00a1ae20004200dd000080e800d9
:109124000080400010407800682602000000000023
:109134008000eb00810f5000050032001e407800d3
:109144000a00070037000700010037000000000094
:109154001e4fe8009e40780010c0b30080cf50003e
:10916400a2ff36000080fa00000006000400fa00a6
:1091740020479800f2cabf00ae40900080cf500054
:1091840025003200f2cabf008080fb0020082000c6
:109194000088b9008000780080ef21000080400042
:1091a400008a020000000000000f780080a6200062
:1091b40021082000f08e0200000000001e0078004c
:1091c400008a0200000000002e4090008080fb0016
:1091d400200820000088b9008000780080ef21007a
:1091e40000804000328a020000000000000f780076
:1091f40080a6200021082000be8d0200000000008f
:109204001e007800328a0200000000002e40900008
:10921400f2eab70001003700000000000080fa0005
:10922400000006001c00fa00881f780010002000cf
:1092340030079800f2cabf000080fb00a1ae2000f6
:109244004200dd0000804000100078000100200092
:10925400b200200003002000820f5000838f5800ca
:1092640076063e00006001000b0037004300370023
:1092740016023700f00237002c033700370337009b
:10928400de03370006043700f4043700f505370021
:109294001706370037063700f2cabf000080fb000c
:1092a400a1ae20004200dd000080e8000080400004
:1092b400104078006826020000000000000f7800cb
:1092c4009e0078000000eb00808f50004e063200b4
:1092d40040a82000c0538800f2cabf000080fb00f1
:1092e400a1ae20004200dd000080400011002000fb
:1092f4000108780000c0eb007feab7000040eb00f3
:109304007eeab7009a100200010000000001be00ce
:1093140040a52e00a10220000200400083804800e6
:1093240080538800915388000080eb008080eb001c
:10933400a0538800b15388006000b80040538800ef
:10934400515388000040eb00e8eab700f2cabf00be
:109354000080fb00a1ae20004200dd000080e80098
:10936400008040001040780053c0b3000001eb00bf
:1093740011002000d442020000000000f2cabf0025
:109384000080fb00a1ae20004200dd000080e80068
:1093940000804000104078000002eb008001eb00e8
:1093a4000001eb00a1c0b300462b02000000000046
:1093b4008080eb00810f500036003a00f2cabf00f3
:1093c4000080fb00a1ae20004200dd000080e80028
:1093d4000080400010407800d42702000000000004
:1093e4008000eb00810f50000b003a005000200079
:1093f40000548800f2cabf000080fb00a1ae200028
:109404004200dd0000804000710020000108780067
:109414000000eb00300798009a10020001000000e1
:109424000001be0080538000915380000000510071
:10943400818059000001be006000b800800f510017
:10944400818f5900f2053400f2cabf000080fb008e
:10945400a1ae20004200dd000080e8000080400052
:10946400104078001a23020000000000f2cabf0076
:109474000080fb00a1ae20004200dd00008040001f
:10948400b1002000010878000000eb0030079800cc
:10949400ea0537009a100200010000000001be0036
:1094a40040a52e00a1022000020040008380480055
:1094b4008053880091538800f2cabf000080fb00eb
:1094c400a1ae20004200dd000080e80000804000e2
:1094d400104078000002eb008001eb000001eb007b
:1094e40001c2b300462b020000000000000f780008
:1094f4009e00780050002000808f5000020036004b
:1095040050002000000f78009e00e800f2cabf005f
:109514000080fb00a2ae20004200dd000080e800d5
:1095240000004100104078000101780041a82000ab
:10953400122702000000000032002000a12a2900a6
:1095440040a82000600a02000000000080007800ab
:109554000000eb00808f500003003a000000eb0095
:10956400005488001700370042002000e12a290037
:1095740040a82000600a0200000000008000eb0008
:10958400810f500003003a001000200000548800ae
:109594000c0037007000200000548800f2cabf009d
:1095a4000080fb00a1ae20004200dd0000804000ee
:1095b40071002000010878000000eb0030079800db
:1095c4009e053700f2cabf000080fb00a1ae200058
:1095d4004200dd000080e800008040001040780078
:1095e4000002eb008001eb000001eb0001c2b300bc
:1095f400462b020000000000000f7800f2cabf00f2
:109604000080fb00a1ae20004200dd000080e800e5
:1096140000804000104078000002eb009e017800ba
:109624000001eb00f1c3b300462b02000000000070
:10963400100798009e0078001e009000810f5000d3
:109644000100360001007800000f7800900520002a
:109654009e007800808f50000c00360050002000df
:1096640000548800f2cabf000080fb00a1ae2000b5
:109674004200dd00008040007100200001087800f5
:109684000000eb00300798006c053700f2cabf00f9
:109694000080fb00a1ae20004200dd000080e80055
:1096a40000804000104078001e01780041a820008e
:1096b4001227020000000000100798009e0090008e
:1096c40040a82000808040000040eb0080487800e3
:1096d40040a820003007070040a82000de0a02004e
:1096e400000000001007980050a82000b2002000dd
:1096f400312b2900600a0200000000008000eb000a
:10970400810f500017003a0050a8200002600200a8
:10971400000000007feab700015480000000eb0065
:10972400808f500003003a0080002000005488001d
:10973400020037009000200000548800f2cabf00e5
:109744000080fb00a1ae20004200dd00008040004c
:1097540021002000010878000000eb003007980089
:10976400360537001e0090000000e900fc004000b0
:1097740080a620000080400090407800f0c2b30032
:1097840080cf50000400320050a82000f29e020056
:10979400000000007ceab700c1a7200091407800d7
:1097a40000c0eb0080cf50001f003a001e00900064
:1097b4000000e900fc00400080a62000008040007a
:1097c40090407800f0c2b30080cf5000080032000f
:1097d4009e00900040a8200080804000f0c2b300aa
:1097e400804878001e0090000000e80010079800f0
:1097f40041a820001e00900000804000a20020002c
:10980400e12b2900940a0200000000001e009000d1
:10981400690040001007980050a82000f29e020042
:10982400000000007ceab7001e0090008000e90000
:1098340040a820000080400040079800080037003e
:109844004e00900090407800e0c2b30080cf5000fa
:10985400080032004e0090000000e9004007980024
:10986400ce00900040a82000808f5000f4ff3a0002
:1098740001003700000000004e0090000000e800e6
:10988400400798000000eb00105488000f003700d8
:109894001054800080004000a0bb280000804000dd
:1098a40010007800800078004e00900020b1020083
:1098b400000000008040eb00814f5000080032009f
:1098c400105480000000e8001054880011548000f7
:1098d400a0002000808f5000edff3600010037000b
:1098e4000000000050a820000260020000000000f8
:1098f4007feab700c1a720009140780000c0eb00c8
:1099040080cf50000e0032007ccabf009ca702002a
:1099140000000000e20060000000eb00808f5000b7
:10992400070032007ccabf0086a9020000000000c4
:109934000000e80058a00200000000007deab70023
:10994400f2cabf000080fb00a1ae20004200dd008f
:109954000080e80000804000104078000002eb0026
:109964008001eb000001eb0001c2b300462b0200b2
:1099740000000000000f78009e0078000000eb005b
:10998400808f50003000320010c0b3007eeab70070
:10999400f2cabf000080fb00a1ae20004200dd003f
:1099a4000080e8000080400010407800ea00470092
:1099b400a0260200000000001e0fe900100620008f
:1099c4009e007800808f50000c003600500020006c
:1099d40000548800f2cabf000080fb00a1ae200042
:1099e4004200dd0000804000710020000108780082
:1099f4000000eb003007980090043700c853800043
:109a0400f2cabf000080fb00a1ae20004200dd00ce
:109a14000080e80000804000104078001e017800bb
:109a240041a82000122702000000000000004400aa
:109a3400c0538800c153800060c2b30080487800de
:109a44000100e800c0538800f2cabf000080fb0098
:109a5400a1ae20004200dd000080e800008040004c
:109a6400104078000002eb008001eb000001eb00e5
:109a7400a1c0b300462b020000000000000f7800d4
:109a84009e00e800f2cabf000080fb00a2ae2000e6
:109a94004200dd000080e800000041001040780032
:109aa400010178008000eb00122702000000000092
:109ab400f2cabf000080fb00a1ae20004200dd001e
:109ac400008040002100200001087800f2cabf0095
:109ad4000080fb00a1ae20004200dd000080e80011
:109ae40000804000104078000002eb008001eb0091
:109af4000001eb00a1c0b300462b020000000000ef
:109b0400000f78009e0078000080eb00808f5000ea
:109b140036003a00f2cabf000080fb00a1ae20006c
:109b24004200dd000080e800008040001040780022
:109b3400d4270200000000008000eb00810f5000d9
:109b44000b003a005000200000548800f2cabf0005
:109b54000080fb00a1ae20004200dd000080400038
:109b640071002000010878000000eb003007980025
:109b74009a100200010000000001be008053800022
:109b84009153800000005100818059000001be0003
:109b94006000b800800f5100818f5900120034001a
:109ba400f2cabf000080fb00a1ae20004200dd002d
:109bb4000080e80000804000104078001a23020072
:109bc40000000000f2cabf000080fb00a1ae20002c
:109bd4004200dd0000804000b10020000108780050
:109be4000000eb0030079800920037009a10020042
:109bf400010000000001be0040a52e00a1022000cb
:109c040002004000838048008053880091538800fc
:109c14009e00780010002000808f500015003a004c
:109c2400f2cabf000080fb00a1ae20004200dd00ac
:109c34000080e800008040001040780022002000ee
:109c44008000eb001227020000000000f2cabf00ef
:109c54000080fb00a1ae20004200dd000080400037
:109c640031002000010878000000eb003007980064
:109c740070003700f2cabf000080fb00a1ae2000d4
:109c84004200dd000080e8000080400010407800c1
:109c94000002eb009e0178000001eb00a1c3b300b9
:109ca400462b0200000000000080e8001007980026
:109cb4000000eb00300798009e0090000001200097
:109cc400808f50000e0036009e00e800f2cabf00ec
:109cd4000080fb00a2ae20004200dd000080e8000e
:109ce4000000410010407800010178008000eb0082
:109cf40012270200000000000000000073ff37007c
:109d0400f2cabf000080fb00a1ae20004200dd00cb
:109d14000080e8000080400010407800eb0047001d
:109d24001e01900012270200000000001e00900097
:109d34008000e9006b0147000040eb0000f178006f
:109d44001e0090001e0f10000040eb0040479800da
:109d5400150037004e4090000080fb00800040005a
:109d6400402a290000804000900078006b004700e2
:109d7400c40a020000000000800078000000eb002c
:109d8400808f500005003a004e40900040040700c8
:109d94001000200030079800070037004e40900064
:109da4000040e80040479800ce40900020c0b30037
:109db40080cf5000e7ff3600be0090000000eb00ab
:109dc400808f50000e003200f2cabf000080fb00fa
:109dd400a1ae20004200dd000080e80000804000c9
:109de400104078000002eb008001eb000001eb0062
:109df400a1c0b300462b020000000000000f780051
:109e04009e00e800f2cabf000080fb00a2ae200062
:109e14004200dd000080e8000000410010407800ae
:109e2400010178008000eb0012270200000000000e
:109e340026ff3700810337007fcabf0080407800c7
:109e44000040eb0080cf50000c00350030002000b3
:109e540000548800f2cabf000080fb00a1ae2000bd
:109e64004200dd00008040007100200001087800fd
:109e74000000eb003007980070033700c1538000e6
:109e84000040eb008048780040a82000420507000d
:109e9400c05388000154800080002000808f50004f
:109ea4000a003a00f2cabf000080fb00a1ae200005
:109eb4004200dd00008040007100200001087800ad
:109ec4000000eb00300798005c033700f2cabf00c3
:109ed4000080fb00a1ae20004200dd0000804000b5
:109ee4004100200001087800e1a72000914078009b
:109ef4000040eb0080cf500007003a00f2cabf00d8
:109f04000080fb00a1ae20004200dd000080400084
:109f140051002000010878000000eb003007980091
:109f24000040eb007eeab70044033700646002009f
:109f34000000000021002000810f50003603320091
:109f4400f2cabf000080fb00a1ae20004200dd0089
:109f5400008040005100200001087800f2cabf00d0
:109f64000080fb00a1ae20004200dd000080e8007c
:109f740000804000104078006826020000000000c5
:109f84006101b800a0538000b1538000800f5100dc
:109f9400818f59001f003a009a100200010000004e
:109fa4000001be00805380009153800000005100e6
:109fb400818059000001be006000b800800f51008c
:109fc400818f590013003400f2cabf000080fb00e7
:109fd400a1ae20004200dd000080e80000804000c7
:109fe400104078001a23020000000000f2cabf00eb
:109ff4000080fb00a1ae20004200dd000080400094
:10a00400b1002000010878000000eb003007980040
:10a014000a0337000154800010002000808f500094
:10a02400080032000154800080002000808f50001e
:10a034006b00360001548000b0002000808f500077
:10a0440067003e000154800080002000808f500093
:10a054001500360001548000b0002000808f5000ad
:10a0640011003e006506070000407800204f98006c
:10a07400ae4890000040eb0080cf50000e003a0044
:10a08400f2cabf000080fb00a1ae20004200dd0048
:10a094000080400071002000010878000000eb00ff
:10a0a40030079800e50237007862020000000000e3
:10a0b40000407800204f9800ae48900020c0b300c4
:10a0c40080cf50000e003a00f2cabf000080fb00af
:10a0d400a1ae20004200dd000080e80000804000c6
:10a0e4001040780068260200000000000000e9002b
:10a0f40001002000a0538800b1538800cf0237002c
:10a10400ae48900010c0b30080cf500034003a0035
:10a11400f2cabf000080fb00a1ae20004200dd00b7
:10a124000080e800008040001040780068260200ab
:10a134000000000001002000a0538800b1538800f3
:10a144009a100200010000000001be0040a52e008c
:10a15400a102200002004000838048008053880050
:10a16400915388004253800053538000a0538000d1
:10a17400b1538000800f5100818f59000c003600cc
:10a18400f2cabf000080fb00a1ae20004200dd0047
:10a194000080e8000080400010407800d4270200ce
:10a1a400000000008000eb00810f50009c023a0088
:10a1b4006000200000548800f2cabf000080fb0049
:10a1c400a1ae20004200dd000080400071002000ac
:10a1d400010878000000eb00300798009702370070
:10a1e400f2cabf000080fb00a1ae20004200dd00e7
:10a1f400008040006100200001087800c1a7200011
:10a204009140780000c0eb0080cf50000c003a0071
:10a214004000200000548800f2cabf000080fb0008
:10a22400a1ae20004200dd0000804000710020004b
:10a23400010878000000eb00300798007f02370027
:10a244006000b8004053880051538800d1a7200013
:10a254009140780000c0eb0080cf500005003a0028
:10a264000080eb008080eb0060538800715388000d
:10a27400040037007dcabf00c1a6200070a30200fd
:10a2840000000000f2cabf000080fb00a1ae200065
:10a294004200dd00008040007100200001087800c9
:10a2a400f2cabf000080fb00a1ae20004200dd0026
:10a2b4000080e800008040001040780023c0b30014
:10a2c4000001eb0011002000d44202000000000055
:10a2d40000548000800040000026290000804000d7
:10a2e4001000780080007800f2cabf000080fb00f4
:10a2f400a2ae20004200dd000080e8000000410022
:10a304001040780002260200000000000154800082
:10a31400c0002000808f500028003a00f2cabf001d
:10a324000080fb00a1ae20004200dd000080e800b8
:10a33400008040001040780041a82000022602005e
:10a3440000000000812c2900f2cabf000080fb003d
:10a35400a2ae20004200dd000080e80000004100c1
:10a36400104078000226020000000000f2cabf007c
:10a374000080fb00a1ae20004200dd000080e80068
:10a38400008040001040780041a82000022602000e
:10a3940000000000f2cabf000080fb00a1ae200054
:10a3a4004200dd000080e80000804000104078009a
:10a3b40051b8280002260200000000000154800069
:10a3c4000000eb00808f50000c003200015480002c
:10a3d40010002000808f500008003200f2cabf0035
:10a3e4000080fb00a1ae20004200dd0000804000a0
:10a3f400b1002000010878001002370011548000d9
:10a40400b0002000808f500023003200b12d2900bd
:10a41400f2cabf000080fb00a2ae20004200dd00b3
:10a424000080e8000000410010407800022602008d
:10a43400000000001054800080004000a0c32800e9
:10a44400008040001000780080007800f2cabf004d
:10a454000080fb00a2ae20004200dd000080e80086
:10a4640000004100104078000226020000000000b5
:10a47400f2cabf000080fb00a1ae20004200dd0054
:10a484000080e800008040001040780051b82800a7
:10a4940002260200000000007ccabf009ca7020044
:10a4a4000000000061006000804078000040eb0084
:10a4b40080cf50000a003200a12e2900f2cabf004a
:10a4c4000080fb00a2ae20004200dd000080e80016
:10a4d4000000410010407800022602000000000045
:10a4e40031302900f2cabf000080fb00a2ae200078
:10a4f4004200dd000080e8000000410010407800c8
:10a504000226020000000000015480001000200018
:10a51400808f500007003200625380007353800024
:10a524000080eb008080eb00800f5100818f590088
:10a534000b00320031312900f2cabf000080fb0059
:10a54400a2ae20004200dd000080e80000004100cf
:10a5540010407800022602000000000014003700ba
:10a56400c1312900f2cabf000080fb00a2ae200066
:10a574004200dd000080e800000041001040780047
:10a58400022602000000000051322900f2cabf0076
:10a594000080fb00a2ae20004200dd000080e80045
:10a5a4000000410010407800022602000000000074
:10a5b400f2cabf000080fb00a1ae20004200dd0013
:10a5c4000080e800008040001040780051b8280066
:10a5d4000226020000000000e1a72000914078005c
:10a5e4000040eb0080cf500008003200f2cabf00e8
:10a5f4000080fb00a1ae20004200dd00008040008e
:10a60400810020000108780011003700f2cabf0061
:10a614000080fb00a1ae20004200dd000080e800c5
:10a62400008040001040780051b828000226020043
:10a6340000000000f2cabf000080fb00a1ae2000b1
:10a644004200dd00008040009100200001087800f5
:10a654000000eb00300798007801370040a8200084
:10a66400d0538800e900370091322900f2cabf00b4
:10a674000080fb00a2ae20004200dd000080e80064
:10a684000000410010407800022602000000000093
:10a6940056003700ae48900000c2b30080cf50008f
:10a6a4000b003a00f2cabf000080fb00a1ae2000fc
:10a6b4004200dd000080e800008040001040780087
:10a6c400b1c2b3008224020000000000470037003a
:10a6d400ae489000f0c2b30080cf500014003600a2
:10a6e400ae48900090c3b30080cf50000400360001
:10a6f400ae48900000c4b30080cf50000c00360078
:10a70400ae489000a0c5b30080cf500004003600ce
:10a71400ae48900000c6b30080cf5000040036005d
:10a72400ae489000a0c7b30080cf5000250036008b
:10a73400f2cabf000080fb00a1ae20004200dd0091
:10a744000080e800008040001040780051c2b3004f
:10a7540082240200000000002e489000e0b00200b5
:10a764000000000080407800f2cabf000080fb00b7
:10a77400a2ae20004200dd000080e800000041009d
:10a784001040780082240200000000002e4890004f
:10a7940002b102000000000080407800f2cabf004d
:10a7a4000080fb00a2ae20004200dd000080e80033
:10a7b40000004100104078008224020000000000e4
:10a7c4000a003700ae489000f2cabf000080fb00c8
:10a7d400a2ae20004200dd000080e800000041003d
:10a7e400104078008224020000000000d253800050
:10a7f40012407800204f98002e4890000080fb0003
:10a804000000ea004f00de00804078000200e8000b
:10a81400d05388000040eb0080cf50009dff3a00e9
:10a82400f2cabf000080fb00a1ae20004200dd00a0
:10a834000080e8000080400010407800d1c3b300dd
:10a84400822402000000000056003700ae48900049
:10a8540000c2b30080cf50000b003a00f2cabf0020
:10a864000080fb00a1ae20004200dd000080e80073
:10a874000080400010407800b1c2b300822402007e
:10a884000000000047003700ae489000f0c2b3005b
:10a8940080cf500014003600ae48900090c3b3003f
:10a8a40080cf500004003600ae48900000c4b300ce
:10a8b40080cf50000c003600ae489000a0c5b30015
:10a8c40080cf500004003600ae48900000c6b300ac
:10a8d40080cf500004003600ae489000a0c7b300fb
:10a8e40080cf500025003600f2cabf000080fb0074
:10a8f400a1ae20004200dd000080e800008040009e
:10a904001040780051c2b30082240200000000000d
:10a914002e489000e0b00200000000008040780063
:10a92400f2cabf000080fb00a2ae20004200dd009e
:10a934000080e800000041001040780082240200fa
:10a94400000000002e48900002b102000000000048
:10a9540080407800f2cabf000080fb00a2ae200055
:10a964004200dd000080e800000041001040780053
:10a9740082240200000000000a003700ae48900064
:10a98400f2cabf000080fb00a2ae20004200dd003e
:10a994000080e8000000410010407800822402009a
:10a9a40000000000d253800012407800204f98002d
:10a9b4002e4890000080fb000000ea004f00de00fb
:10a9c400804078000200e800d05388000040eb008b
:10a9d40080cf50009dff3a00f2cabf000080fb0008
:10a9e400a1ae20004200dd000080e80000804000ad
:10a9f4001040780051b82800022602000000000030
:10aa04007ecabf000040e9007eeab700e1a720004b
:10aa1400914078000040eb0080cf500012ff3a00d4
:10aa2400f2cabf000080fb00a1ae20004200dd009e
:10aa34000080e800008040001040780051b82800f1
:10aa44000226020000000000f2cabf000080fb00e2
:10aa5400a1ae20004200dd000080400091002000f3
:10aa6400010878000000eb00300798007a00070026
:10aa74008000eb00810f50000e0032007ccabf0042
:10aa8400e6a002000000000000c0eb007ceab70072
:10aa9400f2cabf000080fb00a1ae20004200dd002e
:10aaa40000804000b1002000010878001000200060
:10aab40030079800f2cabf000080fb00a1ae20005e
:10aac4004200dd000080e800008040001040780073
:10aad40030240200000000008000eb00810f5000d1
:10aae40051003a001000200030079800530037004e
:10aaf4001000200030079800f2cabf000080fb005d
:10ab0400a1ae20004200dd000080e800008040008b
:10ab1400104078003024020000000000f100200002
:10ab2400810f500042003600805380009153800012
:10ab3400adf70700a2538000b35380006000b80053
:10ab4400800f5100818f59003b003a000000eb0058
:10ab540030079800f2cabf000080fb00a1ae2000bd
:10ab64004200dd00008040009100200001087800d0
:10ab740032003700c1a720009140780000c0eb00ec
:10ab840080cf5000050032007ccabf00e6a002005e
:10ab94000000000000c0eb007ceab700d1a7200051
:10aba4009140780000c0eb0080cf500005003200d7
:10abb4007dcabf00e6a002000000000000c0eb0058
:10abc4007deab700f2cabf000080fb00a1ae2000fe
:10abd4004200dd000080e800008040001040780062
:10abe4001a23020000000000f2cabf000080fb002c
:10abf400a1ae20004200dd00008040008000eb0098
:10ac0400010878000d003700000000000b00370039
:10ac140000000000090037000000000007003700b2
:10ac240000000000050037000000000003003700aa
:10ac3400000000000100370000000000be0090008a
:10ac44000000eb00808f500078f932004f04780048
:10ac54000080fa00000006004600fa00f2cabf00b5
:10ac64000080fb00a1ae20004200dd000080e8006f
:10ac740000804000104078003024020000000000f2
:10ac84001007980062538000735380004053800083
:10ac94005153800000005100818059001e01900032
:10aca40003002000820f5000838f580001003600fb
:10acb4000200be00000f780042538000535380000e
:10acc4001e0078000100200002004000838048003c
:10acd4004053880051538800200037001e0078003c
:10ace40001042000810f5000010036000004200000
:10acf400c3a7200093417800e500470000017800d5
:10ad04000340780040a202000000000010079800f1
:10ad14009e0090000000eb00808f500002003a007b
:10ad24001000200058003700f2cabf000080fb006a
:10ad3400a1ae20004200dd000080e8000080400059
:10ad440010407800e50047001e019000262502000f
:10ad5400000000001e0090001e0f10009e007800ee
:10ad64000000eb00808f5000dcff3a00425380006b
:10ad7400535380006053800071538000800f510052
:10ad8400818f59003f003a00f2cabf000080fb00e7
:10ad9400a1ae20004200dd0000804000a1002000a0
:10ada400010878006000b800a0538800b1538800ff
:10adb4007ccabf008000eb0010a10200000000006c
:10adc4007ccabf00e400470010a10200000000009c
:10add4008000eb00810f50000d00320042538000d0
:10ade40053538000100020000100200002004000a6
:10adf400838048004053880051538800ce4090001f
:10ae0400e0c7b30080cf5000edff3a0001003700e7
:10ae140000000000425380005353800010002000c3
:10ae24000100200002004000838048004053880055
:10ae3400515388007dcabf0001a7200070a30200ff
:10ae4400000000007dcabf00c1a6200070a302005c
:10ae5400000000008000eb00810f500009003a0060
:10ae64000080eb008080eb00605388007153880001
:10ae74007dcabf00e6a002000000000000c0eb0095
:10ae84007deab7000000eb000080fa000000060035
:10ae94000200fa00004f78009e4078000040eb006a
:10aea40080cf500002003a007d0007000c003700fc
:10aeb4009e40780010c0b30080cf500002003a00da
:10aec40009000700060037009e40780020c0b30048
:10aed40080cf500002003a00fe000700000000008e
:10aee4000080fa00000006002c00fa007fcabf00b0
:10aef400804078000040eb0080cf500065003500b2
:10af0400f2cabf000080fb00a1ae20004200dd00b9
:10af14000080e800008040001040780062002000bb
:10af24008000eb001227020000000000f2cabf00fc
:10af34000080fb00a1ae20004200dd000080e8009c
:10af440000804000104078008002eb000002eb001b
:10af54008001eb002200200051b82800ba2802002a
:10af640000000000000f78001e007800630f40000e
:10af7400c00f20001e0f60001e0078004102200058
:10af8400810f50000100360040022000000f7800bd
:10af9400640047001007980016003700f2cabf008b
:10afa4000080fb00a1ae20004200dd000080e8002c
:10afb4000080400010407800420020009e00900075
:10afc4001227020000000000330020001e01900040
:10afd400410020001e0090002cad02000000000083
:10afe4001e007800640f50001e00900063004000b3
:10aff400100798009e0078000000eb00808f50003e
:10b00400e6ff3a009e0090000040eb008048780084
:10b014000000eb00000f7800640047001007980060
:10b02400090037001e00900090407800a0c3b300d0
:10b0340080cf5000090032001e0fe8001e0090006f
:10b044000000e80010079800700220009e007800bd
:10b05400808f5000f3ff360001003700000000002d
:10b064009e0090000040eb00804878001e00900095
:10b074000000e80010079800640047009e0090005c
:10b0840036600200000000007feab7000000000004
:10b0940001003700000000000080fa0000000600f4
:10b0a4000400fa00881f7800f2cabf000080fb0089
:10b0b400a1ae20004200dd000080e80000804000d6
:10b0c400104078008002eb000002eb008001eb00ee
:10b0d4002200200051b82800ba2802000000000015
:10b0e400000f7800c05380008000ea0080ae20008a
:10b0f4000080e90000804000800078001e00780095
:10b10400808f50006b003e005000200000548800e7
:10b11400f2cabf000080fb00a1ae20004200dd00a7
:10b1240000804000710020000108780066003700ac
:10b13400f2cabf000080fb00a1ae20004200dd0087
:10b144000080e80000804000104078000002eb001e
:10b154008001eb000001eb00b1c3b300462b0200f9
:10b164000000000010079800c85380009e00900063
:10b174001e007800810f50000100360001007800a5
:10b18400c453800021af2000914078008180fb00ef
:10b19400a2ae2000c208dd008180e80081004100e9
:10b1a4009141780000017800840078000340780021
:10b1b400122702000000000000004400c053880071
:10b1c400c153800060c2b300804878000100e800e9
:10b1d400c05388009e0090001e007800808f5000ad
:10b1e40025003100f2cabf000080fb00a1ae2000a0
:10b1f4004200dd000080e80000804000104078003c
:10b204008000eb00a0260200000000000a003700c6
:10b21400f2cabf000080fb00a1ae20004200dd00a6
:10b224000080e80000804000104078008000eb00bf
:10b23400a026020000000000f2cabf000080fb004c
:10b24400a1ae20004200dd000080e8000080400044
:10b25400104078000002eb008001eb000001eb00dd
:10b2640001c2b300462b0200000000008000eb0086
:10b27400810f5000e6ff3200f2cabf000080fb00dd
:10b28400a1ae20004200dd000080e8000080400004
:10b29400104078008002eb000002eb008001eb001c
:10b2a4002200200051b82800ba2802000000000043
:10b2b400000f78009e0078000000eb00808f5000a3
:10b2c4009bff3a00000000004f0478000080fa0061
:10b2d400000006000c00fa00f2cabf000080fb0068
:10b2e400a1ae20004200dd000080e80000804000a4
:10b2f400104078008002eb000002eb008001eb00bc
:10b304002200200051b82800ba28020000000000e2
:10b31400000f78009e00780090002000808f50007d
:10b324000600360020002000005488006000b800a9
:10b33400405388005153880015003700f2cabf00fb
:10b344000080fb00a1ae20004200dd000080e80088
:10b3540000804000104078008e80e8001e017800d4
:10b364001227020000000000000f78000e80e800a1
:10b374009e0040000040eb00804878000e80e8000a
:10b3840080090200000000004053880051538800e7
:10b394000080fa00000006000c00fa005007980034
:10b3a4005e009000de0a0200000000002007980002
:10b3b4005e009000100798009e009000010f780036
:10b3c4004d0037001e0078009040780061479800d7
:10b3d4001e0fe8002e0090000000e90020079800ee
:10b3e400ee409000d0c3b30080cf50000400320080
:10b3f400ee40900060c2b30080cf500007003a00d6
:10b404009e0090000040eb00804878001e009000f1
:10b414000000e8001007980037003700ee40900065
:10b42400b0c2b30080cf500007003a009e009000e5
:10b4340000c2b300804878001e0090000000e800bd
:10b44400100798002c003700ee40900050c2b30063
:10b4540080cf500022003a00ae009000100020007f
:10b46400808f500003003e000000eb00200798008e
:10b4740021003700680047008000e8001e007800c3
:10b4840010407800804878001e0fe800e80047006c
:10b494001e00780010407800804878001e0fe800f5
:10b4a4002e0090000000e900200798002e00900074
:10b4b4000000e900200798006800470010007800a9
:10b4c40078b00200000000009e00900080487800e0
:10b4d4001e0090000000e8001007980006003700e6
:10b4e4001e009000ee409000014878001e0090007d
:10b4f4000000e80010079800ae0090000000eb0088
:10b50400808f5000afff3a009e0090000040eb0097
:10b51400804878001e0090000000e80010079800a2
:10b524009e0090000040eb00804878001e009000d0
:10b534000080fa00000006000400fa00000f780002
:10b5440011079800170037009e0078001e00900035
:10b55400c40a0200000000008000eb00810f5000cc
:10b5640006003a001e009000de0a020000000000ff
:10b574000000e8001e004000100037001e007800a4
:10b58400de0a0200000000000000e8001e0f400078
:10b594001e007800de0a0200000000000000e8003f
:10b5a4001e0f40001e007800904078000040eb0021
:10b5b40080cf5000e4ff3a000000eb000080fa0066
:10b5c400000006000600fa00100798002107980002
:10b5d4002e0190009e009000d0c3b3003f000700ee
:10b5e400000f78009e0090000000eb00808f500058
:10b5f400070032001e009000904078000040eb00ed
:10b6040080cf5000020032001e00900062ff07004d
:10b614001e0078000080fa00000006000600fa0010
:10b62400889fbe0010079800210798002e01900003
:10b634009e00900060c2b30028000700000f78004d
:10b644009e00780020002000808f500014003a00f3
:10b654004853800059538000f2cabf000080fb00a9
:10b66400a1ae20004200dd000080e8000080400020
:10b67400104078006826020000000000010020004d
:10b68400800f5400818f5c0005003a002e01900069
:10b694009e0090000040eb0010000700000f7800af
:10b6a4009e0090000000eb00808f500007003200e5
:10b6b4001e009000904078000040eb0080cf5000c6
:10b6c400020032001e00900033ff07001e007800c5
:10b6d4004f04be000080fa00000006000a00fa00d1
:10b6e400889fbe00404798003107980042079800a1
:10b6f400ce4090000040eb0080cf50000f0032009d
:10b70400f2cabf000080fb00a1ae20004200dd00b1
:10b714000080e80000804000104078000002eb0048
:10b724008001eb000001eb00ce409000462b0200ac
:10b7340000000000100798000a003700f2cabf009a
:10b744000080fb00a1ae20004200dd000080e80084
:10b7540000804000104078006826020000000000cd
:10b76400100798009e0090000080eb00808f50002e
:10b7740002003a00200020009d003700ce00900017
:10b7840010002000808f500019003e00be00900081
:10b794000000eb00808f50001500320048538000f9
:10b7a40059538000f2cabf000080fb00a1ae200004
:10b7b4004200dd000080e800008040001040780076
:10b7c4001e0190008000eb00122702000000000020
:10b7d400010020000000540081805c004053880078
:10b7e4005153880010002000000f78006a003700d1
:10b7f400be0090000000eb00808f500015003a005e
:10b804004853800059538000f2cabf000080fb00f7
:10b81400a1ae20004200dd000080e800008040006e
:10b82400104078001e0190008000eb0012270200f7
:10b8340000000000010020000000540081805c0032
:10b8440040538800515388000000eb00000f78003b
:10b85400510037004e0090008080e9001e009000e7
:10b86400808f5000330031004853800059538000ca
:10b874004e0090008080e900f2cabf000080fb0007
:10b88400a2ae20004200dd000080e800000041007c
:10b894001040780001017800be00900012270200d9
:10b8a40000000000010020000000540081805c00c2
:10b8b40040538800515388004853800059538000f6
:10b8c4009e0090004e009000008050008080e800b0
:10b8d400f2cabf000080fb00a2ae20004200dd00df
:10b8e4000080e80000004100104078000101780069
:10b8f4008000eb001227020000000000010020007d
:10b904000000540081805c0040538800515388003b
:10b914004e0090000080e900be009000808040004e
:10b924000040eb008048780010002000000f7800f1
:10b93400190037004853800059538000f2cabf00f1
:10b944000080fb00a1ae20004200dd000080e80082
:10b9540000804000104078001e019000be0090005e
:10b964001227020000000000010020000000540023
:10b9740081805c004053880051538800be009000d1
:10b984001e009000808040000040eb00804878005a
:10b994000000eb00000f7800ce4090000040eb0068
:10b9a40080cf50001100320048538000595380006a
:10b9b400f2cabf000080fb00a1ae20004200dd00ff
:10b9c4000080e80000804000104078008000eb0018
:10b9d400a026020000000000010020000000540026
:10b9e40081805c0040538800515388001e00780019
:10b9f4004f04be000080fa00000006001400fa00a4
:10ba0400889fbe000054800091002000810f5000e8
:10ba14000a00320091002000810f50000501390016
:10ba2400a1002000810f5000b5003200b1002000b9
:10ba3400810f500082003200030137006133290076
:10ba4400f2cabf000080fb00a2ae20004200dd006d
:10ba54000080e80000004100104078008002eb0004
:10ba64000002eb008001eb0042002000ba28020033
:10ba740000000000000f78009e0078000080eb00ba
:10ba8400808f50004f003200f2cabf000080fb00dc
:10ba9400a1ae20004200dd000080e80000804000ec
:10baa400104078001e0178008000eb00122702008d
:10bab40000000000000f78004253800053538000c0
:10bac4001e00780001002000000051008180590010
:10bad4004053880051538800f2cabf000080fb0025
:10bae400a1ae20004200dd000080e800008040009c
:10baf4001040780068260200000000009100200039
:10bb0400810f500003003e001e0fe80010002000cb
:10bb1400ce003700f2cabf000080fb00a1ae2000b7
:10bb24004200dd000080e800008040001040780002
:10bb3400e4004700a20020001227020000000000d9
:10bb4400000f780042538000535380001e00780099
:10bb540001002000000051008180590040538800fa
:10bb64005153880064004700a2002000b13329002b
:10bb7400600a0200000000008000eb00810f50000a
:10bb84000c003a00a0002000005488005ca50200cc
:10bb9400000000007ceab7007ccabf00e400470054
:10bba400e480400062002000eaa5020000000000da
:10bbb40002003700b000200000548800200020005c
:10bbc400a2003700f2cabf000080fb00a1ae200033
:10bbd4004200dd000080e800008040001040780052
:10bbe4006826020000000000e4005000f2cabf0012
:10bbf4000080fb00a2ae20004200dd000080e800cf
:10bc04000000410010407800010178008000eb0042
:10bc14001227020000000000000f78004253800049
:10bc2400535380001e0078000100200000005100e2
:10bc340081805900405388005153880082003700a6
:10bc44004853800059538000f2cabf000080fb00b3
:10bc5400a1ae20004200dd000080e800008040002a
:10bc64001040780068260200000000000100200057
:10bc74000000540081805c004053880051538800c8
:10bc8400f2cabf000080fb00a1ae20004200dd002c
:10bc94000080e80000804000104078004826020040
:10bca40000000000425380005353800030062000ff
:10bcb40001002000800f5100818f590007003600d9
:10bcc40042538000535380000000200001002800ec
:10bcd400800f5100818f590058003600f2cabf000e
:10bce4000080fb00a1ae20004200dd000080400087
:10bcf40071002000010878000000eb0053003700b9
:10bd0400f2cabf000080fb00a1ae20004200dd00ab
:10bd14000080e8000080400010407800682602009f
:10bd240000000000000f78001e0078006101b800d8
:10bd34004053800051538000800f5100818f59007f
:10bd4400260036004053800051538000000f7800d5
:10bd5400220037001e00780001012000810f5000ee
:10bd6400010036000001200021af2000914078003e
:10bd74008180fb00a2ae2000c208dd008180e800c3
:10bd84008100410091417800e400470000017800ff
:10bd940003407800122702000000000010079800fa
:10bda40042538000535380001e0090000100200085
:10bdb400000051008180590040538800515388008d
:10bdc4001e0090001e0f10007ccabf00e400470054
:10bdd4001e019000eaa50200000000009e00780009
:10bde4000000eb00808f5000daff3a0042538000dd
:10bdf400535380006000b800800f5100818f5900b8
:10be040010003a0010002000a0a60200000000006c
:10be1400f2cabf000080fb00a1ae20004200dd009a
:10be24000080400071002000010878000000eb0051
:10be34000600370000000000030037000000000087
:10be44000100370000000000100020004f04be0075
:10be54000080fa00000006004800fa00881f7800fd
:10be640030279800a2538000b35380006000b800cc
:10be7400800f5100818f59000e003a003e2090003f
:10be8400f29e02000000000020479800ae4090009f
:10be940000c0eb0080cf50005300320048a72000c0
:10bea4002e40900086a9020000000000000c7800db
:10beb4001000370040a720001000780058a00200ae
:10bec4000000000020479800ae40900000c0eb0046
:10bed40080cf50004600320040a7200010009000a0
:10bee4006101b800210020002e40900090a30200c0
:10bef40000000000f2cabf000080fb00a1ae2000d9
:10bf04004200dd000080e80000804000104078001e
:10bf14003024020000000000000f780023003700e6
:10bf24001e00780001042000810f5000010036003b
:10bf340000042000e6004700000178002e40900035
:10bf440040a202000000000020079800ae0090000c
:10bf54000000eb00808f500007003a002e40900054
:10bf6400e6a00200000000006000b800a0538800b2
:10bf7400b15388001f003700f2cabf000080fb00e5
:10bf8400a1ae20004200dd000080e80000804000f7
:10bf940010407800e60047002e019000262502009c
:10bfa400000000002e0090001e0f10009e0078007c
:10bfb4000000eb00808f5000d9ff3a0048a7200012
:10bfc4002e40900064a902000000000000007800e8
:10bfd400100498002e409000e6a00200000000002b
:10bfe40000000000030037000000000001003700db
:10bff400000000004f0478000080fa0000000600f2
:10c004000200fa00000f7800720020006134290059
:10c014001e007800600a0200000000008000780022
:10c024000000eb00808f500002003a000040eb005b
:10c034000b00370042002000e13429001e00780084
:10c04400600a0200000000008000eb00810f500035
:10c0540002003a000040eb000100370000c8b300c2
:10c064000080fa00000006000400fa00000f7800c7
:10c07400110798001e00780031352900c40a020017
:10c0840000000000800078000000eb00808f50006a
:10c0940009003a001e00900091352900c40a0200ec
:10c0a400000000008000eb00810f500002003a0005
:10c0b40000c8b300010037000040eb000080fa0024
:10c0c400000006001600fa007ccabf008e80e8005b
:10c0d4004201200000a90200000000000e80e800d8
:10c0e4009200200031362900600a0200000000009e
:10c0f4008000eb00810f500069003a00d03629001f
:10c104008000780040a820009e5a02000000000031
:10c11400000f78009e0078000000eb00808f500034
:10c12400100032001e0078009040780010c3b30065
:10c1340000c068000080fb000000e9004f00de0042
:10c14400004078000080fb00610060004400dd00d6
:10c1540022168000f1fe2f00810061000080700033
:10c1640020168800203729008000780040a820008d
:10c174009e5a020000000000000f78009e00780024
:10c184000000eb00808f5000100032001e00780089
:10c194009040780010c3b30000c068000080fb002a
:10c1a4000000e9004f00de00004078000080fb0042
:10c1b400610060004300dd002216800071ff2f0043
:10c1c400810061000080700020168800703729000b
:10c1d4008000780040a820009e5a02000000000061
:10c1e400000f78009e0078000000eb00808f500064
:10c1f400100032001e0078009040780010c3b30095
:10c2040000c068000080fb000000e9004f00de0071
:10c21400004078000080fb00610060004200dd0007
:10c2240022168000b1ff2f008100610000807000a1
:10c2340020168800c03729008000780040a820001c
:10c244009e5a020000000000000f78009e00780053
:10c254000000eb00808f5000a10032001e00780027
:10c264009040780010c3b30000c068000080fb0059
:10c274000000e9004f00de00004078000080fb0071
:10c28400610060000000400022168000d1ff2f00f2
:10c294008100610000807000201688009000370043
:10c2a4000e80e800b200200011382900600a020064
:10c2b400000000008000eb00810f500003003a00f2
:10c2c40010c0b3007eeab700850037000e80e80096
:10c2d40082002000d1382900600a0200000000001a
:10c2e4008000eb00810f50007d003a006039290086
:10c2f4008000780040a820009e5a02000000000040
:10c30400000f78001e007800104078000080fb00c9
:10c314006101b900f0fc2f00f1ff2f000200400082
:10c32400838048006200200003002000820f500038
:10c33400838f58006a003e00006001000600370049
:10c3440013003700200037002d0037003a00370073
:10c354004700370054003700201680000000d10049
:10c36400614060000004a200614060000080fb00a6
:10c37400610060000000400022168000d1ff2f0001
:10c38400810061000080700020168800540037008e
:10c39400201680004200de00614060000004a2001c
:10c3a400614060000080fb00610060004200dd002d
:10c3b40022168000b1ff2f00810061000080700010
:10c3c4002016880046003700201680004300de0057
:10c3d400614060000004a200614060000080fb0036
:10c3e400610060004300dd002216800071ff2f0011
:10c3f400810061000080700020168800380037003a
:10c40400201680004400de00614060000004a200a9
:10c41400614060000080fb00610060004400dd00ba
:10c4240022168000f1fe2f00810061000080700060
:10c43400201688002a003700201680004500de0000
:10c44400614060000004a200614060000080fb00c5
:10c45400610060004500dd0022168000f1fd2f0020
:10c464008100610000807000201688001c003700e5
:10c47400201680004600de00614060000004a20037
:10c48400614060000080fb00610060004600dd0048
:10c4940022168000f1fb2f008100610000807000f3
:10c4a400201688000e003700201680004700de00aa
:10c4b400614060000004a200614060000080fb0055
:10c4c400610060004700dd0022168000f1f72f00b4
:10c4d40081006100008070002016880000000000c8
:10c4e4000000eb000080fa00000006001400fa00cf
:10c4f4007ccabf00420120008e00780000a902001f
:10c504000000000092002000313629000e0078005f
:10c51400600a0200000000008000eb00810f500060
:10c5240002003a00210007001e003700a20020008c
:10c53400a13929000e007800600a02000000000002
:10c544008000eb00810f500002003a000202070055
:10c554001400370022012000513a29000e0078000f
:10c56400600a0200000000008000eb00810f500010
:10c5740002003a00620007000a0037000e0078004b
:10c58400813b2900c40a0200000000008000eb0087
:10c59400810f500002003a00cd020700010037006d
:10c5a4000000eb000080fa00000006000200fa0020
:10c5b400e8cabf000080fb008000eb00810f500040
:10c5c4000400320011002000810f50000c003200e2
:10c5d400480037004106200040a82000e45a020029
:10c5e4000000000021002000810f500002003a00ea
:10c5f400100020004000370010c0b300e8eab70084
:10c6040040a82000813c2900c40a02000000000068
:10c614008000eb00810f500003003a0040a8200086
:10c62400000f7800020037000000eb00000f7800d4
:10c63400410620001e007800105b0200000000008c
:10c6440021002000810f500002003a001000200059
:10c65400290037009e0078000000eb00808f500016
:10c6640003003a000040eb00e8eab700210037007d
:10c674001e007800de0a020000000000800078003e
:10c68400f0012000808f50000a003e0002022000ca
:10c694000102200020e92000a20a0200000000009c
:10c6a4009e00780020e92000d20a02000000000069
:10c6b40005003700020220009e00780020e92000d7
:10c6c400940a0200000000004c0502000100000072
:10c6d40040a82000b2002000c13c2900940a0200b6
:10c6e40000000000c0002000005488000000eb009f
:10c6f40001003700200020000080fa00000006003e
:10c704003a00fa00889fbe008a1f780048538000d0
:10c7140059538000f2cabf000080fb00a1ae200084
:10c724004200dd000080e8000080400010407800f6
:10c73400682602000000000000057800f2cabf006d
:10c744000080fb00a1ae20004200dd000080e80074
:10c754000080400010407800d42702000000000050
:10c764000000450001002000800f5400818f5c0010
:10c7740062013e00f2cabf000080fb00a1ae2000af
:10c784004200dd000080e800008040001040780096
:10c7940068260200000000006101b80040538000d8
:10c7a40051538000800f5100818f590002003100e5
:10c7b40010002000640137006400470033032000a8
:10c7c400000178006000200001002000b6ec0200a7
:10c7d400000000006400470060119000f1fb2f008e
:10c7e4008100610061109800110137006100200090
:10c7f40040a82000e45a0200000000008000eb0082
:10c80400810f50003f013a00c1052000a0a820007c
:10c81400105b0200000000008000eb00810f50005c
:10c824003a013a0040a82000713d2900c40a0200e0
:10c83400000000008000eb00810f50000f003a0060
:10c844006400470080007800a0a8200098ab020094
:10c85400000000008000eb00810f50002d01320029
:10c8640064014700120078009200900064014700c0
:10c874002009980031099800ed00370040a82000f5
:10c88400a13d2900c40a0200000000008000eb0062
:10c89400810f50000a003a0064004700680040001d
:10c8a40080007800a0a8200098ab020000000000df
:10c8b4008000eb00810f5000dd003a0018013700c2
:10c8c40040a82000d13d2900c40a02000000000055
:10c8d4008000eb00810f500010003a006400470014
:10c8e4006400400080007800a0a8200098ab0200fb
:10c8f400000000008000eb00810f500007013200af
:10c904006401470022009000b200900064014700d7
:10c914004009980051099800c500370040a820003c
:10c92400113e2900c40a0200000000008000eb0050
:10c93400810f50000a003a00640047006c00400078
:10c9440080007800a0a8200098ab0200000000003e
:10c954008000eb00810f5000b5003a00f000370072
:10c9640040a82000613e2900c40a02000000000023
:10c974008000eb00810f50000a003a006400470079
:10c984007000400080007800a0a8200098ab02004e
:10c99400000000008000eb00810f5000a4003a006a
:10c9a400df00370040a82000b13e2900c40a02007d
:10c9b400000000008000eb00810f50007a003a0074
:10c9c400a0a82000000f78000040eb00304798003a
:10c9d400450037001e0fe80001003700000000008a
:10c9e4001e007800904078000040eb0080cf50009b
:10c9f4001e0032001e00780090407800f0c2b300a0
:10ca040080cf5000050036001e007800904078006a
:10ca140090c3b30080cf5000140036001e0078008d
:10ca24009040780000c4b30080cf50000500360069
:10ca34001e0078009040780060c4b30080cf50009e
:10ca44000a0036001e0078009040780000c6b3004b
:10ca540080cf5000dfff36001e0078009040780041
:10ca640060c6b30080cf5000daff3e001e0078009d
:10ca7400904078000040eb0080cf50000f003a0057
:10ca8400090037003e4090008080fb0040a8200051
:10ca94008080400000c3b300804878003e4090008e
:10caa4000040e80030479800be409000b0c0b3009a
:10cab40080cf5000f3ff36000f0037003e40900057
:10cac4000081fb001e0078001040780041a820007f
:10cad40081004100804878001e0fe8003e4090002d
:10cae4000040e80030479800be409000b0c0b3005a
:10caf40080cf5000b9ff36000040eb00304798006b
:10cb040024003700800320000e0040008000e8006d
:10cb14003e4090000080fb00000040007c0140008b
:10cb240080a6200000004100104078008048780072
:10cb3400810320008e8040003e4090000080fb0076
:10cb4400000040000000e8007c01400080a62000b6
:10cb54000000410010407800804878003e4090007a
:10cb64000084fb00800320000e00400010007800c9
:10cb740078b0020000000000e40047008880400014
:10cb8400c102b000904098003e4090000040e80090
:10cb940030479800be40900050c0b30080cf500092
:10cba400d8ff36002200370040a82000f13e2900bb
:10cbb400c40a0200000000008000eb00810f500056
:10cbc4000a003a00a0a82000f0b202000000000011
:10cbd400a1a82000640047007c004000020120005e
:10cbe400940a0200000000001100370040a8200051
:10cbf400413f2900c40a0200000000008000eb004d
:10cc0400810f50000a003a00a1a82000914078004a
:10cc140010c3b30080cf500005003a006400470001
:10cc240060119000010420008100710061109800df
:10cc340042538000535380006000b800800f5100bd
:10cc4400818f5900e9fe3a0064004700d8050200cc
:10cc54000000000040a8200052012000913f29005c
:10cc6400940a02000000000080a92000e4004700ac
:10cc7400fc80400002012000940a02000000000031
:10cc84000040eb00a8eab70040c1b3002047980079
:10cc9400120037002e4090000080fb00fc00400092
:10cca40080a62000008040009040780000c2b300bd
:10ccb40080cf500006003a002e4090008080fb0098
:10ccc40040a82000808040000040eb0080487800ad
:10ccd4002e4090000040e80020479800ae409000ad
:10cce40030c2b30080cf5000eaff3600c0002000fd
:10ccf400005488000000eb0013003700000000001f
:10cd040007003700000000000500370000000000a5
:10cd1400030037000000000001003700000000009d
:10cd240010002000b05e880040a8200042012000ce
:10cd3400e1402900940a020000000000c000200025
:10cd4400005488000000eb004f0578004f04be003b
:10cd54000080fa00000006000400fa00889fbe006c
:10cd6400e8cabf000080fb0011002000810f5000c2
:10cd74003c00320021002000810f50008500320069
:10cd84008000eb00810f5000cd003a00c0bd2000b0
:10cd940098df02000000000021422900f2cabf000f
:10cda4000080fb00a2ae20004200dd000080e8000d
:10cdb40000004100104078008002eb000002eb000c
:10cdc4008001eb0022002000ba28020000000000cd
:10cdd400000f78009e0078000080eb00808f5000e8
:10cde40002003a0010002000b600370042538000d1
:10cdf400535380009e0078006680400001002000ac
:10ce0400000051008180590040538800515388002c
:10ce140048538000595380009e80e800f2cabf0046
:10ce24000080fb00a2ae20004200dd000080e8008c
:10ce34000000410010407800010178008000eb0000
:10ce4400122702000000000001002000000054002e
:10ce540081805c00405388005153880010c0b300a7
:10ce6400e8eab70051422900f2cabf000080fb0083
:10ce7400a2ae20004200dd000080e8000000410076
:10ce8400104078008002eb000002eb008001eb0010
:10ce940042002000ba28020000000000000f7800c1
:10cea4009e0078000080eb00808f50001900320053
:10ceb4001e007800e4004000f2cabf000080fb00be
:10cec400a2ae20004200dd000080e8000000410026
:10ced40010407800010178008000eb001227020066
:10cee40000000000000f780042538000535380007c
:10cef4001e007800010020000000510081805900cc
:10cf0400405388005153880020c0b300e8eab700ba
:10cf140020003700f2cabf000080fb00a1ae200051
:10cf24004200dd000080e8000080400010407800ee
:10cf34006826020000000000e4005000f2cabf00ae
:10cf44000080fb00a2ae20004200dd000080e8006b
:10cf54000000410010407800010178008000eb00df
:10cf64001227020000000000000f780042538000e6
:10cf7400535380001e00780001002000000051007f
:10cf840081805900405388005153880010002000cc
:10cf94004c003700f2cabf000080fb00a1ae2000a5
:10cfa4004200dd000080e80000804000104078006e
:10cfb4006826020000000000000f78001e007800c0
:10cfc4006101b8004053800051538000800f51002c
:10cfd400818f590026003600405380005153800051
:10cfe400000f7800220037001e00780001042000a2
:10cff400810f5000010036000004200021af200002
:10d00400914078008180fb00a2ae2000c208dd00c0
:10d014008180e8008100410091417800000178009e
:10d0240041a82000034078001227020000000000fd
:10d034001007980042538000535380001e00900054
:10d0440001002000000051008180590040538800f5
:10d05400515388001e0090001e0f10001e01900006
:10d0640041a82000c0bd2000d4df02000000000061
:10d074009e0078000000eb00808f5000daff3a0039
:10d0840042538000535380006000b800800f510069
:10d09400818f590008003a0030c0b300e8eab700b5
:10d0a40041a82000c0bd20007ee202000000000074
:10d0b4000000eb00030037001000200001003700df
:10d0c4000000eb004f04be000080fa0000000600e0
:10d0d4000c00fa00889fbe00e8cabf000080fb0075
:10d0e400cf80de00a200200003002000820f500049
:10d0f400838f58004b023e00006001000a00370095
:10d104001f003700a5003700c3003700dc003700dc
:10d11400310137004701370087013700e801370044
:10d124000d0237002502370054750200000000008c
:10d134008000eb00810f50000f003200a042290054
:10d14400206e8800caeda800f0442900106e880003
:10d15400cacda800a0472900306e8800cb0da800d6
:10d1640040a82000c05e88000000eb00d05e88006c
:10d1740010c0b300e8eab700200020002a023700fc
:10d184006400470081002000e45a0200000000000f
:10d1940021002000810f500002003a0010002000fe
:10d1a4002102370064004700214c2900c40a020010
:10d1b400000000008000eb00810f500005003a00e1
:10d1c400c05e8000b06d880020c0b300e8eab700fc
:10d1d4007200370064004700914c2900c40a020021
:10d1e400000000008000eb00810f500005003a00b1
:10d1f400c05e8000d05e880020c0b300e8eab700bb
:10d204006600370064004700e14c2900c40a0200ac
:10d21400000000008000eb00810f500005003a0080
:10d22400c05e8000c06d880020c0b300e8eab7008b
:10d234005a00370064004700314d2900c40a020037
:10d24400000000008000eb00810f500005003a0050
:10d25400c05e8000d06d880020c0b300e8eab7004b
:10d264004e00370064004700814d2900c40a0200c3
:10d27400000000008000eb00810f500005003a0020
:10d28400c05e8000e06d880020c0b300e8eab7000b
:10d294004200370064004700b14d2900c40a02006f
:10d2a400000000008000eb00810f500039003a00bc
:10d2b400b16d80000000eb00808f50000700320049
:10d2c400b06d8000904078000040eb0080cf5000ab
:10d2d40002003a000000eb00b06d8800c16d8000d0
:10d2e4000000eb00808f500007003200c06d80000a
:10d2f400904078000040eb0080cf500002003a00dc
:10d304000000eb00c06d8800d16d80000000eb00d0
:10d31400808f50000b003200d06d80009040780068
:10d324000040eb0080cf500004003200c16d80004b
:10d334000000eb00808f500002003a000000eb0078
:10d34400d06d8800d15e80000000eb00808f50001b
:10d354000a003200d05e8000904078000040eb006c
:10d3640080cf500005003200d05e800080090200aa
:10d374000000000000007800606e8800388202001f
:10d384000000000030c0b300e8eab700200020002d
:10d39400a501370020c0b300e8eab700c05e8000f2
:10d3a4000000ea008000780040a820004006b00099
:10d3b40080804000c05e8000105b0200000000001e
:10d3c40021002000810f500002003a0010002000cc
:10d3d40095013700c85e8000c05e8000de0a02004e
:10d3e4000000000000004400c05e8800c15e8000b0
:10d3f40070ae2000808f500003003100c05e8000ba
:10d404000000e800c05e880010c0b300e8eab7007e
:10d414002000200084013700408202000000000048
:10d424008000eb00810f500004003a00a0c0b3005c
:10d43400e8eab700200020007b0137004e8202009a
:10d444000000000091052000810f500002003e0002
:10d454002000200074013700f04d29005c83020095
:10d4640000000000e05029005c830200000000007e
:10d47400948302000000000040c0b300e8eab70053
:10d4840040820200000000008000eb00810f500089
:10d4940048003a00a0c0b300e8eab700200020002a
:10d4a400610137004e82020000000000000f780086
:10d4b4009e0078000000eb00808f500002003a00cc
:10d4c4002000200058013700f2cabf000080fb0092
:10d4d400a1ae20004200dd000080e8000080400092
:10d4e4001040780068260200000000001007980031
:10d4f4009e0090000000eb00808f500002003a0074
:10d5040010002000480137001e0090009e007800a3
:10d51400808f5000020036001e009000000f78003b
:10d52400200620009e007800808f50000200360004
:10d5340020062000000f78004853800059538000d3
:10d54400f2cabf000080fb00a1ae20004200dd0053
:10d554000080e80000804000104078001e01780040
:10d5640041a8200012270200000000000100200052
:10d574000000540081805c004053880051538800af
:10d5840040a820009e0040000040eb008048780046
:10d5940040a82000ce5902000000000040a820004e
:10d5a4005c8302000000000094830200000000007d
:10d5b40001003700000000004253800053538000f4
:10d5c4006000b800800f5100818f5900b5ff3a0008
:10d5d40050c0b300e8eab700408202000000000037
:10d5e4008000eb00810f500004003a00a0c0b3009b
:10d5f400e8eab700200020000b0137004e82020049
:10d604000000000031062000810f500002003e009f
:10d614002000200004013700705329005c830200bd
:10d6240000000000948302000000000060c0b3000a
:10d63400e8eab70040820200000000008000eb002e
:10d64400810f500004003a00a0c0b300e8eab7001c
:10d6540020002000f40037004e8202000000000089
:10d6640031022000810f500002003e002000200003
:10d67400ed003700805929005c830200000000009f
:10d68400805a29005c83020000000000a01680007c
:10d694004d00de00614060000043b000668202007d
:10d6a40000000000c0c2b300668202000000000057
:10d6b400101680004700de00614060000043b000a7
:10d6c4006682020000000000c0c2b300668202004d
:10d6d40000000000a01680004700de0061406000ea
:10d6e4000043b0006682020000000000c0c2b30024
:10d6f4006682020000000000a01680004600de00e2
:10d70400614060000043b000668202000000000037
:10d71400d0c0b3006682020000000000a0c0b300c5
:10d7240066820200000000009483020000000000f2
:10d7340070c0b300e8eab7004082020000000000b5
:10d744008000eb00810f500004003a00a0c0b30039
:10d75400e8eab70020002000b30037004e82020040
:10d7640000000000d1012000810f500002003e00a3
:10d7740020002000ac003700205b29005c830200fd
:10d784000000000020168000004078006140600026
:10d794000043b0006682020000000000c0c2b30073
:10d7a4006682020000000000201680000000d10004
:10d7b400614060000043b000668202000000000087
:10d7c400c0c2b30066820200000000002016800080
:10d7d4004200de00614060000043b0006682020047
:10d7e40000000000c0c2b300668202000000000016
:10d7f400201680004300de00614060000043b0005a
:10d804006682020000000000c0c2b300668202000b
:10d8140000000000201680004400de00614060002b
:10d824000043b0006682020000000000c0c2b300e2
:10d834006682020000000000201680004500de0021
:10d84400614060000043b0006682020000000000f6
:10d85400c0c2b300668202000000000020168000ef
:10d864004600de00614060000043b00066820200b2
:10d8740000000000c0c2b300668202000000000085
:10d88400201680004700de00614060000043b000c5
:10d894006682020000000000d0c0b300668202006d
:10d8a40000000000a0c0b300668202000000000077
:10d8b400948302000000000080c0b300e8eab700cf
:10d8c40040820200000000008000eb00810f500045
:10d8d40004003a00a0c0b300e8eab700200020002a
:10d8e400510037004e82020000000000f1002000c9
:10d8f400810f500002003e00200020004a00370043
:10d9040000188000000f780051a820001e00780045
:10d91400f0af020000000000905b29005c8302006d
:10d924000000000050a820005c83020000000000fa
:10d93400d0c0b3006682020000000000a0c0b300a3
:10d9440066820200000000009483020000000000d0
:10d9540090c0b300e8eab700408202000000000073
:10d964008000eb00810f500004003a00a0c0b30017
:10d97400e8eab700200020002b0037004e820200a6
:10d9840000000000f1002000810f500002003e0062
:10d994002000200024003700f05b29005c83020093
:10d9a40000000000a0830200000000009483020035
:10d9b40000000000a0c0b300e8eab7004082020003
:10d9c400000000008000eb00810f500013003a00bb
:10d9d4008a750200000000008000eb00810f5000f7
:10d9e40003003a0010002000a05e88000200370007
:10d9f40010002000b05e880040a820001201200022
:10da0400e15c2900940a020000000000c00020002c
:10da1400005488000000eb000300370020002000c1
:10da2400010037000000eb004f04be000080fa0044
:10da3400000006000000fa00100020000100200091
:10da4400a0538800b1538800f2cabf000080fb00d5
:10da5400a1ae20004200dd000080e800008040000c
:10da64001040780030240200000000003101200042
:10da7400810f50000e0036006000b800a0538800eb
:10da8400b1538800f15d2900f2cabf000080fb0099
:10da9400a2ae20004200dd000080e800000041004a
:10daa4001040780002260200000000000100370048
:10dab400000000000080fa00000006000000fa00e8
:10dac400415f2900f2cabf000080fb00a2ae200023
:10dad4004200dd000080e8000000410010407800b2
:10dae40002260200000000000080fa000000060088
:10daf4000200fa00000f78001e00780001002000e8
:10db04003200200003002000820f5000838f580051
:10db14001d003e00006001000300370008003700cc
:10db24000d00370012003700a01680004d00de0003
:10db3400614060000080fb00000f78001400370093
:10db4400101680004700de00614060000080fb008a
:10db5400000f78000e003700a01680004700de009a
:10db6400614060000080fb00000f7800080037006f
:10db7400a01680004600de00614060000080fb00cb
:10db8400000f7800020037000000eb00000f78005f
:10db94009e0078000000eb00808f500002003200ed
:10dba400a05f290001003700d05f290080007800c1
:10dbb400f2cabf000080fb00a2ae20004200dd00dc
:10dbc4000080e800000041001040780002260200b6
:10dbd400000000000080fa00000006000200fa00c5
:10dbe400000f78001e007800010020007200200061
:10dbf40003002000820f5000838f580039003e003c
:10dc040000600100070037000c00370011003700e6
:10dc1400160037001b0037002000370025003700ae
:10dc24002a00370020168000004078006140600020
:10dc34000080fb00000f78002c00370020168000c5
:10dc44000000d100614060000080fb00000f7800fc
:10dc540026003700201680004200de00614060008c
:10dc64000080fb00000f78002000370020168000a1
:10dc74004300de00614060000080fb00000f78007c
:10dc84001a003700201680004400de006140600066
:10dc94000080fb00000f780014003700201680007d
:10dca4004500de00614060000080fb00000f78004a
:10dcb4000e003700201680004600de006140600040
:10dcc4000080fb00000f7800080037002016800059
:10dcd4004700de00614060000080fb00000f780018
:10dce400020037000000eb00000f78009e0078006f
:10dcf4000000eb00808f50000200320010c3b3001c
:10dd04000100370000c3b30021af20009140780028
:10dd14008180fb00a2ae2000c208dd008180e80003
:10dd24008100410011417800804078000240780071
:10dd340082240200000000000080fa0000000600b7
:10dd44000400fa00000f7800110798001e00780004
:10dd5400010020007200200003002000820f500008
:10dd6400838f580039003e0000600100070037002f
:10dd74000c00370011003700160037001b00370075
:10dd840020003700250037002a00370020168000c5
:10dd940000407800614060000080fb00000f7800c4
:10dda4002c003700201680000000d1006140600084
:10ddb4000080fb00000f780026003700201680004a
:10ddc4004200de00614060000080fb00000f78002c
:10ddd40020003700201680004300de006140600010
:10dde4000080fb00000f78001a0037002016800026
:10ddf4004400de00614060000080fb00000f7800fa
:10de040014003700201680004500de0061406000e9
:10de14000080fb00000f78000e0037002016800001
:10de24004600de00614060000080fb00000f7800c7
:10de340008003700201680004700de0061406000c3
:10de44000080fb00000f7800020037000000eb00a8
:10de5400000f78009e0090000000eb00808f5000bf
:10de6400040032009e0078000000eb00808f500018
:10de740008003a009e0090000000eb00808f5000e4
:10de84000e003a009e0078000000eb00808f5000e6
:10de94000a003a0001602900f2cabf000080fb00ba
:10dea400a2ae20004200dd000080e8000000410036
:10deb4001040780002260200000000000080fa00f2
:10dec400000006000a00fa0000188000000f780025
:10ded4000e80e800800078001e007800f0af020099
:10dee40000000000f2cabf000080fb00a1ae2000c9
:10def4004200dd000080e80000804000104078000f
:10df04008e80e80002260200000000000080fa0073
:10df1400000006000200fa00f2cabf000080fb0005
:10df2400a1ae20004200dd000080e8000080400037
:10df3400104078003024020000000000000f780038
:10df4400a2538000b35380006000b800800f5100da
:10df5400818f590058003a0000022000010020007f
:10df6400a0538800b153880053003700a2538000a7
:10df7400b35380000001200001002000800f5100f5
:10df8400818f59000c003a0091602900f2cabf0049
:10df94000080fb00a2ae20004200dd000080e8000b
:10dfa4000000410010407800620020002625020095
:10dfb400000000001e0f1000a0538000b153800029
:10dfc400020220000300200000005100818059005b
:10dfd40022e92000020040009040780000c2b30013
:10dfe40080cf50000c003200a0538000b153800059
:10dff400020220000300200000005100818059002b
:10e0040022e9200002004000904078000040eb002c
:10e0140080cf50000d003a0001612900f2cabf0010
:10e024000080fb00a2ae20004200dd000080e8007a
:10e034000000410010407800620020002625020004
:10e04400000000001e0f100013003700a0538000d2
:10e05400b1538000020220000300200000005100a0
:10e064008180590022e9200002004000904078009d
:10e07400f2cabf000080fb00a2ae20004200dd0017
:10e084000080e80000004100104078008224020073
:10e09400000000001e0f1000a2538000b353800044
:10e0a4000080eb008080eb00020040008380480089
:10e0b400a0538800b15388009e007800c00020005f
:10e0c400808f500006003600a2538000b3538000b6
:10e0d4006000b800800f5100818f5900a3ff3a00ff
:10e0e4000080fa00000006000200fa0070612900b6
:10e0f4008000780040a820009e5a02000000000022
:10e10400000f78009e0078000000eb00808f500024
:10e1140014003200c1612900f2cabf000080fb0074
:10e12400a2ae20004200dd000080e80000004100b3
:10e13400104078000226020000000000f2cabf006e
:10e144000080fb00a1ae20004200dd000080e8005a
:10e1540000804000104078009e00780002260200f3
:10e16400000000000080fa00000006000200fa002f
:10e17400706129008000780040a820009e5a0200a7
:10e1840000000000000f78009e0078000000eb0003
:10e19400808f50000b003200f2cabf000080fb00e9
:10e1a400a1ae20004200dd000080e80000804000b5
:10e1b400104078009e007800022602000000000053
:10e1c4000a00370041622900f2cabf000080fb0048
:10e1d400a2ae20004200dd000080e8000000410003
:10e1e4001040780002260200000000000080fa00bf
:10e1f400000006000200fa001000200001002000c8
:10e20400a0538800b1538800f2cabf000080fb000d
:10e21400a1ae20004200dd000080e8000080400044
:10e224001040780030240200000000009104200017
:10e23400810f50005e00360081ae200091407800ce
:10e2440030c0b30080cf50000e003200c1622900fc
:10e25400f2cabf000080fb00a2ae20004200dd0035
:10e264000080e8000000410010407800022602000f
:10e27400000000006000b800a0538800b15388007b
:10e284004c00370011642900f2cabf000080fb0073
:10e29400a2ae20004200dd000080e8000000410042
:10e2a4001040780002260200000000000040eb004d
:10e2b400004f7800350037009e4078000180fb0055
:10e2c400fc00400080a62000008040001040780040
:10e2d400e0b002000000000080407800f2cabf00f5
:10e2e4000080fb00a2ae20004200dd000080e800b8
:10e2f4000000410010407800822402000000000069
:10e304009e4078000180fb00fc00400080a62000b5
:10e31400008040001040780002b1020000000000bc
:10e3240080407800f2cabf000080fb00a2ae20004b
:10e334004200dd000080e800000041001040780049
:10e3440082240200000000009e4078000180fb004f
:10e35400e300600030002000808f50000a003a0083
:10e36400f2cabf000080fb00a1ae20004200dd0025
:10e374000080e800008040001040780001c2b30033
:10e3840082240200000000001e4fe8009e40780036
:10e39400f0c0b30080cf5000c7ff36006000b80063
:10e3a400a0538800b153880000000000010037002a
:10e3b400000000000080fa00000006000a00fa00d5
:10e3c40030079800410798000040eb00004f7800a8
:10e3d400220037009e4078000040eb0080cf5000c0
:10e3e4000a003200f2cabf000080fb00a1ae200088
:10e3f4004200dd000080e80000804000104078000a
:10e40400e1c2b30082240200000000009e407800b4
:10e414000180fb00e60047000080400010407800c7
:10e424000080fb008e00e800f0af02000000000056
:10e43400f2cabf000080fb00a1ae20004200dd0054
:10e444000080e80000804000104078008e00e80062
:10e4540002260200000000001e4fe8009e407800e3
:10e4640030c0b30080cf5000daff36000080fa00dd
:10e47400000006000000fa00f2cabf000080fb00a2
:10e48400a1ae20004200dd000080e80000804000d2
:10e4940010407800c1d420000226020000000000d1
:10e4a4000080fa00000006000000fa005ccdbf0006
:10e4b40002c4b300824060000040eb0080cf5000f3
:10e4c4000a00320071662900f2cabf000080fb0016
:10e4d400a2ae20004200dd000080e8000000410000
:10e4e4001040780002260200000000000080fa00bc
:10e4f400000006000000fa0002d320001241780058
:10e504008281fb0012d32000124178000281fb00bb
:10e514004811dd00030171000200780022d32000bd
:10e52400124178008281fb0032d32000124178002e
:10e534000281fb004811dd000301710082007800b4
:10e544009eff07000080fa00000006000000fa00a9
:10e5540082d32000124178008281fb0092d32000f4
:10e56400124178000281fb004811dd0003017100b3
:10e5740002007800a2d32000124178008281fb00bf
:10e58400b2d32000124178000281fb004811dd0063
:10e59400030171008200780088ff07000080fa0000
:10e5a400000006000000fa0042d320001241780067
:10e5b4008281fb0052d32000124178000281fb00cb
:10e5c4004811dd00030171000200780062d32000cd
:10e5d400124178008281fb0072d32000124178003e
:10e5e4000281fb004811dd00030171008200780004
:10e5f40072ff07000080fa00000006000000fa0025
:10e60400c2d32000124178008281fb00d2d32000c3
:10e61400124178000281fb004811dd000301710002
:10e6240002007800e2d32000124178008281fb00ce
:10e63400f2d32000124178000281fb004811dd0072
:10e6440003017100820078005cff07000080fa007b
:10e65400000006000000fa0002d4200012417800f5
:10e664008281fb0012d42000124178000281fb0059
:10e674004811dd00030171000200780022d420005b
:10e68400124178008281fb0032d4200012417800cc
:10e694000281fb004811dd00030171008200780053
:10e6a40046ff07000080fa00000006000200fa009e
:10e6b400f2cabf000080fb00a1ae20004200dd00d2
:10e6c4000080e80000804000104078003024020000
:10e6d4000000000011012000810f500005003e00e1
:10e6e4001000200001002000a0538800b1538800ce
:10e6f400400037000040eb00004f78003500370041
:10e704009e4078000040eb0080cf50000a003200a9
:10e71400f2cabf000080fb00a1ae20004200dd0071
:10e724000080e8000080400010407800a1c3b300de
:10e7340082240200000000009e4078000180fb005b
:10e74400c10220008080400010d3200000804000df
:10e7540010407800e0b00200000000008040780023
:10e76400f2cabf000080fb00a2ae20004200dd0020
:10e774000080e8000000410010407800822402007c
:10e78400000000009e4078000180fb00c1022000d0
:10e794008080400010d320000080400010407800aa
:10e7a40002b102000000000080407800f2cabf00fd
:10e7b4000080fb00a2ae20004200dd000080e800e3
:10e7c4000000410010407800822402000000000094
:10e7d4001e4fe8009e40780050c0b30080cf500028
:10e7e400c7ff36006000b800a0538800b15388000a
:10e7f400000000000080fa00000006000200fa0099
:10e80400000f78000080fa00000006000200fa0001
:10e81400000f78000080fa00000006000000fa00f3
:10e824000000fe000080fa00000006000000fa006c
:10e83400f2cabf000080fb00a1ae20004200dd0050
:10e844000080e800008040001040780041a82000cb
:10e8540002260200000000000080fa00000006000a
:10e864000000fa000080fa00000006000000fa0030
:10e874000080fa00000006000000fa000080fa00a0
:10e88400000006000200fa00000f78000080fa0081
:10e89400000006000000fa00f1662900f2cabf0079
:10e8a4000080fb00a2ae20004200dd000080e800f2
:10e8b4000000410010407800022602000000000021
:10e8c4000080fa00000006000000fa00f2cabf004f
:10e8d4000080fb00a1ae20004200dd000080e800c3
:10e8e4000080400010407800302402000000000046
:10e8f400a1042000810f500005003e0010002000fc
:10e9040001002000a0538800b15388000d00370097
:10e9140041672900f2cabf000080fb00a2ae2000bc
:10e924004200dd000080e800000041001040780053
:10e9340002260200000000006000b800a053880016
:10e94400b15388000080fa00000006000000fa00bd
:10e95400b1692900f2cabf000080fb00a2ae20000a
:10e964004200dd000080e800000041001040780013
:10e9740002260200000000000080fa0000000600e9
:10e984000000fa00016a2900f2cabf000080fb00ff
:10e99400a2ae20004200dd000080e800000041003b
:10e9a4001040780002260200000000000080fa00f7
:10e9b400000006000000fa00a15e80000000eb00e9
:10e9c400808f50000b003200016a2900f2cabf0098
:10e9d4000080fb00a2ae20004200dd000080e800c1
:10e9e40000004100104078000226020000000000f0
:10e9f4000a003700b1692900f2cabf000080fb0099
:10ea0400a2ae20004200dd000080e80000004100ca
:10ea14001040780002260200000000000000eb0015
:10ea2400a05e88000080fa00000006000000fa00e2
:10ea3400b15e80000000eb00808f50000b003200bc
:10ea4400016a2900f2cabf000080fb00a2ae2000c8
:10ea54004200dd000080e800000041001040780022
:10ea640002260200000000000a003700b1692900f4
:10ea7400f2cabf000080fb00a2ae20004200dd000d
:10ea84000080e800000041001040780002260200e7
:10ea9400000000000000eb00b05e88000080fa0077
:10eaa400000006000000fa00dccdbf00e240600078
:10eab4000040eb0080cf5000020032000000eb0069
:10eac400110037000040eb00dcedb700dc2da8009e
:10ead40010002000a06e88000000eb00d06e8800bb
:10eae4000000eb00b06e8800820120008000eb0083
:10eaf40060db2000a20a0200000000009001200058
:10eb0400606e8800100020000080fa0000000600fb
:10eb14000000fa00dccdbf00e24060000040eb00e2
:10eb240080cf500002003a000080eb001b00370049
:10eb3400a16e800020002000808f500002003a0067
:10eb440072c602000000000001fc20009140780021
:10eb5400e0cfb30080cf500005003200c0cfbf002b
:10eb64001a23020000000000e0cfb300c0efb7009a
:10eb7400dc2da9000000eb00a06e8800dccdbf00f6
:10eb8400e44060000040eb0080cf500002003200ff
:10eb94000000eb0001003700f06e80000080fa00f6
:10eba400000006000800fa00881f7800a06e8000ac
:10ebb400010020005200200003002000820f5000ba
:10ebc400838f580026063e000060010017063700b8
:10ebd40004003700be003700e3003700f7003700b9
:10ebe40009063700dccdbf00e84060000040eb00c0
:10ebf40080cf50000f0632005ac602000000000009
:10ec04008000eb00810f50000c063200b16d8000d3
:10ec14000000eb00808f500004003a00b16d8000ca
:10ec24000000eb00808f50000f003200506e800017
:10ec3400e10060000000eb00808f5000050032000e
:10ec4400b06d800011c0b3009cc60200000000003b
:10ec540097003700b06d800011c0b3009cc602005d
:10ec64000000000092003700e16d80000000eb001e
:10ec7400808f50000c003200506e8000e80060006d
:10ec84000000eb00808f500007003a00e06d800028
:10ec940001042000b00a020000000000b06d8800ea
:10eca400ca0da9000f003700e16d80000000eb00e1
:10ecb400808f50000b003200506e8000e80060002e
:10ecc4000000eb00808f500006003200e06d8000f1
:10ecd40001042000b00a020000000000b06d8800aa
:10ece400ca0da800b16d80000000eb00808f5000b9
:10ecf40023003a00b16d80000000eb00808f5000cb
:10ed04001f003a00f16d80000000eb00808f50007e
:10ed14000c003200506e8000f00060000000eb0038
:10ed2400808f500007003a00f06d8000010420003d
:10ed3400b00a020000000000b06d8800ca0da900ee
:10ed44000f003700f16d80000000eb00808f500051
:10ed54000b003200506e8000f00060000000eb00f9
:10ed6400808f500006003200f06d80000104200006
:10ed7400b00a020000000000b06d8800ca0da800af
:10ed8400b16d80000000eb00808f500025003a0038
:10ed9400b16d80000000eb00808f500021003a002c
:10eda400016e80000000eb00808f50000d003200e7
:10edb400516e800000022000808060000000eb00a3
:10edc400808f500007003a00006e8000010420008c
:10edd400b00a020000000000b06d8800ca0da9004e
:10ede40010003700016e80000000eb00808f50009f
:10edf4000c003200516e8000000220008080600010
:10ee04000000eb00808f500006003200006e80008e
:10ee140001042000b00a020000000000b06d880068
:10ee2400ca0da800b16d80000000eb00808f500077
:10ee34000b003a00b16d80000000eb00808f5000a1
:10ee440007003a0072c6020000000000000028001b
:10ee5400f06e88000000eb00a06e8800800537008b
:10ee6400506e8000e10060000000eb00808f5000d5
:10ee740008003200b06d80000000e800b06d88002a
:10ee8400b06d8000f1c0b3009cc602000000000019
:10ee940007003700b06d80000000e800b06d880006
:10eea400b06d8000f1c0b3009cc6020000000000f9
:10eeb4009a10020001000000006f8800116f8800a2
:10eec400a06e80000000e800a06e88006405370092
:10eed400e0dc2000cec60200000000008000eb0051
:10eee400810f500013003a009a1002000100000044
:10eef4000001be00006f8000116f8000000151000e
:10ef040081815900808d2b0051002000800f510019
:10ef1400818f59004b05360000002800f06e8800f0
:10ef24000000eb00a06e880072c602000000000022
:10ef34004b05370072c60200000000008000eb00a1
:10ef4400810f500005003a0000002800f06e880090
:10ef54000000eb00a06e880041053700a06e800021
:10ef64000000e800a06e8800626e8000706e800071
:10ef7400816e800094c0b3008201780032c0b30077
:10ef84007621020000000000c0efb70001fc200061
:10ef940091407800e0cfb30080cf50002b053200c1
:10efa400a06e80000000e800a06e88009a100200a5
:10efb40001000000006f8800116f8800c0cfbf00ff
:10efc400f6220200000000008000eb00810f5000d8
:10efd40018003a00dccdbf0002c2b30082406000da
:10efe4000040eb0080cf50000d003a009a10020060
:10eff400010000000001be00006f8000116f80005e
:10f0040000005100818059000001be0000122a0056
:10f0140071002000800f5100818f59000d053400cc
:10f0240010002800f06e880050002000a06e8800b8
:10f034000b053700dcada800d7003700c0cfbf00f8
:10f044008e80e800a026020000000000d06e800040
:10f05400010020005200200003002000820f500015
:10f06400838f5800cc003e0000600100050037008b
:10f0740004003700030037000b003700240037007a
:10f084002b003700d26e80002e40900041de20001d
:10f094008100410080487800d06e80000000e800c4
:10f0a400d06e8800bc0037002e4090000080fb002a
:10f0b40001022000810f500007003200d10220001d
:10f0c400810f500009003200d1002000810f500050
:10f0d4000b003200b0003700dc0da900d06e8000b8
:10f0e4000000e800d06e880008003700dc0da8009e
:10f0f400d06e80000000e800d06e88000300370066
:10f1040050002000d06e880000000000a2003700ec
:10f11400ae409000d0c0b30080cf500099003a00b8
:10f12400d06e80000000e800d06e88009a0037009e
:10f13400ae409000a0c0b30080cf500089003a00d8
:10f144000000eb00d06e8800dccdbf00e140600021
:10f154000040eb0080cf50008c003a000040eb00f0
:10f16400e7edb70040de2000420902000000000085
:10f17400f06e8800b06e800001002000c201200003
:10f1840003002000820f5000838f580073003e005c
:10f19400006001004b003700700037001a00370090
:10f1a4006e003700310037006c0037002f00370045
:10f1b4006a00370038003700680037004100370024
:10f1c40066003700650037003e00370063003700f3
:10f1d40062003700610037003a0037005f003700f3
:10f1e4005e0037005d003700360037005b003700f3
:10f1f4005a003700420037005800370057003700e4
:10f204005600370049003700f16e8000700c200072
:10f21400808f500012003600f16e8000b012200082
:10f22400808f50000e003e00c16d80000000eb0096
:10f23400808f500004003a00c16d80000000eb0094
:10f24400808f50000300320030002000b06e880030
:10f254000200370090002000b06e880002003700e2
:10f26400d0012000b06e88003d003700f16e8000b0
:10f27400e0142000808f500004003a00b06e80003b
:10f284000000e800b06e880002003700d0012000c2
:10f29400b06e880032003700f16e8000b00e20009e
:10f2a400808f500004003a00b06e80000000e80037
:10f2b400b06e880002003700d0012000b06e8800d4
:10f2c40027003700f16e8000700c2000808f500002
:10f2d40008003600f16e8000b0122000808f5000cc
:10f2e40004003e00b06e80000000e800b06e8800ac
:10f2f40002003700d0012000b06e880018003700eb
:10f30400f16e800020162000808f500004003a0027
:10f31400b06e80000000e800b06e88000200370084
:10f32400d0012000b06e88000d003700f16e80001f
:10f33400700c2000808f500005003600f16e8000b4
:10f34400b0122000808f500001003e00dc4da80068
:10f35400d0012000b06e88000100370000000000da
:10f364000d003700ae409000d0c0b30080cf5000f5
:10f3740008003200d06e80000000e900d06e8800e2
:10f384000500370000000000030037000000000003
:10f394000100370000000000c0cfbf006826020053
:10f3a400000000008000eb00810f500023ff3a00b2
:10f3b400c0cfbf003024020000000000f103200091
:10f3c400810f500025043600b06e80006101b80042
:10f3d4000080eb008080eb00020040008380480046
:10f3e400d201200003002000820f5000838f5800b8
:10f3f40003043e00006001001d00370000043700d4
:10f404002f003700fe03370038003700fc033700b5
:10f414008c003700fa033700e0003700f8033700a8
:10f424000601370030013700f50337006401370067
:10f434007f0137002c013700f1033700a7013700a3
:10f44400c201370028013700ed033700ec01370013
:10f4540008023700ea033700360337005a0337003f
:10f464006b033700e6033700cb033700cf033700c5
:10f47400c16d80000000eb00808f500005003a0051
:10f4840041df2900c0cfbf000226020000000000b7
:10f494000400370051e02900c0cfbf00022602005b
:10f4a40000000000c0cfbf000824020000000000dc
:10f4b400b06e80000000e800b06e8800d103370011
:10f4c40061e12900c0cfbf00022602000000000055
:10f4d400c0cfbf000824020000000000b06e80000e
:10f4e4000000e800b06e8800c6033700506e80004c
:10f4f400e20060000000eb00808f50000700320043
:10f50400c06d8000406f8800406f8000de0a0200fa
:10f5140000000000000f78003b003700c06d800041
:10f52400506f8800506f8000de0a02000000000067
:10f53400000f7800340037000040eb0020479800ab
:10f5440019003700506e8000e20060000000eb00fc
:10f55400808f5000090032002e4090000081fb0093
:10f56400416f800011407800e30147008071790009
:10f574000100e800406f8800080037002e4090002a
:10f584000081fb00516f800011407800e3014700c7
:10f59400807179000100e800506f88002e409000cf
:10f5a4000040e800204798002e4090008080fb0037
:10f5b4001e007800808f500004003100ae4090009f
:10f5c40020c0b30080cf5000deff36002e409000f4
:10f5d4000080fb001e0f10002e4090008080fb0076
:10f5e4006301470063004700430020009aae020015
:10f5f40000000000c0cfbf00e3004700420020002d
:10f6040026250200000000009e0078000000eb00a8
:10f61400808f5000c8ff3a0031e22900c0cfbf00fc
:10f624000226020000000000c0cfbf000824020030
:10f6340000000000b06e80000000e800b06e88009a
:10f6440070033700506e8000e40060000000eb009f
:10f65400808f500007003200d06d8000406f88001a
:10f66400406f8000de0a020000000000000f7800f6
:10f674003b003700d06d8000506f8800506f8000d1
:10f68400de0a020000000000000f7800340037009a
:10f694000040eb002047980019003700506e8000ae
:10f6a400e40060000000eb00808f5000090032008d
:10f6b4002e4090000081fb00416f800011407800d3
:10f6c400e3014700807179000100e800406f880081
:10f6d400080037002e4090000081fb00516f80002d
:10f6e40011407800e3014700807179000100e800cf
:10f6f400506f88002e4090000040e800204798009a
:10f704002e4090008080fb001e007800808f500007
:10f7140004003100ae40900020c0b30080cf500000
:10f72400deff36002e4090000080fb001e0f10000c
:10f734002e4090008080fb00630147006300470077
:10f74400430020009aae020000000000c0cfbf00ba
:10f75400e3004700420020002625020000000000cc
:10f764009e0078000000eb00808f5000c8ff3a0034
:10f7740031e22900c0cfbf000226020000000000d1
:10f78400c0cfbf000824020000000000b06e80005b
:10f794000000e800b06e88001a03370061e2290017
:10f7a400c0cfbf000226020000000000516e80009e
:10f7b40000042000808060000000eb00808f500077
:10f7c4000a003200106e8000c1de200047040700ea
:10f7d400406f8800626f8000416f8000c0cfbf001f
:10f7e400262502000000000009003700106e80008a
:10f7f400c1de2000d5030700506f8800626f8000cf
:10f80400516f8000c0cfbf00262502000000000019
:10f8140021e32900c0cfbf0002260200000000003f
:10f82400c0cfbf000824020000000000b06e8000ba
:10f834000000e800b06e8800f2023700e16d80003d
:10f844000000eb00808f500010003200506e8000ea
:10f85400e80060000000eb00808f50000b003a00cd
:10f86400e06d8000c1de2000b8030700506f8800ff
:10f87400616f80000000eb00808f500003003200b5
:10f88400c0002000b06e8800de023700e16d800009
:10f894000000eb00808f500010003200506e80009a
:10f8a400e80060000000eb00808f50000b00320085
:10f8b400e06d8000c1de20000c040700406f88006a
:10f8c400616f80000000eb00808f50000300320065
:10f8d400c0002000b06e8800ca023700f00020008b
:10f8e400b06e8800c702370061e32900c0cfbf00b3
:10f8f4000226020000000000506e8000e800600054
:10f904000000eb00808f500004003200b16e8000d4
:10f91400c0002000808f500013003200506e800021
:10f92400f00060000000eb00808f50000400320003
:10f93400b16e800000012000808f50000a00320068
:10f94400516e800000022000808060000000eb0007
:10f95400808f50000a003200b16e80004001200008
:10f96400808f500006003a00626f8000416f800073
:10f97400c0cfbf00262502000000000005003700ac
:10f98400626f8000516f8000c0cfbf002625020047
:10f994000000000021e32900c0cfbf0002260200be
:10f9a40000000000c0cfbf000824020000000000d7
:10f9b400b06e80000000e800b06e8800910237004d
:10f9c400506e8000e80060000000eb00808f500063
:10f9d40007003200416f8000606f800000804000ab
:10f9e400c1de2000c1030700406f88000600370015
:10f9f400516f8000606f800000804000c1de2000f5
:10fa040052030700506f8800616f80000000eb0014
:10fa1400808f500003003200c0002000b06e8800c8
:10fa240078023700b06e80000000e800b06e8800f5
:10fa3400f16d80000000eb00808f50001000320058
:10fa4400506e8000f00060000000eb00808f5000da
:10fa54000b003a00f06d8000c1de20003b0307007c
:10fa6400506f8800616f80000000eb00808f5000b1
:10fa74000300320000012000b06e880061023700ec
:10fa8400f16d80000000eb00808f50001000320008
:10fa9400506e8000f00060000000eb00808f50008a
:10faa4000b003200f06d8000c1de20008f030700e0
:10fab400406f8800616f80000000eb00808f500071
:10fac4000300320000012000b06e88004d023700b0
:10fad40030012000b06e88004a023700506e80006a
:10fae400f00060000000eb00808f5000070032003f
:10faf400416f8000606f800000804000c1de200004
:10fb04007a030700406f880006003700516f8000b9
:10fb1400606f800000804000c1de20000b030700fe
:10fb2400506f8800616f80000000eb00808f5000f0
:10fb34000300320000012000b06e8800310237005b
:10fb4400b06e80000000e800b06e8800016e800096
:10fb54000000eb00808f500011003200516e8000d5
:10fb640000022000808060000000eb00808f5000c5
:10fb74000b003a00006e8000c1de2000f302070093
:10fb8400506f8800616f80000000eb00808f500090
:10fb94000300320040012000b06e880019023700d3
:10fba400016e80000000eb00808f500011003200d5
:10fbb400516e800000022000808060000000eb0095
:10fbc400808f50000b003200006e8000c1de2000e8
:10fbd40046030700406f8800616f80000000eb005f
:10fbe400808f50000300320040012000b06e880076
:10fbf4000402370070012000b06e88000102370053
:10fc0400516e800000022000808060000000eb0044
:10fc1400808f500007003200416f8000606f8000c9
:10fc240000804000c1de200030030700406f8800e0
:10fc340006003700516f8000606f80000080400034
:10fc4400c1de2000c1020700506f8800616f800090
:10fc54000000eb00808f50000300320040012000c0
:10fc6400b06e8800e7013700b06e80000000e80045
:10fc7400b06e880001e42900c0cfbf000226020054
:10fc840000000000b06e80000000e800b06e880044
:10fc94000000eb00c06e8800c0cfbf000824020043
:10fca40000000000d7013700c06e80000100200072
:10fcb4009200200003002000820f5000838f580020
:10fcc4001e013e0000600100090037001a003700e1
:10fcd400390037004a0037006800370079003700e0
:10fce40097003700a8003700c7003700e10037004d
:10fcf400116e80000000eb00808f500004003a0079
:10fd0400116e80000000eb00808f5000070032006d
:10fd140010002000c06e880071e42900c0cfbf002d
:10fd24000226020000000000190137002000200014
:10fd3400c06e880016013700516e80000004200058
:10fd4400808060000000eb00808f50000d003200c6
:10fd5400116e8000c0cfbf00022602000000000028
:10fd6400106e8800106e8000904078000040eb0018
:10fd740080cf5000f3003a0020002000c06e8800bd
:10fd840003013700116e8000c0cfbf0002260200bd
:10fd940000000000106e8800106e80009040780013
:10fda4000040eb0080cf5000e8003a002000200023
:10fdb400c06e8800f6003700e16d80000000eb00a3
:10fdc400808f500004003a00e16d80000000eb00d9
:10fdd400808f50000700320030002000c06e880081
:10fde400e1e42900c0cfbf000226020000000000a9
:10fdf400e700370040002000c06e8800e4003700b0
:10fe0400506e8000e80060000000eb00808f50001e
:10fe14000d003200e16d8000c0cfbf000226020059
:10fe240000000000e06d8800e06d800090407800e4
:10fe34000040eb0080cf5000c6003a004000200094
:10fe4400c06e8800d2003700e16d8000c0cfbf00d3
:10fe54000226020000000000e06d8800e06d8000d2
:10fe6400904078000040eb0080cf5000bb003a0087
:10fe740040002000c06e8800c5003700f16d80008e
:10fe84000000eb00808f500004003a00f16d800008
:10fe94000000eb00808f500007003200500020006b
:10fea400c06e880051e52900c0cfbf0002260200c1
:10feb40000000000b600370060002000c06e88001b
:10fec400b3003700506e8000f00060000000eb00cb
:10fed400808f50000d003200f16d8000c0cfbf0054
:10fee4000226020000000000f06d8800f06d800022
:10fef400904078000040eb0080cf500099003a0019
:10ff040060002000c06e8800a1003700f16d800001
:10ff1400c0cfbf000226020000000000f06d880080
:10ff2400f06d8000904078000040eb0080cf5000de
:10ff34008e003a0060002000c06e880094003700f4
:10ff4400216e80000000eb00808f500004003a0016
:10ff5400216e80000000eb00808f5000070032000b
:10ff640070002000c06e8800c1e52900c0cfbf002a
:10ff740002260200000000008500370080002000f7
:10ff8400c06e880082003700516e80000008200097
:10ff9400808060000000eb00808f50000d00320074
:10ffa400216e8000c0cfbf000226020000000000c6
:10ffb400206e8800206e8000904078000040eb00a6
:10ffc40080cf50006b003a0080002000c06e880093
:10ffd4006f003700216e8000c0cfbf0002260200f0
:10ffe40000000000206e8800206e800090407800a1
:10fff4000040eb0080cf500060003a0080002000f9
:020000040001f9
:10000400c06e88006200370031e22900c0cfbf0013
:10001400220020002625020000000000316e80002e
:100024000000eb00808f500004003a00316e800025
:100034000000eb00808f500003003200900020008d
:10004400c06e88005200370031e22900c0cfbf00e3
:10005400220020002625020000000000a00020004d
:10006400c06e8800b06e80000000e800b06e8800aa
:1000740047003700516e800000102000808060002f
:100084000000eb00808f500015003200316e8000bc
:10009400c0cfbf000226020000000000306e8800be
:1000a400306e8000904078000040eb0080cf50001c
:1000b40034003a0031e22900c0cfbf002200200002
:1000c4002625020000000000a0002000c06e880069
:1000d400b06e80000000e800b06e88002c0037008d
:1000e400316e8000c0cfbf00022602000000000075
:1000f400306e8800306e8000904078000040eb0045
:1001040080cf500021003a0031e22900c0cfbf0067
:10011400220020002625020000000000a00020008c
:10012400c06e8800b06e80000000e800b06e8800e9
:100134001700370000000000150037000000000021
:100144001300370000000000110037000000000019
:100154000f003700000000000d0037000000000011
:100164000b00370000000000090037000000000009
:100174000700370000000000050037000000000001
:1001840003003700000000000100370000000000f9
:10019400c16e8000a0002000808f50000600320055
:1001a400c0cfbf0030240200000000000104200082
:1001b400810f5000bcfe3e00c0cfbf0008240200e7
:1001c400000000008f003700b06e80000000e800df
:1001d400b06e8800406e8000506f880080e6290071
:1001e400706f88000000eb00906e8800516f8000f3
:1001f4000000eb00808f500005003200506f80003b
:10020400e1e629000e0b020000000000906e880059
:10021400416e80000000eb00808f500004003a0023
:10022400416e80000000eb00808f50003f003200e0
:10023400706f8000904078000040eb0080cf500049
:100244004c00320027003700906e800063004000ad
:10025400906e8800586f8000906e80008000780057
:10026400506f80000080500000017800516f8000c2
:10027400c0cfbf002625020000000000000044009b
:10028400506f8800916e8000506f8000808f500006
:100294000b003a00c0cfbf00e1c2b30082240200c9
:1002a400000000008000eb00810f500008003a00bd
:1002b400906e800063005000906e88000d0037003f
:1002c400906e800063005000906e88000900370033
:1002d400506f8000e1e629000e0b020000000000d0
:1002e400906e8800916e80000000eb00808f5000bb
:1002f400d5ff3a00516f8000c0cfbf000226020034
:1003040000000000506f8800716f8000c0cfbf00f4
:100314000226020000000000706f8800c0cfbf00fa
:10032400082402000000000012003700dccdbf00ea
:10033400f04060000040eb0080cf50000d00320020
:10034400706f8000904078000040eb0080cf500038
:1003540008003200716f8000c0cfbf000226020087
:1003640000000000706f8800c0cfbf0008240200a6
:1003740000000000706f8000904078000040eb00a7
:1003840080cf500003003a00b06e80000000e80007
:10039400b06e88001b003700b06e80000000e800db
:1003a400b06e880020e72900406f8800406f80000d
:1003b400904078000040eb0080cf500008003200ed
:1003c400416f8000c0cfbf00022602000000000081
:1003d400406f8800c0cfbf00082402000000000066
:1003e400406f8000904078000040eb0080cf5000c8
:1003f40002003a0050002000a06e8800010037007f
:100404000000000016003700c0cfbf001a2302000e
:1004140000000000e0cfb300c0efb7000000eb0025
:10042400a06e8800000000000d00370000000000ee
:100434000b00370000000000090037000000000036
:10044400070037000000000005003700000000002e
:100454000300370000000000010037000000000026
:100464004f0478000080fa00000006000000fa0043
:10047400dc6da8000080fa00000006000000fa000d
:10048400a16e80000100ea00010070004f00de0050
:100494000080fa00000006000000fa00b16e80003f
:1004a400b0012000808f5000020032000000eb00f9
:1004b40003003700c0cfbf0030240200000000005a
:1004c4000080fa00000006000200fa00004f7800e5
:1004d400916e800030002000808f50000c003a00a4
:1004e400c0cfbf00e1c2b3008224020000000000bc
:1004f4008000eb00810f5000030032000000eb008d
:10050400906e8800020037000000eb0043003700c3
:10051400906e800011002000810f50000f00320007
:1005240011002000810f5000040039002100200038
:10053400810f5000190032002e0037009e407800d1
:10054400d0c0b30080cf500027003a00906e8000e6
:100554000000e800906e8800260037009e40780076
:10056400a0c0b30080cf500004003a00906e800019
:100574000000e800906e88001e0037009e4078005e
:10058400d0c0b30080cf500019003200906e8000bc
:100594000000e900906e880016003700e0c2b30046
:1005a4009e40780080cf500004003a00906e800096
:1005b4000000e800906e88000e0037009e4078002e
:1005c400d0c0b30080cf500004003a00906e800089
:1005d4000000e900906e8800060037000000eb0080
:1005e400906e88000300370000000000010037000f
:1005f40000000000c0cfbf009e40780082240200ab
:10060400000000008000eb00810f500002003a005f
:100614000000eb0001003700100020000080fa0009
:10062400000006000600fa00100798002107980051
:100634000000eb00000f78000f0037001e00900050
:10064400104078009e0090008100e8001107980097
:100654009dff07008000eb00810f50000200320074
:100664001e0fe800040037001e0090000000e9009f
:10067400100798000c0037002e0090008000ea005c
:100684002e009000008070004f00de008040780053
:100694002e0090000000e900200798000040eb00c5
:1006a40080cf5000e5ff3a001e0078000080fa0079
:1006b400000006000400fa00100798000000eb0098
:1006c400000f78000f0037001e00900010407800e3
:1006d4009e0090008100e800110798007aff07004f
:1006e4008000eb00810f5000020032001e0fe80072
:1006f400040037001e0090000000e9001007980075
:10070400050037001e009000904078000040eb0088
:1007140080cf5000ecff3a001e0078000080fa0001
:10072400000006000000fa00c0cfbf000824020049
:10073400000000000080fa00000006000000fa003b
:10074400dc8da8000080fa00000006000800fa0012
:1007540020079800310798002e009000000f7800c1
:100764003e0090008000eb00010878000040eb00a0
:100774003047980040003700ae409000c0c3b3003b
:1007840080cf500009003a003e4090000004a000d1
:1007940030479800ae009000010f78003e009000b2
:1007a4008080eb000108780007003700ae4090001d
:1007b40000c4b30080cf500003003a003e409000d4
:1007c4000014a000304798003e409000e1406000d3
:1007d4000040eb0080cf500010003a003e409000f3
:1007e400e24060000040eb0080cf50000b003a0074
:1007f400ae40900000c2b30080cf5000040032002d
:10080400ae409000c0c2b30080cf500003003a0055
:100814002e009000000f780017003700ae409000c3
:10082400c0c2b30080cf5000220032003e4090008e
:10083400e14060000040eb0080cf5000090032002e
:100844003e409000e24060000040eb0080cf50004a
:1008540004003200ae409000e0c3b30080cf5000eb
:10086400160032003e009000100078008000e8007e
:100874003e009000010878002e009000904078001f
:10088400214798002e4090000080fb000000ea0001
:100894004f00de00804078002e0090000000e80049
:1008a400200798000040eb0080cf5000b2ff3a00d0
:1008b40003003700000000000100370000000000c2
:1008c4003e409000e24060000040eb0080cf5000ca
:1008d40003003a003e0090008000eb00010878001d
:1008e4001e0078000080fa00000006000800fa00ec
:1008f40020079800310798002e009000000f780020
:100904003e0090008000eb00010878000040eb00fe
:100914003047980040003700ae409000c0c3b30099
:1009240080cf500009003a003e4090000004a0002f
:1009340030479800ae009000010f78003e00900010
:100944008080eb000108780007003700ae4090007b
:1009540000c4b30080cf500003003a003e40900032
:100964000014a000304798003e409000e140600031
:100974000040eb0080cf500010003a003e40900051
:10098400e24060000040eb0080cf50000b003a00d2
:10099400ae40900000c2b30080cf5000040032008b
:1009a400ae409000c0c2b30080cf500003003a00b4
:1009b4002e009000000f780017003700ae40900022
:1009c400c0c2b30080cf5000220032003e409000ed
:1009d400e14060000040eb0080cf5000090032008d
:1009e4003e409000e24060000040eb0080cf5000a9
:1009f40004003200ae409000e0c3b30080cf50004a
:100a0400160032003e009000100078008000e800dc
:100a14003e009000010878002e009000904078007d
:100a2400214798002e4090000080fb000000ea005f
:100a34004f00de00804078002e0090000000e800a7
:100a4400200798000040eb0080cf5000b2ff3a002e
:100a54000300370000000000010037000000000020
:100a64003e409000e24060000040eb0080cf500028
:100a740003003a003e0090008000eb00010878007b
:100a84001e0078000080fa00000006000400fa004e
:100a9400d7c2a800d3c2a9000000eb00001288004e
:100aa400b0012000101288000000eb002012880022
:100ab4004302a80042a2a80041e2a8003f050700a3
:100ac4000e80e800d1c1b300590507002e40900004
:100ad400004f78009e4078000180fb00e800600031
:100ae4000000eb00808f5000f4ff3a009e40780035
:100af4000180fb00e10060000000eb00808f5000eb
:100b0400eeff320010002000e07b88000000eb00c4
:100b1400c07b88008040eb0080c0b300cd05070097
:100b24008040eb0090c0b300ca05070091ccb3002d
:100b3400c0c0b300c705070091c0b300d0c0b30064
:100b4400c405070091ccb300a0c0b300c1050700e1
:100b540091c0b300b0c0b300be050700a1ccb30080
:100b640040c0b300bb05070091c0b30050c0b30040
:100b7400b8050700a1ccb30020c0b300b505070039
:100b840091c0b30030c0b300b20507000040eb00d1
:100b940074040700002020004a060700d1c0b300f7
:100ba4000040eb00ab05070021c3b30020c0b30035
:100bb400a805070021c1b30040c0b300a505070084
:100bc40001c4b30030c0b300a2050700f1c3b300f1
:100bd40090c0b3009f05070021c1b30060c0b300fb
:100be4009c050700c1c0b30070c0b300990507009d
:100bf400e1ceb300a0c0b3009605070051c0b30016
:100c0400b0c0b30093050700403020002d06070054
:100c14005dcdbf008040780040c0b3008d05070063
:100c24005ecdbf008040780050c0b3008905070046
:100c34005fcdbf008040780020c0b3008505070069
:100c440060cdbf008040780030c0b300810507004c
:100c540061cdbf00804078000040eb007d050700b7
:100c640062cdbf008040780010c0b3007905070052
:100c74008040eb0050c1b300760507000e00e80089
:100c840021c1b300ea0407001e4090007eefb700c4
:100c94000110200000c1b300e9050700214723002b
:100ca40040c1b300e60507008000eb000040eb0004
:100cb400e30507000000eb000206070041c0b30093
:100cc400f0c1b300b50507000080fa00000006007b
:100cd4000200fa0011c0b3000e0078002f050700cf
:100ce4001e0078004200de00614060000080fb00ce
:100cf4000080fa00000006000200fa00f1c1b3000f
:100d04000e007800ca0407001e40780068406000a6
:100d14000080fb000000e9004f00de000080fa00c4
:100d2400000006000200fa00e17b80000000eb00f6
:100d3400808f500017003a0010002000e07b8800ec
:100d4400c07b80000000e900000f78009e0078005e
:100d5400909c2000808f500002003600909c200060
:100d6400000f780001c4b300e0c1b3008b05070095
:100d74001e40780080407800c0c0b30035050700ed
:100d84001e40900080407800d0c0b30031050700b9
:100d940001003700000000000080fa000000060097
:100da4000a00fa0090112000c605070065004700fc
:100db40091c1b3009e0407005e4090006047980014
:100dc400e0002000bf05070064004700e1c0b30055
:100dd400970407004e409000004f980063004700be
:100de400f1c0b300920407003e409000104f9800f9
:100df40090112000b30507000e80e80091c1b300f4
:100e04008b040700ae4090006e40900080cf5000ed
:100e1400e6ff3a00c0002000aa0507000e00e80023
:100e2400c1c0b300820407001e40900060479800d0
:100e3400d1c0b3000e0078007d0407001e40780086
:100e440070479800ce0090003e009000808f5000c4
:100e540006003600be0090004e00900080805000d6
:100e6400909c2000008040000a003700ce009000d3
:100e74003e009000808f500002003a00909c2000b9
:100e840004003700be0090004e0090000080500027
:100e94000000e9000080fa00000006001a00fa00d1
:100ea400300f9800410f980090112000850507002d
:100eb4000e00e80091c1b3005d0407001e409000dd
:100ec400004f78000000eb007e0507009e4078008c
:100ed4000040eb0080cf500002003a000000eb001d
:100ee40061003700e17b80000000eb00808f500040
:100ef40003003a008bff07000000eb005a003700a4
:100f0400c07b8000d07b88007acfbf00804078000f
:100f14000040eb00cf0407007bcfbf008040780087
:100f240010c0b300cb0407000e80e800410120008c
:100f3400110307000e80e80010089000bab1020007
:100f4400000000008e80e800900898000e80e80001
:100f540090007800909c2000808f50001f003e007d
:100f64000e80e80010407800e14060000040eb0093
:100f740080cf500019003a000e80e800a0009000d5
:100f840000002800808060000000eb00808f50008b
:100f940012003a000e80e80020009000f00060008b
:100fa4000000eb00808f50000c003a000e80e80037
:100fb40090009000e05e2000808f500007003e000b
:100fc4000e80e800a00090000008200080806000ef
:100fd4000000eb00808f500001003a000000fe008a
:100fe4000e80e80010007800c07b88003e08900066
:100ff4008e80e800ec80400062002000940a020029
:1010040000000000ce08900000c0eb00804878008b
:101014000e80e800b050900080c0b30080cf500034
:101024000e003a000e80e800a05090000040eb0053
:1010340080cf5000050032000e80e800a0509000e0
:1010440060c0b30080cf500004003a000e80e80076
:1010540020509000ce089000804878000000eb00fb
:10106400e07b8800100020000080fa0000000600e9
:101074000600fa00000f7800214798002207980024
:10108400b1ccb30020c0b3007204070091c0b30018
:1010940030c0b3006f040700ae009000809d2000b4
:1010a400008040002007980064004700104078004a
:1010b4008040780060c0b300660407006400470005
:1010c400104090008040780070c0b30061040700b5
:1010d4001e0078006100200040030700610020002a
:1010e400d0d520003d03070080c0b3001d030700d6
:1010f400ae4090000040eb0080cf500002003a0068
:101104000040eb000100370060c0b3001503070086
:101114000080fa00000006001800fa0001c8b300bd
:10112400f0c1b3009d04070001c8b300f0c1b300cf
:1011340071040700a1c0b300c0c1b3006e0407006e
:1011440081c0b300f0c1b30094040700e1f72000ac
:101154009140780050c0b30080cf500005003200a9
:10116400e1f720009140780060c0b30080cf5000c8
:1011740087003a000000eb00000f78000000000038
:101184006a004700c1c1b300a90307002e489000bc
:101194000080fb00ea0060000000eb00808f50003c
:1011a40005003a001e0fe800703e20009e00780003
:1011b400808f5000f2ff360069004700c1c1b300c0
:1011c4009b0307001e489000e24060000040eb00d3
:1011d40080cf500004003a00703e20009e0078004a
:1011e400808f50006a00360081c0b300f0c1b300a4
:1011f40041040700680047008040eb008c030700af
:101204000e489000404f98006700470011c0b3009b
:10121400870307007e409000504f98006600470007
:1012240061c0b300820307006e409000604f9800d5
:101234006500470071c0b3007d0307005e40900065
:10124400704f98007e0090000000e800700798003e
:101254006e489000804078000040eb00fd030700da
:101264007e4890008040780010c0b300f903070066
:1012740070004700810020003f0207000040eb009f
:10128400204798003600370064004700c1c1b3000e
:10129400670307004e409000e24060000040eb000e
:1012a40080cf500032003200700047009000900060
:1012b40000002200808060000000eb00808f50005e
:1012c4002b00320001c8b300f0c1b300330407009f
:1012d40001c8b300f0c1b30007040700a1c0b30004
:1012e400c0c1b3000404070081c0b300f0c1b3005f
:1012f4002a0407000000000063004700c1c1b300d6
:101304004b0307003e4090000080fb00ea006000b1
:101314000000eb00808f5000f7ff320081c0b30063
:10132400f0c1b300f40307006e48900080407800d9
:101334000040eb00c70307007e489000804078001f
:1013440010c0b300c30307007000470081002000f1
:10135400090207002e4090000040e8002047980052
:10136400ae409000f0c0b30080cf5000c6ff3600fe
:101374004e489000804078000040eb00b503070021
:101384005e4890008040780010c0b300b1030700ad
:101394000080fa00000006000400fa00100798001c
:1013a400d17b80001e00900000804000740040004b
:1013b400000f78009e007800909c2000808f5000e1
:1013c400040036009e00780060632f000080400017
:1013d400000f78001e407800804078000040eb0049
:1013e4009c0307001e4090008040780010c0b300aa
:1013f400980307000080fa00000006000600fa00c7
:10140400200798000e00e80021c0b300080307007d
:101414001e4090002047980031c0b3000e007800b1
:10142400030307001e40780030479800640047001b
:10143400104078008040780020c0b3008503070086
:1014440064004700104090008040780030c0b30032
:10145400800307001e0090000080fa0000000600d0
:101464000600fa00200798000e00e8008040eb0018
:10147400ef0207001e4090002047980011c0b300ff
:101484000e007800ea0207001e40780030479800fa
:101494006400470010407800804078000040eb0072
:1014a4006c030700640047001040900080407800ff
:1014b40010c0b300670307001e0090000080fa000c
:1014c400000006000a00fa0030079800410798005f
:1014d400d17b80003e0090000080400074004000fa
:1014e400100798009e009000909c2000808f500070
:1014f400040036009e00900060632f0000804000ce
:10150400100798000e00e8008040eb00c8020700b6
:101514001e4090004047980011c0b3000e007800b0
:10152400c30207001e407800504798002e409000e8
:10153400804078000040eb00460307003e409000e6
:101544008040780010c0b300420307004e009000b2
:101554000c000700100798004e409000804078006f
:101564000040eb003b0307005e40900080407800a1
:1015740010c0b300370307001e0090000080fa007b
:10158400000006002200fa00001798006000b8006e
:101594003007980041079800630047008040eb0043
:1015a400a30207003e409000404798000e80e800e8
:1015b40011c0b3009e0207002e40900050479800cf
:1015c4002e0037000e10900041012000810f5000c2
:1015d400010036004001200050079800de00900012
:1015e4006c004700640107005e0090008e109000bc
:1015f40000805000001798006a004700100078002f
:10160400e10060000000eb00808f50000800320011
:10161400ec0047005e009000808040000040eb003a
:10162400804878005e0090000000e80050079800b1
:101634006c0f47000d0037003e019000ce01900072
:101644001e00780010007800010020000200400015
:101654008380480030079800410798001e8fe800f7
:101664005e0090000080e90050079800de009000c2
:101674000000eb00808f5000efff3a008e109000c6
:101684000000eb00808f5000ceff3a004e409000e7
:10169400804078000040eb00ee0207005e409000be
:1016a4008040780010c0b300ea0207003e009000ba
:1016b4006101b8004e0090000100200002004000cb
:1016c400838048003007980041079800be009000ce
:1016d4004e00900000804000300798003e009000cb
:1016e4000080ea000080fa00000006001800fa00fa
:1016f400881f7800100f9800210f9800320f98006f
:101704000000eb00000f78000000eb0010079800c9
:101714009e0890000080eb00808f50000f003a007c
:1017240010002000000f78006c00470021c0b300b7
:101734003f0207004e4890000080fb00100f980005
:10174400720047000004e8006b00470031c0b3009a
:10175400370207003e489000004c7800ae08900025
:101764000080eb00808f50000f003a001000200032
:10177400100798006a0047008040eb002c02070025
:101784002e4890000080fb00200f98007400470052
:101794000004e8006900470011c0b30024020700f8
:1017a4001e489000004c7800be08900010002000f5
:1017b400808f500058003e009e0090000000eb0017
:1017c400808f50000a003a00680047008040eb0018
:1017d400170207000e489000604f9800670047000a
:1017e40011c0b300120207007e409000704f9800b1
:1017f4009e0078000000eb00808f50000a003a0041
:101804006600470021c0b300090207006e40900043
:10181400005798006500470031c0b3000402070078
:101824005e40900010579800740047001040780004
:10183400804078000040eb008602070074004700f7
:101844000000e800104078008040780010c0b30029
:101854008002070072004700104078008040780042
:1018640020c0b3007b020700720047000000e800bc
:10187400104078008040780030c0b3007502070043
:1018840002003700a2000700360107003e0890005e
:101894008000ea0080807000cf08de00814078007c
:1018a4000000e900300f98000040eb0080cf5000aa
:1018b400f4ff3a009e0090000000eb00808f50007f
:1018c40008003a006e489000804078000040eb0029
:1018d400600207007e4890008040780010c0b3008a
:1018e4005c0207009e0078000000eb00808f50002f
:1018f40079003a000e5090008040780020c0b30078
:10190400540207001e5090008040780030c0b3009d
:1019140050020700700037009e0078000000eb00c2
:10192400808f50000c0032009e0890003e0890000a
:1019340000804000000f98000e5090008040780016
:1019440020c0b300430207001e509000804078007e
:1019540030c0b3003f020700ae0890003e0890007c
:10196400008040000000e900300f980000000000f3
:1019740064004700f1c1b300ad0107004e40900080
:1019840002c2b300824060000040eb0080cf5000f0
:10199400f7ff3a0074004700104078008040780058
:1019a40000c1b3002b020700740047000000e800e8
:1019b400104078008040780010c1b3002502070071
:1019c40072004700104078008040780040c1b300a6
:1019d40020020700720047000000e8001040780071
:1019e4008040780050c1b3001a020700ae0890008e
:1019f400909c2000808f500008003e00be0890009c
:101a0400909c2000808f500004003600be08900097
:101a140060632f0000804000300f9800760047007c
:101a2400104078008040780020c1b300090207000c
:101a3400760047000000e8001040780080407800fd
:101a440030c1b3000302070001c1b300f0c1b30009
:101a54002902070001c2b300f0c1b3004f0207001e
:101a64009e0090000000eb00808f50001a003200ae
:101a74003e0890000000e800300f9800ae08900087
:101a8400909c2000808f500008003e00be0890000b
:101a9400909c2000808f500004003600be08900007
:101aa40060632f0000804000300f980076004700ec
:101ab40010407800804078000040eb00e50107000a
:101ac400760047000000e80010407800804078006d
:101ad40010c0b300df0107004f0478000080fa0053
:101ae400000006000200fa00f1c1b3000e00780005
:101af4004f0107001e4078000042b2000080fb0046
:101b04000000e9004f00de000080fa00000006003b
:101b14000200fa00d7c2a90041e2a9004342a8008a
:101b240041e2a80000a023004012880000128000b7
:101b3400e20060000000eb00808f5000fbff3a00e1
:101b440000128000e10060000000eb00808f500074
:101b5400f6ff320041e2a9004342a90041e2a80095
:101b640040128000004f7800d7c2a8001e407800c1
:101b74000080fa00000006000a00fa00300798000e
:101b840041079800d7c2a900a00320004012880092
:101b94000000eb00000f7800be0090000000eb0096
:101ba400808f5000030032003e0090000000e900e6
:101bb4003007980000128000e20060000000eb0093
:101bc400808f5000fbff3a0000128000e1006000ab
:101bd4000000eb00808f5000f6ff320040128000be
